:100000000C94040F0C94350F0C94350F0C94350F91
:100010000C94350F0C94350F0C94350F0C94350F50
:100020000C94350F0C94350F0C94350F0C94350F40
:100030000C94350F0C94D9700C94350F0C94350F2B
:100040000C94350F0C94350F0C94350F0C94350F20
:100050000C94350F0C94350F0C94350F0C943E6DA9
:100060000C94350F0C94BCD20C9492D20C94350F96
:100070000C94350F0C94350F0C94350F0C94350FF0
:100080000C94350F0C94350F0C94350F0C94350FE0
:100090000C9468D20C943ED20C94350F0C9464727C
:1000A0000C94350F0C94350F0C94350F0C94350FC0
:1000B0000C94350F0C94350F0C94350F0C94350FB0
:1000C0000C94350F0C94350F0C94350F0C9414D2FE
:1000D0000C94EAD10C94350F0C94C0D10C9496D1A9
:1000E0000C94350F084AD73B3BCE016E84BCBFFD54
:1000F000C12F3D6C74319ABD56833DDA3D00C77FF8
:1001000011BED9E4BB4C3E916BAAAABE0000008090
:100110003F07634236B79BD8A71A39685618AEBA5C
:10012000AB558C1D3CB7CC5763BD6DEDFD753EF6F0
:10013000177231BF000000803F08000000BE92240B
:1001400049123EABAAAA2ABECDCCCC4C3E00000040
:1001500080BEABAAAAAA3E00000000BF000000803B
:100160003F0000000000084178D3BB4387D1133D16
:10017000190E3CC3BD4282AD2B3E68EC8276BED9DF
:100180008FE1A93E4C80EFFFBE01C4FF7F3F00001E
:10019000000000000C9412590C9467570C94AED3D5
:1001A0000C949C5C0C94CE600C94444D0C94EAD35B
:1001B0000C94C36A0C948A6D0C94F14D0C949E6B54
:1001C0000C94A16A0C9493500C942A4D0C941D6BC2
:1001D0000C941E610C941A6B0C94815F0C94EDA925
:1001E0000C94FB4C0C944BA90C94C76A0C94BD73F3
:1001F0000C9482AB0C944CA90C94D9A90C94A850E3
:100200000C94EC6A0C943B4D0C94A76A0C944D4DE5
:100210000C942C6B0C948C550C947B520C948C6A23
:100220000C94926A0C94F24C0C947B500C94B96A26
:100230000C94CFAB0C94CC6A0C94D84C0C94C35A4D
:100240000C94C4530C9418510C94FA4D0C949F5078
:100250000C941C6B0C94B9610C9496500C94D36064
:100260000C94F5510C94396A0C94CD6A0C946C6B17
:100270000C94C3A90C94E3A90C94A1A90C94E14C8F
:100280000C94AB6A0C94B36C0C9416590C94886063
:100290000C94FF5E0C9413510C9463580C94A5506D
:1002A0000C94B14C0C94D16A0C94426C0C94895F00
:1002B0000C94CB530C94B7580C94B5A90C94CFA9BB
:1002C0000C94A2500C941B6B0C94805C0C9492A91F
:1002D0000C94E9600C943F6B0C947D510C94C64CCB
:1002E0000C946C570C9453510C94335E0C949A6A92
:1002F0000C94154E0C94CC580C9484510C94966A22
:100300000C949E6A0C948A510C943F560C940C4E9B
:100310000C9499500C94B16A0C94CF4C0C9490505E
:100320000C94D0580C94BF6A0C94736C0C941661A6
:100330000C949B6B0C94B56A0C949C500C94034EDB
:100340000C94C9600C94564D0C94C85D0C941A4CD6
:100350004E414E494E495459494E46CDCCCC3D0AAA
:10036000D7233C17B7D13877CC2B329595E6241F8D
:10037000B14F0A000020410000C84200401C462046
:10038000BCBE4CCA1B0E5AAEC59D7400407A10F319
:100390005A00A0724E18090010A5D4E80000E876B3
:1003A00048170000E40B54020000CA9A3B0000000A
:1003B000E1F505000080969800000040420F000023
:1003C00000A08601000000102700000000E80300E4
:1003D0000000006400000000000A000000000001AE
:1003E00000000000002C76D888DC674F0823DFC1AE
:1003F000DFAE59E1B1B796E5E3E453C63AE6519969
:100400007696E8E6C28426EB898C9B62ED407C6F91
:10041000FCEFBC9C9F40F2BAA56FA5F490055A2A48
:10042000F75C936B6CF9676DC11BFCE0E40D47FE54
:10043000F520E6B500D0ED902E0300943577050049
:1004400080841E080000204E0A000000C80C3333D0
:1004500033330F986E12831141EF8D2114893BE6DF
:100460005516CFFEE6DB18D1844B381BF77C1D9068
:100470001DA4BBE424203284725E228100C9F124D1
:10048000ECA1E53D274D4D43353838334D413D20F6
:1004900000482D6669656C643A20280020202020E1
:1004A000202020202020202020202020002020206C
:1004B000202020202020202020202020200020205C
:1004C000202020202020202020202020202000204C
:1004D000202020202020202020202020202020003C
:1004E000202020202020202020202020202020002C
:1004F000202020202020202020202020202020001C
:1005000044233A43616C6962726174696F6E00449E
:100510002A3A53657474696E67730044423A5265AF
:10052000736574204C6F676765720044433A436C8F
:10053000656172204C43440043303A416D6D6F6EEB
:1005400069610043393A4E697472617465004338D9
:100550003A466F7263652F4D6173730043373A43B8
:100560006F6E6475637469766974790043363A44D2
:100570006973736F6C766564204F320043312D359B
:100580003A536C6F74312D35204F6E0044443A4D10
:10059000756C746953656E736F72730044393A43B6
:1005A000757272656E7400566F6C746167652B436B
:1005B000757272656E740044383A456C6563747286
:1005C00069630044373A4D6F74696F6E0044363A80
:1005D00044532054656D700044353A555620496E99
:1005E00074656E736974790044343A4F3220636FD6
:1005F0006E632E0044333A434F3220636F6E632E96
:100600000044323A504D28313A322E353A313029B1
:100610000044323A504D28313A322E353A313029A1
:100620002A0044313A5475726269646974790044ED
:10063000303A566F6C7461676500393A6F722033D7
:100640004420616363656C2E00393A496E636C2EF9
:1006500020616E672E00383A70482076616C7565AF
:1006600000373A49522054656D7000373A4952209C
:1006700054656D702A00363A4D61676E6574696322
:10068000206669656C6400353A476173204C657675
:10069000656C00343A495220466C616D6500333A0E
:1006A0004C6967687420496E742E00323A616E643A
:1006B0002048656967687400323A54656D7020504F
:1006C0007265737375726500313A54656D702048B8
:1006D000756D696469747900303A536F756E642082
:1006E0004C6576656C00303A536F756E64204C65CE
:1006F00076656C2A0054696D65206C617073653A8B
:1007000000576946692049503A0023756E6B6E6F39
:10071000776E00236E6F20616D6D6F6E6961206C66
:1007200069622100236E6F206E69747261746520A6
:100730006C69622100456E61626C6520776974683E
:1007400020442300466F7263652053656E736F7299
:1007500000234E65656420746F20656E61626C6570
:1007600020262063616C69627261746520666F7215
:1007700063652073656E736F72004E6F74206361E2
:100780006C69627261746564004543206572720031
:10079000234E65656420746F2063616C69627261C9
:1007A00074652045432070726F6265002350726546
:1007B000737320442320746F20656E61626C652022
:1007C0000050686F6E652053656E736F72004163F1
:1007D00063656C65726174696F6E004F7269656EF6
:1007E000742E2F496E636C2E00416E672E20566565
:1007F0006C6F6369747900436F6D702E20262048FA
:100800002D6669656C64004750530050726F7869BB
:100810006D697479004C6967687420496E74656EFF
:1008200073697479004169722050726573737572CF
:10083000650054656D7020262048756D6964697483
:1008400079004D6F74696F6E00555620496E742E95
:1008500000555620496E74656E73697479004F3285
:1008600020436F6E6300434F3220436F6E6300532B
:10087000656E736F72206572726F722100234E6F06
:100880002073656E736F722100434F3220436F6E89
:1008900063004D6561737572696E6700234E6F204A
:1008A00054422073656E736F723F00234E6F207346
:1008B000656E736F722100536F756E64204C6576A0
:1008C000656C004D6561737572696E672E2E00232D
:1008D0004E6F2073656E736F722100536F756E6477
:1008E000204C6576656C00234E6F2073656E736FC8
:1008F0007220666F722074656D7020262068756D99
:10090000696469747921004E6F2053656E736F724C
:10091000210020666F722074656D70202620687536
:100920006D696469747921002353656E736F722059
:100930004572726F72200053656E736F722045723C
:10094000726F7221002357726F6E672073656E732A
:100950006F7220666F722074656D70202620687536
:100960006D6964697479210057726F6E67205365F1
:100970006E736F72210054656D702048756D6964E7
:10098000697479004C6967687420496E74656E7388
:1009900069747900466C616D6520495200482D6686
:1009A00069656C64005365617263682044697265AF
:1009B0006374696F6E00234E6F2070482073656EFC
:1009C000736F72210070482076616C756500234951
:1009D0006E76616C6964206B65792100204D756CC1
:1009E000746973656E736F7273004D756C7469739F
:1009F000656E736F72730044697361626C65004564
:100A00006E61626C65005265626F6F74696E672E0D
:100A10002E2E002344413A2D323300237265706C30
:100A20006965733D0067657453656C6654657374DE
:100A300042697428293A20006973496E746572729C
:100A4000757074456E61626C65642831293A2000C6
:100A5000676574496E746572727570744D617070FB
:100A6000696E672831293A2000676574496E74659C
:100A70007272757074536F757263652831293A20EC
:100A800000676574496E74657272757074536F7522
:100A900072636528293A200067657452617465287D
:100AA000293A20332E31343135393F006163636593
:100AB0006C2E69734C6F77506F77657228293A20D6
:100AC00000616363656C2E697341736C65657028A2
:100AD000293A2000616363656C2E69735461705319
:100AE0006F757263654F6E5A28293A2000616363FF
:100AF000656C2E6973546170536F757263654F6EC8
:100B00005928293A2000616363656C2E697354612A
:100B100070536F757263654F6E5828293A200061D3
:100B20006363656C2E697341637469766974795384
:100B30006F757263654F6E5A28293A2000616363AE
:100B4000656C2E69734163746976697479536F7546
:100B50007263654F6E5928293A20006973416374A6
:100B60006976697479536F757263654F6E58282979
:100B70003A20006973546170446574656374696FE9
:100B80006E4F6E5A28293B2066616C73653F2000CA
:100B90006973546170446574656374696F6E4F6EF8
:100BA0005A28293B20747275653F2000697354618F
:100BB00070446574656374696F6E4F6E5928293B84
:100BC0002066616C73653F200069735461704465F1
:100BD00074656374696F6E4F6E5928293B20747277
:100BE00075653F2000697354617044657465637472
:100BF000696F6E4F6E5828293B2066616C73653FA4
:100C000020006973546170446574656374696F6E24
:100C10004F6E5828293B20747275653F2000676528
:100C200074537570707265737342697428293B2020
:100C300066616C73653F20006765745375707072F0
:100C400065737342697428293B20747275653F206F
:100C50000069734163746976697479416328293A3C
:100C600020006973496E61637469766974795A45C5
:100C70006E61626C656428293A20006973496E616F
:100C80006374697669747959456E61626C6564282C
:100C9000293A20006973496E6163746976697479D1
:100CA00058456E61626C656428293A200069734179
:100CB000637469766974795A456E61626C656428FB
:100CC000293A2000697341637469766974795945DA
:100CD0006E61626C656428293A200069734163740F
:100CE000697669747958456E61626C656428293A41
:100CF00020006765744672656546616C6C44757268
:100D00006174696F6E28293A2000676574467265C0
:100D10006546616C6C5468726573686F6C642829F1
:100D20003A200067657454696D65496E6163746942
:100D30007669747928293A2000676574496E616381
:100D40007469766974795468726573686F6C642825
:100D50002920006765744163746976697479546801
:100D6000726573686F6C6428292000676574446F2E
:100D700075626C6554617057696E646F77282920BD
:100D800000676574446F75626C655461704C617482
:100D9000656E637928293A20006765745461704450
:100DA00075726174696F6E28293A20006765744115
:100DB0007869734F66667365742826782C202679C7
:100DC0002C20267A293A2000676574546170546893
:100DD000726573686F6C6428293A200058595A204C
:100DE00047733A200058595A20434F554E54533AAE
:100DF0002000736574206761696E735B5D3A002043
:100E00006661696C656400207375636365737366FE
:100E1000756C00236761696E735F6F7269675B5DF4
:100E20003A00234C3347343230304420636F6E6EC7
:100E3000656374696F6E00756E6B6E6F776E0032EE
:100E400030303020647073003530302064707300AF
:100E50003235302064707300236779726F207363BA
:100E6000616C653D00234E6F204C33473432303087
:100E700044206779726F2073656E736F722F636899
:100E800065636B20776972696E672100416E676CDC
:100E900065732F00496E636C2E20616E672E004EC5
:100EA0006F2073656E736F72210049522054656D17
:100EB0007065726174757265004D656173757269F4
:100EC0006E672E2E004E6F2073656E736F723F003B
:100ED00049522054656D7065726174757265004D7C
:100EE0006561737572696E672E2E00234E6F2073D5
:100EF000656E736F7220666F7220504D21004E6FC9
:100F00002073656E736F722100206E672F4C005046
:100F10004D313A322E353A3130004D65617375727C
:100F2000696E672E2E004E6F2053656E736F7221AF
:100F3000004E6F20445320546865726D6F6D657468
:100F400065722100445320546865726D2E004D6F08
:100F500074696F6E0046696E64696E6720576946F2
:100F600069204950007365703D006976616C3D00F1
:100F70006E697465723D00230043616C2E204661EA
:100F8000696C65640043616C2E20446F6E65004E91
:100F90006F206E656564210043616C6962726174E3
:100FA0006421004D61676E65746F6D6574657200D4
:100FB00043616C696272617465202E2E3630730055
:100FC000466F7263652053656E736F720043616C88
:100FD00069627261746500496E76616C6964206B48
:100FE000657900313D4F4B20303D526563616C2E79
:100FF0000062756666657220736F6C6E2E00436FBB
:101000006E6475637469766974790043616C6962B2
:101010007261746500496E76616C6964206B6579F4
:1010200000313D4F4B20303D4578697400496E20BA
:101030007361742E20736F6C6E2E00446973736F2E
:101040006C766564204F320043616C696272617432
:101050006500496E76616C696420502850612900F2
:101060005365614C6576656C2050285061293A00C3
:1010700043616C696272617465205000416972203D
:1010800054656D70286F43293A0043616C2E204DE2
:101090006F74696F6E004453542054656D702073F3
:1010A000656E736F720043757272656E742073653E
:1010B0006E736F72004F322073656E736F720055DE
:1010C000562073656E736F720043616C6962726162
:1010D0007465004661696C65640054422063616C0C
:1010E0002E20646F6E65005570706572204C696DBE
:1010F00069743A3E004C6F776572204C696D697473
:101100003A3E005475726269646974790046616997
:101110006C65640070482063616C2E20646F6E659E
:10112000007048313020507265737320420070485F
:101130003420507265737320410043616C696272A0
:10114000617465004E45543D426C7565746F6F74F3
:1011500068204C45004E45543D426C7565746F6F78
:101160007468004E45543D57694669005365747470
:10117000696E67204661696C6564005365747469C3
:101180006E6720446F6E65004368616E6765204E30
:101190006574776F726B3E00547970653A00425403
:1011A0002F57694669204E6574776F726B004368EC
:1011B000616E67652053656E736F723E0043757292
:1011C00072656E742053656E736F72004F7468653C
:1011D0007200496E642E20342D32306D410041433F
:1011E00053373132203C33304100414353373132A1
:1011F000203C32304100414353373132203C3541AD
:10120000003E4D617820566F6C743A3E0043686131
:101210006E676520766F6C746167653E0054797007
:10122000652000566F6C746167652053656E736F3F
:1012300072004368616E6765207479706520746F11
:101240000053656E736F723D4448540054656D7071
:101250002048756D696469747900295C67411F8550
:101260006341B81E5D413D0A5741A47051410AD700
:101270004B4152B846418FC24141C3F53C41E17AEE
:101280003841F6283441F6283041EC512C41E17ABE
:101290002841CDCC2441AE4721418FC21D415C8FF6
:1012A0001A41295C1741EC511441AE471141666661
:1012B0000E4114AE0B41B81E09415C8F064100007F
:1012C00004418FC2014152B8FE40713DFA407B1487
:1012D000F64085EBF1408FC2ED409A99E9408FC20C
:1012E000E540713DE2406666DE4048E1DA40295C57
:1012F000D740F628D440C3F5D040B81ECD40234592
:10130000432043616C6962726174696F6E2053752A
:10131000636365737366756C002349737375652029
:1013200045433D4520746F205361766520616E64AE
:101330002045786974002345432043616C2E205377
:1013400075636365737366756C2C4B3D0023454371
:101350002043616C6962726174696F6E20466169D5
:101360006C656400234661696C65642C5472792055
:10137000416761696E00466F726365004D6173730A
:101380000028303D6F6C6420484D43353838333B7E
:10139000313D6E6577204D4D433538383329002374
:1013A0004D61676E657469632053656E736F723D3E
:1013B0000028303D6175746F3B313D616363656C3E
:1013C0003B323D696E636C20616E676C653B203318
:1013D0003D616E672076656C290023416363656C0F
:1013E00065726174696F6E20413D002354696D65BB
:1013F000206475726174696F6E3D002354696D6578
:1014000020696E74657276616C3D002354656D7061
:1014100020262048756D69646974792073656E7340
:101420006F723A204448540028303D426C75657410
:101430006F6F74683B313D576946693B323D426C82
:101440007565746F6F7468204C452900234E657470
:101450003D00235556207A65726F20766F6C74615B
:101460006765203D002343616C6962726174656445
:10147000204F3220636F6E63203D0023566F6C74E3
:101480006167652073656E6F723A00556E6B6E6FA3
:10149000776E00496E647573747269616C20342DC7
:1014A00032306D4100414353373132204D61783D38
:1014B0003541002343757272656E742073656E73D7
:1014C0006F723A0023547572626964697479207688
:1014D0006F6C74616765733A00234C434420616408
:1014E00064726573733D307800235365612D6C65BC
:1014F00076656C2050726573737572653D00234F7D
:10150000532076657273696F6E3A2000234D6F62C7
:10151000696C65204C6F67676572204E616D653A36
:101520002000696E7075742044535463616C696265
:10153000726174653A0023444F2043616C696272A2
:101540006174696F6E204661696C65640023444F65
:101550002043616C6962726174696F6E20537563B8
:101560006365737366756C0023444F205361747513
:10157000726174696F6E2043616C69627261746933
:101580006F6E2046696E697368656421002350752B
:101590007420444F2070726F626520696E746F20F2
:1015A00073617475726174696F6E206F78796765A5
:1015B0006E2077617465722100235479706520274D
:1015C000312720666F72204F4B206F722027302703
:1015D00020746F206578697400237363616C6520E3
:1015E000666163746F723D002350757420302E3134
:1015F000306B672077656967687420666F72206357
:10160000616C69627261746F6E0043616C696272D1
:1016100061746520302E31306B6700313D4F4B20B7
:10162000303D4578697400234E6F20666F726365A4
:101630002073656E736F7220485837313121002353
:101640004858373131205343414C453D00485837C5
:101650003131205343414C45002350726573732050
:10166000313D4F4B206F7220303D45786974003119
:101670003D4F4B20303D4578697400546172653AA6
:101680004E6F20776569676874002352656D6F76C9
:101690006520616C6C2077656967687420746F20C1
:1016A0007461726520666F72207A65726F002343E1
:1016B000616C6962726174696F6E20646F6E65003F
:1016C000235374617274002343616C6962726174A4
:1016D000696F6E204D6F6465002343616C696272AF
:1016E0006174696F6E20636F6D706C657465640002
:1016F00023526F7461746520746865206C6F67672E
:10170000657220696E20382D736861706564207081
:1017100061746820322D332074696D657300234332
:10172000616C6962726174696E67206D61676E6574
:10173000746F6D6574657220666F72203630732E1B
:101740002E2E004D4D43353838334D413D2000237A
:101750005461726520666F7263652073656E736F86
:10176000720054464F5243450023536574757020F0
:10177000666F7263652073656E736F720049464FC2
:10178000524345002343616C69627261746520664F
:101790006F7263652073656E736F720043464F52BC
:1017A0004345004D41535300464F524345002349A2
:1017B000737375652045433D5320746F20737461C6
:1017C00072742045432063616C6962726174696F51
:1017D0006E00235075742045432070726F62652D32
:1017E0003E3134313375532F636D206F72203132A7
:1017F0002E38386D532F636D2062756666657220D2
:10180000736F6C7574696F6E0020766F6C746167AE
:10181000653D00235475726269646974792055705E
:10182000706572204C696D69743A200020766F6C87
:10183000746167653D0023547572626964697479E7
:10184000204C6F776572204C696D69743A200023D3
:10185000547572626964697479204C6F776572207F
:101860004C696D69742056696E663A20004D617846
:101870002072616E67653D0023566F6C7461676509
:101880002073656E736F723A00342D32306D4100F3
:10189000414353373132204D61783D004143533746
:1018A0003132204D61783D354100234375727265B8
:1018B0006E742073656E736F723A00234453205424
:1018C0006865726D6F6D657465722063616C6962C5
:1018D000726174656420666F722023004453540063
:1018E000234E6F206E65656420746F2063616C69A0
:1018F00062726174652063757272656E74207365BF
:101900006E736F7221002341435337313220637568
:101910007272656E742073656E736F72206F666687
:1019200073657420563D00235556207A65726F20EA
:10193000766F6C74616765203D0055565A00234FE1
:101940003220766F6C253D00234F322063616C6935
:1019500062726174696F6E3A200023566F6C746115
:1019600067652870483D3130293A0023566F6C7402
:101970006167652870483D34293A00504834005565
:1019800054454D503D004448543D004149413D00BF
:101990004149413D00413D002354696D6520647516
:1019A000726174696F6E3D002354696D6520696EC4
:1019B00074657276616C3D00576946692049503AFA
:1019C00000234D5320456E61626C656400234D53C6
:1019D0002044697361626C656400235265737420EE
:1019E000706172616D657465727320746F206465D7
:1019F0006661756C742076616C756573004C6F67F9
:101A0000676572204E616D653A2000697465726188
:101A100074696F6E3D0073656E736F72233D004392
:101A2000757272656E74207374617475733A206395
:101A300079636C653D006E6379636C653D006E7320
:101A4000656E736F72733D006D61786E73656E7352
:101A50006F72733D00656E61626C65643D00234D7D
:101A6000756C746973656E736F7273206D656173E5
:101A70007572656D656E742073657474696E6773D5
:101A80003A002353657474696E6773206F66206132
:101A90006C6C2073656E736F72733A002353697AAE
:101AA00065206F6620686561646572202B20616C1B
:101AB0006C2073656E736F72733A20002353697ADA
:101AC00065206F66206865616465723A20004F6624
:101AD00066206169722D636F6E64210049742773FB
:101AE00020746F6F20636F6F6C210054656D7020E0
:101AF00069732066696E6521004973206169722DE2
:101B0000636F6E64206F6E3F004974277320717598
:101B100069746520686F74210049742773207665A5
:101B2000727920686F742120004F666620616972A7
:101B30002D636F6E6421004974277320746F6F20CA
:101B4000636F6F6C210054656D7020697320666946
:101B50006E6521004973206169722D636F6E642088
:101B60006F6E3F0049742773207175697465206832
:101B70006F74210049742773207665727920686F2D
:101B800074210054656D702048756D6964697479BD
:101B9000002320616E6420726561647920746F2077
:101BA0007573652100206D6F62696C65206C6F67CD
:101BB0006765722073746172746564200043616CA0
:101BC0006962726174696F6E2050726573737572A9
:101BD000653D00536561206C6576656C2050286317
:101BE000616C63293D00234572726F723A707265B1
:101BF000737375726520424D503038352C20636800
:101C000065636B20776972696E67210049522054C1
:101C1000656D702073656E736F7220666F756E648C
:101C200000206D6F62696C65206C6F67676572205C
:101C300073746172746564202E2E2E2000576946DD
:101C4000692049503A00235769466920495020616C
:101C50006464726573733A20002323205345534C08
:101C60006F676765722023230023232057656C6309
:101C70006F6D65202323004C4344206164647265CA
:101C800073733D30780053656E736F7220736C6FA1
:101C90007420616E6420747970653A00005EBCE265
:101CA000613FDD83C29C7E20A3FD1F41009D23BEBA
:101CB00046DB65F88C11AF32CA57E9740000210089
:101CC000240027002A002D0030003300010100000D
:101CD000040107010A0100002200250028002B0052
:101CE0002E003100340002010000050108010B0143
:101CF000000020002300260029002C002F003200C5
:101D0000000100000301060109010505050507059D
:101D100008080808020202020A0A08080404040467
:101D20000101010101010101030303030303030393
:101D3000040707070C0C0C0C0C0C0C0C0202020222
:101D400006060606060606060B0B0B0B0B0B0B0B0B
:101D500001021020200808102040102040800201BD
:101D600002010804020101020408102040808040A2
:101D700020100804020180040201804020100804A1
:101D8000020108040201010204081020408001023F
:101D900004081020408000000A0B02090C0D0E08F8
:101DA0000703040100000000000000000000000024
:101DB0000000000000000000000000000000000023
:101DC00000001211100000000000000000000000E0
:101DD00000000000000000000000000023456E64C9
:101DE000206F66204D756C746973656E736F722019
:101DF0004379636C652300496E76616C6964206B7E
:101E000065792100EAD3AED311241FBECFEFD1E212
:101E1000DEBFCDBF00E00CBF1CE0A0E0B2E0ECEB09
:101E2000FDEC01E00BBF02C007900D92A038B10796
:101E3000D9F726E1A0E8BCE001C01D92AB32B207A1
:101E4000E1F71FE0C3E0DFE000E006C021970109F1
:101E5000802FFE010E94ECE3C230D10780E008072A
:101E6000A9F70E9425D70C94CCE60C9400000F93A0
:101E70001F93CF93DF93CDB7DEB7A2970FB6F89439
:101E8000DEBF0FBECDBF8E010B5E1F4F682FC80196
:101E90000E94AD7018870F831D821E82198289E00F
:101EA0008A8381E08B838C831C8A1B8ACE010196F6
:101EB0000E940270CE0101960E94A56E60E0CE01E4
:101EC00001960E94966FA2960FB6F894DEBF0FBEE1
:101ED000CDBFDF91CF911F910F9108950F931F9365
:101EE00060E08091A6040E94456C83E090E0019739
:101EF000F1F761E08091A6040E94456C83E290E0D6
:101F00000197F1F760E08091A6040E94456C8091F2
:101F1000A4049091A5049927FC01E05BF24E649122
:101F2000FC01E65FF24EE491F0E0EE0FFF1FE0519E
:101F3000F34E8591949100E717E120E030E0462FC1
:101F40000E94E6D2611571058105910529F06F5F48
:101F50007F4F8F4F9F4F9F700E94C8DE20E030E47C
:101F60004CE156E40E9440E12091D10C3091D20C1A
:101F70004091D30C5091D40C0E9427DF20E030E038
:101F800048E453E40E9440E11F910F910895CF92DD
:101F9000DF92EF92FF920E946E0F6B017C0120E0B6
:101FA00030E040E050E40E9449E2181624F40E9418
:101FB0006E0F6B017C0120E030E040E050E4C7018F
:101FC000B6010E9449E2181624F40E946E0F6B01BC
:101FD0007C0120E030E040E050E4C701B6010E94FF
:101FE00049E2181624F40E946E0F6B017C0120E078
:101FF00030E040E050E4C701B6010E9449E2181603
:1020000024F40E946E0F6B017C0120E030E040E080
:1020100050E4C701B6010E9449E218162CF4C12C05
:10202000D12CE12C80E4F82EC701B601FF90EF908F
:10203000DF90CF900895CF93DF9320919D042223CA
:10204000A9F02091FB04222389F0EC016FED86E1D9
:1020500096E10E9435CB8C819D81892B39F0BE01A0
:1020600086E196E1DF91CF910C9452D1DF91CF912F
:10207000089580919D04882349F08091FB04882372
:1020800029F060E086E196E10C94BD7308950F930A
:102090001F93CF93DF938C011092D60C1092D50C26
:1020A000C091D50CD091D60CC832D105A4F4809142
:1020B0000C020E94B76CCC0FDD1FC654D14F998320
:1020C00088838091D50C9091D60C01969093D60C74
:1020D0008093D50CE5CF0E9409AE20E030E040EAC5
:1020E00050E40E9427DF20E030E040E85AE30E94FD
:1020F00027DF0430110599F420E030E040E650E499
:102100000E9427DF9B01AC0160E070E080E890E472
:102110000E9461E0DF91CF911F910F9108950A30E5
:10212000110569F420E030E040E650E40E9427DF2A
:102130009B01AC0160E070E080E291E4E9CF60E0F7
:1021400070E0CB01E7CF23E333E948E853E40E9492
:1021500040E120E030E040E85FE30E9462E00E945E
:102160006AE326E636EA45EA53E40E9427DF6093F5
:10217000D10C7093D20C8093D30C9093D40C08950F
:1021800081E08093FB0480919D04882341F088E0E6
:102190008093211660E086E196E10C948B7308959C
:1021A00080919D04811110C081E080939D048093F3
:1021B000FB0480911C16982F946090931C168C60E1
:1021C0000E94E9AC0C94C0108091FB048823D1F3E9
:1021D0001092211660E086E196E10E948B731092C6
:1021E000FB0480911C168B7F80931C1688600E94D4
:1021F000E9AC10929D0408952F923F924F925F9206
:102200006F927F928F929F92AF92BF92CF92DF9206
:10221000EF92FF920F931F93CF93DF936C01C7E66A
:10222000D5E083EB882E84E0982E01EE12E1EE24B7
:10223000E394F12C22E1222E312C33E1432E512C58
:1022400040E1642E712C51E1A52EB12C8091B30494
:102250009091B4048E159F050CF4C9C021E0C216FC
:10226000D10409F0BDC0F80182AD93ADF4019383B0
:102270008283F40182819381009709F58A819B8191
:1022800090930B0280930A02F4018281938184303F
:102290009105C1F52A813B8130930D0220930C02F8
:1022A0008531910509F47BC08631910509F040C064
:1022B0002A813B813093900420938F044EC081305B
:1022C000910539F48A819B8190939F0480939E04A9
:1022D000DBCF8230910539F48A819B81909309028A
:1022E00080930802D1CF039779F68A819B819093DE
:1022F00007028093060261E37CE08BE195E10E9496
:102300009AC5C2CF8530910539F42A813B8130933B
:102310008E0420938D04C4CF8630910529F2873036
:102320009105B9F42A813B8130939404209393045E
:102330008731910591F42A813B8128303105B1F52F
:102340007092A7046092A604B092A504A092A4047F
:1023500004C08A30910509F0A3CF9C012B503109AC
:102360002A30310590F42A813B8130930702209373
:10237000060239E1389FB001399F700D11246C5E5F
:102380007D4F8BE195E10E94FDC58FEFE81AF80AB9
:102390002296E2E08E0E911C0E5F1F4F57CF2A81CE
:1023A0003B813093920420939104D7CF273031059D
:1023B00049F43092A7042092A6045092A5044092BA
:1023C000A404CBCF2630310541F621E030E0309334
:1023D000A7042093A6041092A5041092A404BDCFD4
:1023E000F40182819381F80193AF82AF42CFDF91F4
:1023F000CF911F910F91FF90EF90DF90CF90BF9002
:10240000AF909F908F907F906F905F904F903F9094
:102410002F9008954F925F926F927F929F92AF920A
:10242000BF92CF92DF92EF92FF920F931F93CF93C1
:10243000DF93982E8EE0A82EB12CEE24EA9493E040
:10244000F92E0FEF13E0D12CC12CD0E0C0E0412CCD
:10245000512C3201892D0E94B76CC817D90708F496
:102460004AC0C816D90608F46C018017910708F411
:1024700044C08E159F0508F47C01BC0190E080E00B
:102480000E94C6DE9B01AC01C301B2010E9462E062
:102490002B013C0165E070E080E090E00E94FF6C61
:1024A00081E0A81AB108B1F6BE016C0D7D1D6E0D5C
:1024B0007F1D600F711F90E080E00E94C6DE9B01CF
:1024C000AC01C301B2010E9461E020E030E040E2D3
:1024D00051E40E9440E1DF91CF911F910F91FF9055
:1024E000EF90DF90CF90BF90AF909F907F906F90D4
:1024F0005F904F900895EC01B8CF8C01BECFCF9282
:10250000DF92EF92FF92CF93C0911013C4304CF43E
:10251000C1300CF04BC0CC2359F160E070E0CB012E
:102520003FC0C430D1F70E940A1220E030E040EAF8
:1025300050E40E9427DF20E030EC4FE754E40E9493
:1025400040E120E030E040EA50E40E9440E120E039
:1025500030E040E851E40E9427DF20E030E040E82E
:1025600050E40E9462E020E030E04AE754E416C004
:102570000E940A1220E030E040EA50E40E9427DF87
:1025800020E030EC4FE754E40E9440E12091111329
:102590003091121340911313509114130E9440E193
:1025A000CF91FF90EF90DF90CF9008950E940A1294
:1025B0002AE137E64CE950E40E9427DF209111130D
:1025C0003091121340911313509114130E9461E043
:1025D0006B017C01EC2FEE0FFF0BE15AFA4F60818B
:1025E0007181072E000C880B990B0E94C8DE9B019D
:1025F000AC01C701B601D2CF1F93CF93DF93182F41
:10260000CAEBDEE0812F0E94B76C899399936CE34B
:1026100070E080E090E00E94FF6C8FE0CA30D80745
:1026200089F70E9409AE20E030E040EA50E40E94C1
:1026300027DF20E030E040E85AE30E9427DFDF9107
:10264000CF911F910895CF93DF93FC0124813581B1
:10265000232B99F0EC01BC018BE99FE00E9460D133
:102660006EE170E080E090E00E94FF6CBE0182E7C6
:1026700091E1DF91CF910C9460D1DF91CF910895DA
:10268000CF93DF93FC0124813581232B69F0EC018A
:10269000BC0182E791E10E9452D1BE018BE99FE02B
:1026A000DF91CF910C9452D1DF91CF910895809119
:1026B0009D048823F9F08091FB048823D9F081E000
:1026C0000E94E9AC8BE39FE10197F1F760E080E0C5
:1026D0000E94FAAC60EF74E086E196E10E9472D14C
:1026E00061E080E00E94FAAC60EE74E086E196E181
:1026F0000C9472D10895EF92FF920F931F93CF9392
:10270000DF9320919D04222309F461C02091FB04F2
:10271000222309F45CC08A01EB017C01209719F1A6
:10272000C095D09561E08C2F0E94FAACB70186E18C
:1027300096E10E9452D16FEC74E086E196E10E942E
:1027400072D1F701848161E08C0F0E94FAACB8016C
:10275000110F880B990BDF91CF911F910F91FF9073
:10276000EF900C94FF6C0E94326DAB01BC01809124
:10277000900C9091910CA091920CB091930C8C596B
:102780009F4FAF4FBF4F84179507A607B707F8F4C1
:1027900061E080E00E94FAACB70186E196E10E9418
:1027A00052D16EEB74E086E196E10E9472D161E055
:1027B000F70184810E94FAAC0E94326D6093900C04
:1027C0007093910C8093920C9093930CC0CFDF91F7
:1027D000CF911F910F91FF90EF900895FF920F936B
:1027E0001F93CF93DF93EC01F62E08811981C80166
:1027F0000E94E8DFF81621F06F2DC8010E94F0DF7B
:10280000CE01DF91CF911F910F91FF900895DC01D0
:10281000ED91FC910190F081E02D19948F929F929F
:10282000AF92BF92CF92DF92EF92FF920F931F93DE
:10283000CF93DF938C01862F0B30110509F092C0E6
:1028400090912E15992309F0F89462E10E9470C0CE
:10285000EC0180912E15882309F07894209701F1DE
:1028600080E090ECA9E7B4EC8093211590932215B9
:10287000A0932315B09324158093251590932615C6
:10288000A0932715B0932815CE3F8FEFD80709F4F2
:102890009DC0CF3FDC0709F4EFC1CCEFDFEF24C1CF
:1028A000C0912915E0902A156E2D70E090E080E02F
:1028B0000E94C8DE2DEC3CEC4CEC5DE30E9427DF6F
:1028C0004B015C016C2F70E090E080E00E94C8DE5C
:1028D0009B01AC01C501B4010E9462E06093211527
:1028E000709322158093231590932415D0912B1566
:1028F000F0902C156D2F6F7770E090E080E00E94D3
:10290000C8DE4B015C016F2D70E090E080E00E941A
:10291000C8DE2DEC3CEC4CEC5DE30E9427DF9B0114
:10292000AC01C501B4010E9462E0D7FD19C06093FB
:102930002515709326158093271590932815CE0D95
:10294000CD0FCF0D81E090E020912D15C21302C074
:1029500090E080E0892B09F487C0CFEFDFEF8CC1D6
:102960009058E5CFCFEFDFEF0631110509F0BCC07D
:1029700090912E15992309F0F89461E00E9470C09F
:10298000EC0180912E15882309F07894209709F1A5
:1029900080E090ECA9E7B4EC809321159093221588
:1029A000A0932315B0932415809325159093261595
:1029B000A0932715B0932815CF3FDC0709F45CC11D
:1029C000209709F451C0229609F067CFCEEFDFEFD0
:1029D0008BC0C0912A15D09129156091291570914D
:1029E0002A1576276727762790E080E00E94C6DECA
:1029F0002DEC3CEC4CEC5DE30E9427DF609321154D
:102A0000709322158093231590932415E0902C1534
:102A1000F0902B156F2D6F77762F6E2D90E080E064
:102A20000E94C6DE2DEC3CEC4CEC5DE30E9427DFFF
:102A3000F7FC18C060932515709326158093271511
:102A4000909328158C2F8D0F8E0D8F0DC1E0D0E047
:102A500090912D15891302C0D0E0C0E0D195C195A9
:102A6000D109AACF9058E6CFC0902115D090221559
:102A7000E0902315F090241520E030E048EC52E47B
:102A8000C701B6010E9449E2D0E0C0E0181614F474
:102A9000CBEFDFEF20E030E0A901C701B6010E94D3
:102AA000C1DE87FF02C0CAEFDFEFC0902515D090CE
:102AB0002615E0902715F090281520E030E048EC2E
:102AC00052ECC701B6010E94C1DE87FF02C0C9EF08
:102AD000DFEF20E030E040EF52E4C701B6010E9492
:102AE00049E218160CF4C3C00C30110509F0C4C03B
:102AF0008CE50E94DFAC70E060E089EC94E10E941C
:102B0000071489EC94E10E94887365E08CE50E94CB
:102B10003AAD10924B0F80934A0FC82FD0E0209708
:102B200009F4A8C0C530D1050CF4B6C00BEC1DE00B
:102B30000E9427ADF80180870F5F1F4FC8018B5C93
:102B40009D408C179D07A4F3C091D30D0091D40D27
:102B5000602F70E090E080E00E94C8DE2DEC3CEC3D
:102B60004CEC5DE30E9427DF6B017C016C2F70E071
:102B700090E080E00E94C8DE9B01AC01C701B60175
:102B80000E9462E06B017C01C092CB0DD092CC0D13
:102B9000E092CD0DF092CE0DD091D50D1091D60DC5
:102BA0006D2F6F7770E090E080E00E94C8DE4B01EF
:102BB0005C01612F70E090E080E00E94C8DE2DECA7
:102BC0003CEC4CEC5DE30E9427DF9B01AC01C501AE
:102BD000B4010E9462E0D7FD5DC06093CF0D709399
:102BE000D00D8093D10D9093D20DC00FCD0FC10F9A
:102BF0008091D70DC813B1CE20E030E048EC52E40C
:102C0000C701B6010E9449E2D0E0C0E0181614F4F2
:102C1000CBEFDFEF20E030E040EA50E4C701B6013F
:102C20000E94C1DE87FF02C0CAEFDFEFC090CF0D68
:102C3000D090D00DE090D10DF090D20D20E030E09A
:102C400040EF51ECC701B6010E94C1DE87FF02C010
:102C5000C9EFDFEF20E030E040EF52E4C701B601FA
:102C60000E9449E2181644F4C8EFDFEF05C0C8EF30
:102C7000DFEF3ACFCEEFDFEFCE01DF91CF911F91A3
:102C80000F91FF90EF90DF90CF90BF90AF909F900B
:102C90008F9008959058A1CFCDEFDFEFEDCFCF9378
:102CA000DF93EC019A01AB01E889F98982E0808326
:102CB000211581EE38074105510581F160E079E089
:102CC0008DE390E00E9430E0215031094109510923
:102CD0005695479537952795EC85FD851082EE85AD
:102CE000FF852083188EEC89FD8986E08083EA8940
:102CF000FB89808180618083EA89FB89808188608B
:102D00008083EA89FB89808180688083EA89FB89E6
:102D100080818F7D8083DF91CF910895E889F98943
:102D2000108220E1D9CF2F923F924F925F926F9203
:102D30007F928F929F92AF92BF92CF92DF92EF924B
:102D4000FF920F931F93CF93DF93CDB7DEB76697B4
:102D50000FB6F894DEBF0FBECDBF1C0185ED90E12C
:102D60000E94DCB040E855E260E070E085ED90E163
:102D70000E944F1664E670E080E090E00E94FF6CD5
:102D80008CED95E0A0E0B0E08093D9109093DA103C
:102D9000A093DB10B093DC1064E670E080E090E07C
:102DA0000E94FF6C8FEF8A8781E08B8786E88C8793
:102DB0001D861E861F86188A198A89E78A8BC1019B
:102DC000880F991F9E8B8D8BD12CC12CF12CE12C5F
:102DD000412C512C320185ED90E10E9492A9089777
:102DE0004CF049E050E0BE01665F7F4F85ED90E119
:102DF0000E944CA965E070E080E090E00E94FF6CCA
:102E000010E000E0812C912C540185ED90E10E94AE
:102E1000C3A9892B39F4F4E08F169104A104B104FD
:102E20000CF04EC0023011050CF04AC085ED90E167
:102E30000E94C3A9892B69F085ED90E10E94A1A9A8
:102E4000E1E0F0E0EC0FFD1FE00FF11F80830F5F6A
:102E50001F4F65E070E080E090E00E94FF6C023060
:102E6000110509F073C099818A8598136FC09A8102
:102E70008C8598136BC0FE013396FC8BEB8B85ED34
:102E800090E10E94C3A9892B39F4F4E08F169104D4
:102E9000A104B1040CF053C00930110509F05CC065
:102EA0008B8190E0982F88272C81820F911D092E0D
:102EB000000CAA0BBB0B480E591E6A1E7B1E43C09A
:102EC0008FEFC81AD80AE214F30434F4ED89FE89AE
:102ED000EC15FD0509F07FCF85ED90E10E94DCB097
:102EE000E114F10409F47101C301B2010E94C8DECA
:102EF0004B015C01B701FF0C880B990B0E94C8DEE7
:102F00009B01AC01C501B4010E9440E166960FB679
:102F1000F894DEBF0FBECDBFDF91CF911F910F910F
:102F2000FF90EF90DF90CF90BF90AF909F908F90E9
:102F30007F906F905F904F903F902F900895043056
:102F400011050CF0ADCFFFEFEF1AFF0A8FEF881AD3
:102F5000980AA80AB80A59CF85ED90E10E94A1A964
:102F6000EB89FC898193FC8BEB8B0F5F1F4F87CF25
:102F70004F925F926F927F92AF92BF92CF92DF9209
:102F8000FF920F931F93CF93DF9300D000D0CDB764
:102F9000DEB75C0185ED90E10E94DCB040E052ECD0
:102FA00061E070E085ED90E10E944F168CED95E0B8
:102FB000A0E0B0E08093D9109093DA10A093DB10DA
:102FC000B093DC1064E670E080E090E00E94FF6C5B
:102FD000D12CC12CF12C65E070E080E090E00E94E3
:102FE000FF6C10E000E0412C512C3201F1103AC08E
:102FF00085ED90E10E94C3A9892B31F485E1481643
:1030000051046104710474F5033011055CF585ED1C
:1030100090E10E94C3A9892B69F085ED90E10E949F
:10302000A1A9E1E0F0E0EC0FFD1FE00FF11F8083AC
:103030000F5F1F4F65E070E080E090E00E94FF6C42
:10304000023011054CF089818B3B31F4FF24F3945D
:103050008A818A3A09F0F12C8FEF481A580A680AD7
:10306000780AC4CF8FEFC81AD80A64E670E080E00F
:1030700090E00E94FF6CAC14BD0409F0ACCF8F2D22
:1030800026960FB6F894DEBF0FBECDBFDF91CF916D
:103090001F910F91FF90DF90CF90BF90AF907F90E6
:1030A0006F905F904F900895CF93DF93EC01FB01F9
:1030B000248135810E94D4C8CE01DF91CF9108953B
:1030C000CF92DF92EF92FF920F931F93CF93DF93F4
:1030D000CDB7DEB762970FB6F894DEBF0FBECDBF97
:1030E00020919C0D222309F4D8C02091C10D30916C
:1030F000C20D263531050CF0D0C040919B04509193
:103100009C04493D5F400CF0C8C08C012F5F3F4FCD
:103110003093C20D2093C10D0E94326DC090940D6A
:10312000D090950DE090960DF090970D6C197D095B
:103130008E099F090E94C6DE20E030E04AE754E491
:103140000E9440E16093980D7093990D80939A0DC1
:1031500090939B0D80919B0490919C0488359240A4
:1031600034F488E592E090939C0480939B048091D2
:103170009B0490919C0438E9E32E3DE0F32E9C01E2
:1031800028593D406901C6018E0D9F1D9A83898390
:10319000F70161917F01CE0101960E94EE13FCE9D7
:1031A000EF16FDE0FF0679F780919B0490919C0457
:1031B000049690939C0480939B04B801CE010196E1
:1031C0000E94BAC8CE0101960E94B6C7BC01CE01CA
:1031D0000D960E94BAC8CE0101960E9457C8F80108
:1031E00084819581849708F123E230E050E040E04B
:1031F000B801CE0101960E94D4C8BE016F5F7F4F17
:10320000CE0107960E94BAC8CE0107960E94B6C7A3
:10321000BC01CE010D960E94FBC7CE0107960E940D
:1032200057C8CE0101960E9457C849895A8941154D
:10323000510549F08DE99DE0009729F0BC01CE01D0
:103240000D960E948FB080919B0490919C0421EC7C
:10325000C22E2DE0D22E0DE91DE09C012D593D40DE
:103260007901C701800F911F9A838983F8016191C9
:103270008F01CE0101960E94EE13C016D10689F788
:1032800080919B0490919C04849690939C048093DD
:103290009B04CE010D960E9457C862960FB6F89413
:1032A000DEBF0FBECDBFDF91CF911F910F91FF9079
:1032B000EF90DF90CF900895AF92BF92CF92DF92C0
:1032C000EF92FF920F931F93CF93DF93CDB7DEB7AB
:1032D00062970FB6F894DEBF0FBECDBF20919D045C
:1032E000222309F447C02091FB04222309F442C0A1
:1032F0007A016B015C010E94326DAB01BC018091CF
:103300008C0C90918D0CA0918E0CB0918F0C8C59DF
:103310009F4FAF4FBF4F84179507A607B70750F5CC
:1033200060E08FEFC816D806B1F580E00E94FAACD5
:1033300000E0B50186E196E10E9452D16DEA74E0A9
:1033400086E196E10E9472D1F501848160E0800FF0
:103350000E94FAAC0E94326D60938C0C70938D0CBD
:1033600080938E0C90938F0CB701FF0C880B990BF8
:103370000E94FF6C62960FB6F894DEBF0FBECDBF01
:10338000DF91CF911F910F91FF90EF90DF90CF9041
:10339000BF90AF90089580E00E94FAAC0E94326D19
:1033A00028EE33E040E050E00E94FEDFCA01B901A0
:1033B00020E831E541E050E00E94FEDFAB01BC01B6
:1033C000CE0101960E94A4C5BE016F5F7F4FCE0162
:1033D00007960E94BAC866E77BE0CE0107960E9476
:1033E0001EC7BC01CE010D960E94BAC8CE01079639
:1033F0000E9457C8CE0101960E9457C8BE01635F64
:103400007F4F86E196E10E9452D109891A89C11441
:10341000D10431F00C0D1D1D60E0802F0E94FAAC2C
:10342000CE010D960E9457C884CFBF92CF92DF92F3
:10343000EF92FF920F931F93CF93DF93CDB7DEB739
:1034400062970FB6F894DEBF0FBECDBF6C018B0143
:103450007A0180919D04882369F18091FB0488237F
:1034600049F177FF37C00095109560E0802F0E94EA
:10347000FAACB60186E196E10E9452D16CE974E0A3
:1034800086E196E10E9472D1F601848160E0800FAE
:103490000E94FAAC0E94326D60938C0C70938D0C7C
:1034A00080938E0C90938F0CB701FF0C880B990BB7
:1034B0000E94FF6C62960FB6F894DEBF0FBECDBFC0
:1034C000DF91CF911F910F91FF90EF90DF90CF9000
:1034D000BF90089560E080E00E94FAAC0E94326DD7
:1034E00028EE33E040E050E00E94FEDFCA01B9015F
:1034F00020E831E541E050E00E94FEDFAB01BC0175
:10350000CE0101960E94A4C5BE016F5F7F4FCE0120
:1035100007960E94BAC866E77BE0CE0107960E9434
:103520001EC7BC01CE010D960E94BAC8CE010796F7
:103530000E9457C8CE0101960E9457C8BE01635F22
:103540007F4F86E196E10E9452D1B98860E08B2DD1
:103550000E94FAAC0115110531F40B2DCE010D9628
:103560000E9457C886CF60E0802F0E94FAACF6CF49
:10357000CF93DF93EC01483085E058076105710572
:1035800009F448C008F099C0493481E05807610542
:10359000710509F4B2C008F040C0443481E0580716
:1035A0006105710509F476C000F5413481E05807E2
:1035B0006105710509F456C048F440345140610575
:1035C000710509F4E4C061E37CE0E3C0423481E0CA
:1035D00058076105710509F409C14334514061057B
:1035E000710589F76DE87BE0D4C0463481E0580767
:1035F0006105710509F40CC108F49FC0473481E0EE
:1036000058076105710509F455C0483451406105FA
:103610007105C9F66CED75E0BCC0423085E0580715
:103620006105710509F4E2C000F5443781E05807EF
:103630006105710509F4F2C040F44237514061055B
:10364000710509F66FEE77E0A4C0411585E05807D3
:103650006105710509F49BC0413055406105710554
:1036600009F0B1CF63E97BE094C0453085E05807AD
:103670006105710509F461C080F4433085E05807A5
:103680006105710509F4AECF4430554061057105FF
:1036900009F099CF6AE87BE07CC0463085E05807A6
:1036A0006105710509F4B4C04730554061057105E5
:1036B00009F089CF6AED75E06CC04D3B82E4580794
:1036C0008FEF6807710509F4AFC008F048C04F3E9E
:1036D00080E158078FEF6807710561F3F8F4423312
:1036E00085E058076105710509F4ACCF48F449300D
:1036F00055406105710509F066CF6EED75E049C072
:10370000443385E058076105710509F487C04D3FD2
:1037100052406F4F710509F495CF55CF4D3D82E270
:1037200058078FEF6807710509F478C048F4473EE1
:1037300058416F4F710509F046CF67E87BE029C01B
:103740004F3C80E358078FEF6807710509F4A2CF5B
:10375000473C58436F4F710509F45CCF34CF47396C
:1037600088E658078FEF6807710509F47BCF48F5A5
:103770004D3A82E558078FEF6807710509F451C08B
:1037800078F4453B5A446F4F710509F01CCF69ED41
:1037900077E0CE010E94C3C8CE01DF91CF9108959A
:1037A000453A8AE558078FEF6807710509F4A5CFF8
:1037B0004D3952466F4F710509F005CF62E079E04F
:1037C000E8CF473588EA58078FEF6807710519F188
:1037D00080F445388AE758078FEF68077105C1F014
:1037E000473658496F4F710509F0EDCE60E97BE02F
:1037F000D0CF4F3480EB58078FEF6807710509F47D
:10380000F1CE4D33524C6F4F710509F41BCFDBCE17
:1038100068ED75E0BECF6BEF7AE0BBCF6BE778E089
:10382000B8CF68E379E0B5CF6BEF77E0B2CF1F9305
:10383000CF93DF9300D000D0CDB7DEB7182F8091A3
:10384000771390917813019709F062C0112331F03A
:1038500065E874E082E791E10E9472D10E9418C08D
:10386000112339F04AE050E0682F82E791E10E948D
:103870000CCB0E94FFBD112309F440C00E940FBC75
:1038800060EE75E0CE0101960E94C3C84091FC1421
:103890005091FD146091FE147091FF14CE010196B9
:1038A0000E9471C767EE75E0CE0101960E94C5C700
:1038B000409100155091011560910215709103150A
:1038C000CE0101960E9471C76BEE75E0CE010196A4
:1038D0000E94C5C7409104155091051560910615C9
:1038E00070910715CE0101960E9471C7CE01019615
:1038F0000E942313CE0101960E9457C826960FB648
:10390000F894DEBF0FBECDBFDF91CF911F91089518
:103910008AE097E5A4EFB2E48093120F9093130F1F
:10392000A093140FB093150F8BE794E1A6E6B3E4D0
:1039300080930E0F90930F0FA093100FB093110F61
:103940008DEC9CEEA2ECB3E480930A0F90930B0FE6
:10395000A0930C0FB0930D0F89E29CE5AFE8BFE395
:103960008093390590933A05A0933B05B0933C05AD
:1039700087ED93EAA0E9BFE3809335059093360580
:10398000A0933705B09338058AE097EDA3E8BFE32D
:103990008093310590933205A0933305B09334059D
:1039A0008EE10E94DFAC61E070E089EC94E10E945E
:1039B000071486EF98E2ACE9BFE380933D0590934E
:1039C0003E05A0933F05B093400560E489EC94E187
:1039D0000E946C6B63E070E089EC94E10E94071434
:1039E00089EC94E10E9488738091280F9091290FAF
:1039F00018161906C4F461EF75E082E791E10E94A0
:103A00007CCC60913D0570913E0580913F05909181
:103A1000400542E050E00E941ECC65E076E082E77F
:103A200091E10E9423CB111105C01092290F109231
:103A3000280F64CF81E090E09093290F8093280FA6
:103A40000E947ECC5BCF3F924F925F926F927F92AB
:103A50008F929F92AF92BF92CF92DF92EF92FF929E
:103A60000F931F93CF93DF93CDB7DEB7EB970FB6CE
:103A7000F894DEBF0FBECDBF2B013C0188E390E17F
:103A80000E94DCB064E670E080E090E00E94FF6C91
:103A900040E855E260E070E088E390E10E944F1654
:103AA00064E670E080E090E00E94FF6C6AE17FE0F5
:103AB00088E894E10E94D6C768E874E1CE010196D7
:103AC0000E94BAC842E350E06FEF7FEFCE0101964B
:103AD0000E94151ACE0101960E9457C86FE07FE040
:103AE00088E894E10E94D6C768E874E1CE010196A7
:103AF0000E94BAC842E350E06FEF7FEFCE0101961B
:103B00000E947B13CE0101960E9457C88091E20D5E
:103B10009091E30D8D7F312CD12CC12CF12CE12C17
:103B200010E000E0019709F47AC09E01205E3F4F4B
:103B300039AF28AFCE014E969BAF8AAF0E94326D4F
:103B40006419750986099709683B7B4081059105D1
:103B500008F065C088E390E10E94C3A9892B09F4AD
:103B60004DC08CED95E0A0E0B0E080933C109093C8
:103B70003D10A0933E10B0933F100E94DEAF97FD22
:103B80003DC082349105C9F7DE0111964D015D01FA
:103B90000E94DEAF97FF39C089818D3479F590E0BE
:103BA00080E0D4012D914D01820F911DEAADFBAD56
:103BB000AE17BF07B1F78E5B9F4F2E8D30E0322FCF
:103BC00022274F8D240F311D82179307B9F40C81E2
:103BD00010E0102F00278D81080F111DEE80F12CB1
:103BE000FE2CEE248F81E80EF11CC884D12CDC2C35
:103BF000CC248985C80ED11C3324339462E370E051
:103C000080E090E00E94FF6C99CFD5018D935D011B
:103C1000E8ADF9ADAE17BF0709F0BACFBDCF0E942E
:103C2000326D6419750986099709683B7B408105E7
:103C3000910510F43110BBC00E94571368E874E17D
:103C4000CE0180960E94BAC842E350E066E070E080
:103C5000CE0180960E94151ACE0180960E9457C808
:103C6000332009F4CCC082E090E09093E30D809380
:103C7000E20DB601CE01C2960E94D1C5B701CE01B8
:103C80008C960E94D1C5B801CE0180960E94D1C504
:103C9000BE01605E7F4FCE0186960E94BAC860E684
:103CA00077E0CE0186960E941EC7BE01645D7F4FFD
:103CB0000E9434C760E677E00E941EC7BE016E5CBA
:103CC0007F4F0E9434C7BC018EE894E10E94FBC77D
:103CD000CE0186960E9457C8CE0180960E9457C892
:103CE000CE018C960E9457C8CE01C2960E9457C83A
:103CF0006EE874E1CE0180960E94BAC84AE050E0B6
:103D00006FEF7FEFCE0180960E947B13CE018096ED
:103D10000E9457C869E07FE086E196E10E9472D177
:103D2000B601CE01C2960E94D1C5B701CE018C96D4
:103D30000E94D1C5B801CE0186960E94D1C56DE022
:103D400076E0CE0180960E94C3C8BE016A5D7F4FB7
:103D5000CE0180960E9434C76EE277E00E941EC7B3
:103D6000BE01645D7F4F0E9434C76EE277E00E941F
:103D70001EC7BE016E5C7F4F0E9434C76DE176E0C6
:103D80000E941EC7BC018EE894E10E94FBC7CE01D1
:103D900080960E9457C8CE0186960E9457C8CE01D1
:103DA0008C960E9457C8CE01C2960E9457C862E303
:103DB00070E080E090E00E94FF6C88E390E10E9458
:103DC000DCB062E370E080E090E00E94FF6CEB9674
:103DD0000FB6F894DEBF0FBECDBFDF91CF911F911C
:103DE0000F91FF90EF90DF90CF90BF90AF909F909A
:103DF0008F907F906F905F904F903F9008956EEFFF
:103E00007EE08EE894E10E94D6C76EE874E1CE01B0
:103E100080960E94BAC84AE050E070E060E0CE01AF
:103E200080960E947B13CE0180960E9457C86BEE4D
:103E30007EE08EE894E10E94D6C78091E20D9091D9
:103E4000E30D029709F0B3CF1092E30D1092E20D4B
:103E5000AECF0F931F93CF93DF9300D000D0CDB799
:103E6000DEB720916E0E2223A9F08C0168E379E081
:103E7000CE0101960E94C3C8B801CE0101960E94EE
:103E800034C7BC0182E791E10E9460D1CE01019666
:103E90000E9457C826960FB6F894DEBF0FBECDBF5E
:103EA000DF91CF911F910F910895CF93DF93CDB7FD
:103EB000DEB72C970FB6F894DEBF0FBECDBF8130B2
:103EC000910509F06EC0909358138093571363E6E1
:103ED00071E1CE0101960E94B1C8CE0101960E9407
:103EE000291FCE0101960E9457C863E276E0CE01F9
:103EF00001960E94C3C86EEF75E1CE0101960E9443
:103F000034C7BC01CE0107960E94BAC848EC50E005
:103F10006FEF7FEFCE0107960E94151ACE0107962C
:103F20000E9457C8CE0101960E9457C88BE99FE0B6
:103F30000E94DCB040E052EC61E070E08BE99FE071
:103F40000E944F1690E080E00E9465B062E376E048
:103F5000CE0101960E94C3C86AE076E1CE010196C7
:103F60000E9434C7BC01CE0107960E94BAC840ED3A
:103F700057E06FEF7FEFCE0107960E947B13CE01D3
:103F800007960E9457C8CE0101960E9457C881E04B
:103F90002C960FB6F894DEBF0FBECDBFDF91CF9148
:103FA00008950097E1F5109258131092571365E5A4
:103FB00071E1CE0101960E94B1C8CE0101960E9426
:103FC000291FCE0101960E9457C869E276E0CE0112
:103FD00001960E94C3C86EEF75E1CE0101960E9462
:103FE00034C7BC01CE0107960E94BAC848EC50E025
:103FF0006FEF7FEFCE0107960E94151ACE0107964C
:104000000E9457C8CE0101960E9457C88BE99FE0D5
:104010000E94DCB040E855E260E070E08FCF823073
:104020009105A9F4909358138093571364E471E1B8
:10403000CE0101960E94B1C8CE0101960E94291FAF
:10404000CE0101960E9457C86DE276E0C0CF80E0B5
:104050009FCFBF92CF92DF92EF92FF920F931F9369
:10406000CF93DF93CDB7DEB762970FB6F894DEBF7C
:104070000FBECDBF8C016B016EE277E0CE010D96D5
:104080000E94C3C867E77FE0C8010E94B1C87601FB
:104090002FEFE21AF20AB701CE0101960E94D1C5B4
:1040A000BE016F5F7F4FCE0107960E94BAC860E6DF
:1040B00077E0CE0107960E941EC7BC01C8010E948E
:1040C000CFC7CE0107960E9457C8CE0101960E9425
:1040D00057C88AE0B82EBE9CC001BF9C900D112429
:1040E000FC01E857FC4E7F018081082E000C990BE3
:1040F0000E945BE6892B09F4B2C0B701CE0101969C
:104100000E94C3C8BE016F5F7F4FCE0107960E9419
:10411000BAC861E77BE0CE0107960E941EC7BC01CA
:10412000C8010E94CFC7CE0107960E9457C8CE0192
:1041300001960E9457C8BC9CC001BD9C900D1124E3
:104140009C0128573C4E7901F9016685062E000C2A
:10415000770BCE0101960E94D1C5BE016F5F7F4FE4
:10416000CE0107960E94BAC862E57CE0CE010796B0
:104170000E941EC7BE01635F7F4F0E9434C7BC010F
:10418000C8010E94CFC7CE0107960E9457C8CE0132
:1041900001960E9457C860E77FE0C8010E9447C7A8
:1041A000F7016785062E000C770BCE0101960E9461
:1041B000D1C5BE016F5F7F4FCE0107960E94BAC87E
:1041C000BE01635F7F4FCE0107960E9434C7BC01DA
:1041D000C8010E94CFC7CE0107960E9457C8CE01E2
:1041E00001960E9457C86AE67FE0C8010E9447C74F
:1041F000F70160897189CE0101960E94D1C5BE0187
:104200006F5F7F4FCE0107960E94BAC8BE01635F01
:104210007F4FCE0107960E9434C7BC01C8010E949F
:10422000CFC7CE0107960E9457C8CE0101960E94C3
:1042300057C865E67FE0C8010E9447C7F701628959
:104240007389CE0101960E94D1C5BE016F5F7F4F79
:10425000C8010E94CFC7CE0101960E9457C8CE0167
:104260000D960E9457C8C80162960FB6F894DEBF3B
:104270000FBECDBFDF91CF911F910F91FF90EF90B7
:10428000DF90CF90BF9008954F925F926F927F9290
:104290009F92AF92BF92CF92DF92EF92FF920F93D5
:1042A0001F93CF93DF93CDB7DEB7A9970FB6F894DE
:1042B000DEBF0FBECDBF982E882351F080916E0EC9
:1042C000882331F061E37CE082E791E10E9423CB17
:1042D0000E9417C260E08DE20E9455C160E18DE24C
:1042E0000E9455C168E08DE20E9455C110E000E0D7
:1042F00010928B0E10928C0E10928D0E10928E0ECC
:1043000010928F0E1092900E1092910E1092920EAB
:104310001092930E1092940E1092950E1092960E8B
:104320001092A30E1092970E1092980E1092990E62
:1043300010929A0E10929B0E10929C0E10929D0E4F
:1043400010929E0E10929F0E1092A00E1092A10E2F
:104350001092A20E1092A40E1092A50E1092A60E0C
:104360001092A70E0E9417C289E60E94DFAC6FE090
:1043700089EC94E10E946C6B89EC94E10E94887353
:1043800089E60E94DFAC41E050E069E670E089EC2C
:1043900094E10E94D4730E9427ADF82E89EC94E139
:1043A0000E94887383EDF81609F4A1C5043611053F
:1043B00009F01DC610E04090311550903215609004
:1043C000331570903415498E5A8E6B8E7C8EC0904A
:1043D0003515D0903615E0903715F0903815CD8E04
:1043E000DE8EEF8EF8A28091391590913A15A0914A
:1043F0003B15B0913C158EA39FA3A8A7B9A789A38D
:104400009AA3ABA3BCA3992009F44AC062E27EE060
:1044100082E791E10E9472D167E07EE0111102C053
:104420006FEF7DE082E791E10E9472D182E791E136
:104430000E9408CB63E17EE0CE0101960E94B1C8E4
:10444000CE0101960E94291FCE0101960E9457C8F5
:104450008E01075E1F4F5E0195E2A90EB11CD801C7
:104460006D917D918D919D918D0146E050E00E946E
:104470001ECC6EE277E082E791E10E947CCCA01630
:10448000B10669F761E37CE0CE0101960E94C3C8E2
:10449000CE0101960E94291FCE0101960E9457C8A5
:1044A00023E938E144E85FE3C301B2010E9427DF5A
:1044B0002B013C014D865E866F86788A22E430E6C9
:1044C00045E85FE3C701B6010E9427DF6B017C016D
:1044D000C98ADA8AEB8AFC8A25E83BEE41E95FE388
:1044E0006EA17FA188A599A50E9427DF6D8B7E8B89
:1044F0008F8B988F40923115509232156092331500
:1045000070923415C0923515D0923615E092371559
:10451000F09238156093391570933A1580933B15D6
:1045200090933C15992009F4A2C080916E0E8823C7
:1045300009F49DC062EF7DE0CE0101960E94B1C8F2
:10454000CE0101960E94291FCE0101960E9457C8F4
:104550008E01035F1F4F6E01B9E1CB0ED11C7801B4
:10456000F80161917191819191918F0142E050E048
:104570000E941ECC6EE277E082E791E10E947CCC43
:10458000C016D10669F761E37CE0CE0101960E9476
:10459000C3C8CE0101960E94291FCE0101960E9438
:1045A00057C84DE355E166E070E082E30E94FBC02E
:1045B000A0903D15B0903E15C0903F15D09040158D
:1045C000009141151091421565EE7DE082E791E181
:1045D0000E9472D14AE050E0B50182E791E10E9469
:1045E0002FCC6EE277E082E791E10E947CCC4AE03A
:1045F00050E0B60182E791E10E942FCC6EE277E0B5
:1046000082E791E10E947CCC4AE050E0B80182E769
:1046100091E10E942FCC61E37CE082E791E10E946E
:1046200023CBCE0101960E9497C16CED7DE082E71D
:1046300091E10E9472D18E010F5F1F4FD8016D91E1
:104640007D918D919D918D014AE050E00E941ECC9C
:104650006EE277E082E791E10E947CCCE016F10601
:1046600069F761E37CE082E791E10E9423CB61E09E
:104670008DE10E9455C19920B1F080916E0E882382
:1046800091F068EC7DE082E791E10E9472D1AE0189
:104690004B5D5F4F61E070E08DE10E94FBC08DA13A
:1046A00090E00E9469CC62E08EE10E9455C163E017
:1046B0008FE10E9455C164E080E20E9455C19920BB
:1046C00009F450C080916E0E882309F44BC06CEA47
:1046D0007DE082E791E10E9472D1AE014B5D5F4FB8
:1046E00061E070E08EE10E94FBC0CDA0D12CAE0154
:1046F0004B5D5F4F61E070E08FE10E94FBC0EDA079
:10470000F12CAE014B5D5F4F61E070E080E20E94F2
:10471000FBC00DA110E04AE050E0B60182E791E154
:104720000E942FCC6EE277E082E791E10E947CCC80
:104730004AE050E0B70182E791E10E942FCC6EE29F
:1047400077E082E791E10E947CCC4AE050E0B8013A
:1047500082E791E10E942FCC61E37CE082E791E166
:104760000E9423CB65E081E20E9455C19920B1F0FF
:1047700080916E0E882391F069E97DE082E791E1F6
:104780000E9472D1AE014B5D5F4F61E070E081E24B
:104790000E94FBC08DA190E00E9469CC66E082E29D
:1047A0000E9455C19920B1F080916E0E882391F03E
:1047B00061E87DE082E791E10E9472D1AE014B5D3C
:1047C0005F4F61E070E082E20E94FBC08DA190E04B
:1047D0000E9469CC67E083E20E9455C19920B1F044
:1047E00080916E0E882391F06BE67DE082E791E187
:1047F0000E9472D1AE014B5D5F4F61E070E083E2D9
:104800000E94FBC08DA190E00E9469CC68E084E228
:104810000E9455C19920B1F080916E0E882391F0CD
:1048200063E57DE082E791E10E9472D1AE014B5DCC
:104830005F4F61E070E084E20E94FBC08DA190E0D8
:104840000E9469CC69E085E20E9455C19920B1F0CF
:1048500080916E0E882391F069E37DE082E791E11B
:104860000E9472D1AE014B5D5F4F61E070E085E266
:104870000E94FBC08DA190E00E9469CC6AE086E2B4
:104880000E9455C19920B1F080916E0E882391F05D
:1048900063E27DE082E791E10E9472D1AE014B5D5F
:1048A0005F4F61E070E086E20E94FBC08DA190E066
:1048B0000E9469CC6BE088E20E9455C19920B1F05A
:1048C00080916E0E882391F06AE07DE082E791E1AD
:1048D0000E9472D1AE014B5D5F4F61E070E088E2F3
:1048E0000E94FBC08DA190E00E9469CC6CE089E23F
:1048F0000E9455C1992009F479C080916E0E8823D9
:1049000009F474C062EF7CE082E791E10E9472D109
:10491000AE014B5D5F4F61E070E089E20E94FBC039
:104920008DA190E00E9469CC6BED7CE082E791E183
:104930000E9472D166E070E087E20E943AC190E086
:104940000E9469CC64EC7CE082E791E10E9472D124
:1049500065E070E087E20E943AC190E00E9469CC75
:104960006DEA7CE082E791E10E9472D164E070E040
:1049700087E20E943AC190E00E9469CC64E97CE041
:1049800082E791E10E9472D162E070E087E20E94CA
:104990003AC190E00E9469CC6BE77CE082E791E14C
:1049A0000E9472D161E070E087E20E943AC190E01B
:1049B0000E9469CC62E67CE082E791E10E9472D1BC
:1049C00070E060E087E20E943AC190E00E9469CC0A
:1049D00061E57CE082E791E10E9472D163E070E0E2
:1049E00087E20E943AC190E00E9469CC41E067E012
:1049F00070E087E20E946CC141E063E070E087E212
:104A00000E946CC141E063E070E08AE20E946CC1E8
:104A1000992091F080916E0E882371F068E37CE01C
:104A200082E791E10E9472D163E070E08AE20E9425
:104A30003AC190E00E9469CC40E063E070E08AE215
:104A40000E946CC1992091F080916E0E882371F0C4
:104A50006EE17CE082E791E10E9472D163E070E058
:104A60008AE20E943AC190E00E9469CC41E062E093
:104A700070E08AE20E946CC1992091F080916E0EE4
:104A8000882371F062E07CE082E791E10E9472D1BC
:104A900062E070E08AE20E943AC190E00E9469CC34
:104AA00040E062E070E08AE20E946CC1992091F0DF
:104AB00080916E0E882371F065EE7BE082E791E1D4
:104AC0000E9472D162E070E08AE20E943AC190E0F6
:104AD0000E9469CC41E061E070E08AE20E946CC112
:104AE000992091F080916E0E882371F069EC7BE043
:104AF00082E791E10E9472D161E070E08AE20E9457
:104B00003AC190E00E9469CC40E061E070E08AE246
:104B10000E946CC1992091F080916E0E882371F0F3
:104B20006CEA7BE082E791E10E9472D161E070E083
:104B30008AE20E943AC190E00E9469CC41E070E0B4
:104B400060E08AE20E946CC1992091F080916E0E23
:104B5000882371F060E97BE082E791E10E9472D1E5
:104B600070E060E08AE20E943AC190E00E9469CC65
:104B700040E070E060E08AE20E946CC1992091F010
:104B800080916E0E882371F063E77BE082E791E10C
:104B90000E9472D170E060E08AE20E943AC190E027
:104BA0000E9469CC41E066E070E087E20E946CC13F
:104BB00041E065E070E087E20E946CC141E064E0A2
:104BC00070E087E20E946CC140E062E070E087E242
:104BD0000E946CC140E061E070E087E20E946CC11D
:104BE00040E070E060E087E20E946CC1992009F427
:104BF00075C080916E0E882309F470C06BE57BE070
:104C000082E791E10E9472D166E070E08BE20E943F
:104C10003AC190E00E9469CC6DE37BE082E791E1CC
:104C20000E9472D165E070E08BE20E943AC190E090
:104C30000E9469CC6FE17BE082E791E10E9472D132
:104C400064E070E08BE20E943AC190E00E9469CC7F
:104C500066E07BE082E791E10E9472D162E070E061
:104C60008BE20E943AC190E00E9469CC6DEE7AE03E
:104C700082E791E10E9472D161E070E08BE20E94D4
:104C80003AC190E00E9469CC64ED7AE082E791E15C
:104C90000E9472D170E060E08BE20E943AC190E025
:104CA0000E9469CC61EC7AE082E791E10E9472D1C6
:104CB00063E070E08BE20E943AC190E00E9469CC10
:104CC0006CEA7AE082E791E10E9472D164E070E0E0
:104CD0008CE20E943AC190E00E9469CC40E064E01E
:104CE00070E08CE20E946CC1AE014B5D5F4F61E0F1
:104CF00070E08CE20E94FBC06DA1607F66608CE278
:104D00000E9455C1992009F45EC080916E0E8823DF
:104D100009F459C068E97AE082E791E10E9472D112
:104D2000AE014B5D5F4F61E070E08CE20E94FBC022
:104D30006DA16F706650770B072E000C880B990BD6
:104D40000E94C8DE9B01AC0160E070E080E090E46E
:104D50000E9414E320E030E048EC50E40E9427DF9A
:104D60000E9420CC61E87AE082E791E10E9472D152
:104D7000AE014B5D5F4F61E070E080E30E94FBC0DD
:104D80006DA14AE050E082E791E10E940CCB69E618
:104D90007AE082E791E10E9472D161E070E080E305
:104DA0000E943AC190E00E9469CC60E57AE082E717
:104DB00091E10E9472D161E070E08FE20E943AC1FD
:104DC00090E00E9469CC41E061E070E08FE20E94D7
:104DD0006CC1992091F080916E0E882371F068E388
:104DE0007AE082E791E10E9472D161E070E08EE2A8
:104DF0000E943AC190E00E9469CC41E061E070E01D
:104E00008EE20E946CC140E067E070E081E30E94A6
:104E10006CC1992009F455C080916E0E882309F465
:104E200050C065E27AE082E791E10E9472D167E0CA
:104E300070E081E30E943AC190E00E9469CC67E390
:104E400076E082E791E10E947CCCAE014B5D5F4F42
:104E500061E070E080E00E94FBC08DA10E94C971FA
:104E600061E37CE082E791E10E9423CB0DE110E059
:104E700069E679E082E791E10E947CCC40E150E074
:104E8000B80182E791E10E942FCC6BE376E082E7E4
:104E900091E10E947CCCAE014B5D5F4F61E070E020
:104EA000802F0E94FBC08DA10E94C97161E37CE04C
:104EB00082E791E10E9423CB0F5F1F4F0A33110558
:104EC000B9F6A9960FB6F894DEBF0FBECDBFDF913D
:104ED000CF911F910F91FF90EF90DF90CF90BF90F7
:104EE000AF909F907F906F905F904F9008956FEA82
:104EF00080E20E9400C260E081E20E9400C268E09D
:104F000082E20E9400C260E283E20E9400C289E263
:104F10009CE5AFE8BDE38093A80E9093A90EA09303
:104F2000AA0EB093AB0E60E084E20E9400C2043689
:104F3000110509F43FCA11E0992009F43CCA68E55B
:104F40007EE0CE0101960E94B1C8CE0101960E947A
:104F50004013CE0101960E9457C889E60E94DFAC3B
:104F600063E289EC94E10E946C6B89EC94E10E940D
:104F7000887389E60E94DFAC41E050E069E670E0AA
:104F800089EC94E10E94D47390914A0F80914B0F69
:104F90009817F1F30E9427AD8C0189EC94E10E94EF
:104FA0008873C80124E0959587952A95E1F7837069
:104FB000992768E47EE08130910559F06FE37EE047
:104FC0008230910531F060E57EE0892B11F067E3D6
:104FD0007EE0CE0101960E94B1C8CE0101960E94EA
:104FE0002313CE0101960E9457C8192DE4C965E626
:104FF0007EE0CE0101960E94B1C8CE0101960E94CA
:105000002313CE0101960E9457C864EF71E080E03F
:1050100090E00E94FF6C0F5F1F4F6AC94F925F9232
:105020006F927F928F929F92AF92BF92CF92DF92B8
:10503000EF92FF921F93CF93DF93CDB7DEB72C97FC
:105040000FB6F894DEBF0FBECDBF182F8091890D2B
:105050008111D2C080E492E090930F0280930E02FF
:105060000E94886D8093CC1581E492E00E94886D47
:105070008093CD1582E492E00E94886D8093CE15D6
:1050800083E492E00E94886D8093CF1580E492E0E3
:105090000E94886D8F3FE1F0E0900E02F0900F02C9
:1050A00030EDA32E35E1B32E6501C7018C5C95412F
:1050B0004C0124EDC21625E1D20609F441C0C40119
:1050C0008C0D9D1D0E94886DF60181936F01F1CFBB
:1050D00081E492E00E94886D8F3FF1F682E492E0D5
:1050E0000E94886D8F3FC1F683E492E00E94886D34
:1050F0008F3F91F680E090E0A0E8BFE38093CC156D
:105100009093CD15A093CE15B093CF152CECC22E55
:1051100025E1D22EF12CE12C80910E0290910F020C
:10512000E4E0EE16F10409F4B7CFF60161916F01E6
:105130008E0D9F1D0E94F0DFFFEFEF1AFF0AECCFEC
:10514000C70104960E94886D8F3F99F5C7010596A7
:105150000E94886D8F3F69F5C70106960E94886D91
:105160008F3F39F5C70107960E94886D8F3F09F57B
:1051700080E090E0A0E8BFE38093D0159093D11534
:10518000A093D215B093D315F12CE12CF5016191C8
:105190005F0180910E0290910F0204968E0D9F1D6B
:1051A0000E94F0DFFFEFEF1AFF0A24E0E216F1049D
:1051B00069F78091CC159091CD15A091CE15B09145
:1051C000CF158093C8159093C915A093CA15B093B5
:1051D000CB150E94326D6093850D7093860D809380
:1051E000870D9093880D81E08093890D68EE73E0C0
:1051F00080E090E00E94FF6C80917D0D81110DC0D8
:105200000E94326D6093790D70937A0D80937B0DBF
:1052100090937C0D81E080937D0D0E94326DC09053
:10522000790DD0907A0DE0907B0DF0907C0D6C198B
:105230007D098E099F09693E73408105910508F437
:105240004BC10E94326D6093790D70937A0D8093FB
:105250007B0D90937C0D8BE30E94B76CBC01990F82
:10526000880B990B0E94C8DE20E030E040E85AE34A
:105270000E9427DF20E030E44CE955E40E9427DF5C
:105280006B017C01C092750DD092760DE092770D86
:10529000F092780D87E390E00E94370F4B015C019C
:1052A0008092100290921102A0921202B092130208
:1052B00020E030E04AE754E4C701B6010E9427DF4E
:1052C00020E030E04DE454E40E9440E120E030E092
:1052D00048E453E40E9440E16B017C01C092DC157C
:1052E000D092DD15E092DE15F092DF152091C81501
:1052F0003091C9154091CA155091CB150E9427DFF6
:105300002B013C0120E030E040E250E40E9449E201
:1053100018160CF02AC18091D0159091D115A0914A
:10532000D215B091D3158093C8159093C915A09349
:10533000CA15B093CB152091C8153091C91540916D
:10534000CA155091CB15C701B6010E9427DF6B012A
:105350007C0120E030E048EC51E4C501B4010E943A
:1053600061E020E53DE847E95CE30E9427DF20E0BB
:1053700030E040E85FE30E9462E09B01AC01C701BE
:10538000B6010E9440E1AB01BC014093C4155093AB
:10539000C5156093C6157093C71522E0CE01079618
:1053A0000E945FC86EE376E0CE0101960E94C3C8FA
:1053B000BE01695F7F4FCE0101960E9434C762E44F
:1053C00076E00E941EC7BC0188E894E10E94FBC7FA
:1053D000CE0101960E9457C8CE0107960E9457C879
:1053E00040911002509111026091120270911302CB
:1053F00021E0CE0107960E945FC86DEB76E0CE01FA
:1054000001960E94C3C8BE01695F7F4FCE0101961D
:105410000E9434C7BC0184E994E10E94FBC7CE011D
:1054200001960E9457C8CE0107960E9457C868E8A7
:1054300074E1CE0101960E94BAC86EE277E0CE0117
:1054400001960E941EC764E974E10E9434C768E4B3
:1054500076E00E941EC7BC018EE894E10E94FBC763
:10546000CE0101960E9457C864E974E1CE0101960D
:105470000E94BAC84AE050E06FEF7FEFCE0101967C
:105480000E94151ACE0101960E9457C865E070E08F
:1054900080E090E00E94FF6C62E079E0CE0101962E
:1054A0000E94C3C8CE0101960E941B10CE01019636
:1054B0000E9457C868E874E1CE0101960E94BAC8FC
:1054C0004AE050E06FEF7FEFCE0101960E947B1320
:1054D000CE0101960E9457C80E94326DC090850D82
:1054E000D090860DE090870DF090880D6C197D09A5
:1054F0008E099F096235734081059105E0F00E9495
:10550000326D6093850D7093860D8093870D909317
:10551000880D87E390E00E94370F6093100270932C
:10552000110280931202909313026EE170E080E00A
:1055300090E00E94FF6C11112BC010E0812F2C967F
:105540000FB6F894DEBF0FBECDBFDF91CF911F9194
:10555000FF90EF90DF90CF90BF90AF909F908F9093
:105560007F906F905F904F90089520E030E040E092
:1055700050E4C301B2010E94C1DE87FFDCCE8091FE
:10558000CC159091CD15A091CE15B091CF15CBCE65
:105590008090100290901102A0901202B09013021D
:1055A0004090750D5090760D6090770D7090780D4D
:1055B0004092D4155092D5156092D6157092D71599
:1055C0008092D8159092D915A092DA15B092DB1579
:1055D000123059F0133009F431C1113009F0ADCF58
:1055E0001093740D1092730DA9CF8091740D8823C0
:1055F00009F4A3CFC090DC15D090DD15E090DE1546
:10560000F090DF1526E636E646E65FE3C701B60111
:105610000E9449E218160CF0B3C023E333E343EFD2
:105620005FE3C701B6010E94C1DE87FFA9C020E089
:1056300030E048EC51E4C501B4010E9461E020E58E
:105640003DE847E95CE30E9427DF20E030E040E8E6
:105650005FE30E9462E02FE23DED44EB5FE30E94D6
:1056600027DF60936F0D7093700D8093710D909391
:10567000720D20E038E240E258E460916F0D7091C5
:10568000700D8091710D9091720D0E9427DF20E0C6
:1056900030E04AE754E40E9440E1A30192010E94F5
:1056A00040E14B015C0120E030E040E05FE30E941C
:1056B00049E218160CF0B0C020E030E040EC5FE3A7
:1056C000C501B4010E94C1DE87FFA6C08092C81543
:1056D0009092C915A092CA15B092CB1526E636E66F
:1056E00046E65FE3C701B6010E9449E218160CF0D6
:1056F00075C023E333E343EF5FE3C701B6010E94C4
:10570000C1DE87FF6BC08092CC159092CD15A09220
:10571000CE15B092CF1581E08093730D66E373E1EF
:10572000CE0101960E94B1C8CE0101960E9440139D
:10573000CE0101960E9457C84091C8155091C915D5
:105740006091CA157091CB1523E0CE0101960E949D
:105750005FC8CE0101960E942313CE0101960E94DC
:1057600057C869E173E1CE0101960E94B1C8CE012C
:1057700001960E942313CE0101960E9457C8DECEE7
:1057800020E030E040E151E4C701B6010E9449E267
:1057900018160CF06ECF26E636E646E851E4C7014F
:1057A000B6010E94C1DE87FF64CF20E030E048EC04
:1057B00051E4C501B4010E9461E020E53DE847E9FC
:1057C0005CE30E9427DF20E030E040E85FE30E94D6
:1057D00062E02BE734E14EE451E441CF20E030E0D9
:1057E00040E151E4C701B6010E9449E218160CF0ED
:1057F00092CF26E636E646E851E4C701B6010E949C
:10580000C1DE87FF88CF8092D0159092D115A092EB
:10581000D215B092D3157FCF1092730D64E673E169
:10582000CE0101960E94B1C8CE0101960E942313B9
:10583000CE0101960E9457C815E180CE8091740D6B
:10584000882309F47ACE82E791E10E9408CB809107
:10585000730D882309F47DC0C090DC15D090DD1550
:10586000E090DE15F090DF1526E636E646E65FE3CB
:10587000C701B6010E9449E21816ECF523E333E3B1
:1058800043EF5FE3C701B6010E94C1DE87FF33C06B
:105890009CECC92E95E1D92EF12CE12CF6016191F9
:1058A0006F0180910E0290910F028E0D9F1D0E943C
:1058B000F0DFFFEFEF1AFF0A24E0E216F10471F7C0
:1058C0001092730D1092740D1A3008F444C06DE4F8
:1058D00073E11E3109F032CECE0101960E94B1C8AB
:1058E000CE0101960E942313CE0101960E9457C853
:1058F0001092930D23CE20E030E040E151E4C70147
:10590000B6010E9449E21816DCF626E636E646E8BD
:1059100051E4C701B6010E94C1DE87FFD1CF80EDFF
:10592000C82E85E1D82EF12CE12CF60161916F0192
:1059300080910E0290910F0204968E0D9F1D0E9481
:10594000F0DFFFEFEF1AFF0A24E0E216F10469F737
:10595000B7CF1EE1B5CF133009F0F0CD6EEF72E195
:10596000BBCF8F929F92AF92BF92CF92DF92EF9276
:10597000FF920F931F93CF93DF93CDB7DEB72C9792
:105980000FB6F894DEBF0FBECDBFD82E0DB71EB731
:105990008091630D811105C00E94326D81E080937A
:1059A000630D80915B0D811105C00E94326D81E015
:1059B00080935B0D8091530D811105C00E94326D63
:1059C00081E08093530D60E08D2D0E94776C64E63A
:1059D00070E080E090E00E94FF6C1092520D1092F7
:1059E000510DE090510DF090520D4EE1E416F1048E
:1059F000D4F48D2D0E94B76CF701EE0FFF1FEB5E04
:105A0000F24F918380836EE170E080E090E00E942D
:105A1000FF6C8091510D9091520D01969093520D13
:105A20008093510DDECF87E390E00E94370F6093A3
:105A30008504709386048093870490938804E5E13D
:105A4000FDE027ED3CE0D9018DE0E135F80729F0D4
:105A5000819191918D939D93F7CF8EE190E09093FA
:105A6000140D8093130DADB6BEB6ADB7BEB7DC97BF
:105A70000FB6F894BEBF0FBEADBFEDB7FEB73196FF
:105A80004F01DF0180E0F901619171919F016D93F8
:105A90007D938F5F8E31B9F78DE190E0F40130E0B6
:105AA00020E0281739079CF4619171912F5F3F4FD7
:105AB000E080F180E616F706A4F76F0142E0C41A11
:105AC000D108D601ED92FC9271836083EACF0197F1
:105AD00029F7F401668D778D848D958D680F791F78
:105AE00077FF02C06F5F7F4F759567950FB6F8948B
:105AF000BEBE0FBEADBE072E000C880B990B0E94D8
:105B0000C8DE20E030E44CE955E40E9427DF20E0C5
:105B100030EC4FE754E40E9440E16B017C01C092FD
:105B20008D0DD0928E0DE0928F0DF092900D20E0B1
:105B300030E040E05FE36091C30D7091C40D80914F
:105B4000C50D9091C60D0E9462E00E94ECE1FB0140
:105B5000EE0FFF1FEE0FFF1FE65AFD4E2591359108
:105B600045915491C701B6010E9427DF2091C70DCE
:105B70003091C80D4091C90D5091CA0D0E9440E16D
:105B8000AB01BC0140936B0D50936C0D60936D0D98
:105B900070936E0D22E0CE0107960E945FC868E503
:105BA00076E0CE0101960E94C3C8BE01695F7F4FB7
:105BB000CE0101960E9434C76CE576E00E941EC7B4
:105BC000BC0188E894E10E94FBC7CE0101960E94C7
:105BD00057C8CE0107960E9457C84091850450913E
:105BE0008604609187047091880421E0CE010796B5
:105BF0000E945FC86DEB76E0CE0101960E94C3C89B
:105C0000BE01695F7F4FCE0101960E9434C7BC017F
:105C100084E994E10E94FBC7CE0101960E9457C817
:105C2000CE0107960E9457C868E874E1CE0101963C
:105C30000E94BAC864E974E1CE0101960E9434C79B
:105C400062E676E00E941EC7BC018EE894E10E94E5
:105C5000FBC7CE0101960E9457C864E974E1CE01EA
:105C600001960E94BAC84AE050E070E060E0CE01C0
:105C700001960E94151ACE0101960E9457C865E050
:105C800070E080E090E00E94FF6C62E079E0CE017D
:105C900001960E94C3C8CE0101960E941B10CE013E
:105CA00001960E9457C868E874E1CE0101960E94EF
:105CB000BAC84AE050E06FEF7FEFCE0101960E9434
:105CC0007B13CE0101960E9457C80FB6F8941EBFF1
:105CD0000FBE0DBF2C960FB6F894DEBF0FBECDBF22
:105CE000DF91CF911F910F91FF90EF90DF90CF90B8
:105CF000BF90AF909F908F9008952F923F924F92B8
:105D00005F926F927F928F929F92AF92BF92CF924B
:105D1000DF92EF92FF920F931F93CF93DF93CDB754
:105D2000DEB768970FB6F894DEBF0FBECDBF2B016C
:105D30003C010E94326D6D877E878F87988B88E348
:105D400090E10E94DCB062E370E080E090E00E94AD
:105D5000FF6C61E08091A6040E94776C60E0809106
:105D6000A4040E94776C64E670E080E090E00E94FA
:105D7000FF6C6091A0047091A1048091A2049091A5
:105D8000A3040E94A3100E94C70F7B018C010E94F4
:105D9000DA6C4B015C0160E570E080E090E00E940D
:105DA000FF6C62E776E08EE894E10E949AC520E0FD
:105DB00030E04AE754E4C301B2010E9427DF6D8B53
:105DC0007E8B8F8B988F412C512C320160E070E0DC
:105DD000CB010E94C8DE2D893E894F89588D0E94D3
:105DE000C1DE87FF87C10E94326D2D853E854F85BC
:105DF0005889621B730B840B950B0E94C6DE20E052
:105E000030E04AE754E40E9440E1AB01BC0123E0EA
:105E1000CE0101960E945FC8BE016F5F7F4F88E888
:105E200094E10E9412C8CE0101960E9457C80E94B8
:105E3000C70FD62EC72E382E292E0E94DA6C698BFA
:105E40007A8B8B8B9C8BDC01CB0188199909AA0971
:105E5000BB094C015D0191ED891697E09906A104FB
:105E6000B104BCF020E030E0A9016D2D7C2D832D24
:105E7000922D0E9449E2181684F426EA3BE944EC8C
:105E80005BE36D2D7C2D832D922D0E94C1DE87FF5B
:105E900010C0812C912C54012EC026EA3BE944EC21
:105EA0005BEB6D2D7C2D832D922D0E9449E21816FF
:105EB00084F3C501B40128EE33E040E050E00E94D5
:105EC000FEDFCA01B9010E94C8DE4B015C019701E7
:105ED000A8016D2D7C2D832D922D0E9461E020E084
:105EE00030E04AE754E40E9427DFA50194010E94B4
:105EF00040E14B015C0168E874E1CE0101960E942B
:105F0000BAC865E577E0CE0101960E941EC7BC01C4
:105F100088E894E10E94FBC7CE0101960E9457C811
:105F200023E04D2D5C2D632D722DCE0101960E9434
:105F30005FC8BE016F5F7F4FCE0107960E94BAC84F
:105F400060E976E0CE0107960E941EC7BC0182E898
:105F500094E10E94FBC7CE0107960E9457C8CE016C
:105F600001960E9457C822E0B501A401CE01079610
:105F70000E945FC86BEB77E0CE0101960E94C3C818
:105F800068E874E1CE0101960E9434C763E976E0C7
:105F90000E941EC762E874E10E9434C76FE278E095
:105FA0000E941EC7BE01695F7F4F0E9434C767E928
:105FB00076E00E941EC7BC018EE894E10E94CFC724
:105FC000CE0101960E9457C8CE0107960E9457C87D
:105FD00020E030E0A901C501B4010E9449E287FD3B
:105FE00006C06EE277E082E894E10E94C5C722E035
:105FF000B501A401CE0101960E945FC8BE016F5F8A
:106000007F4FCE0107960E94BAC867E976E0CE01BD
:1060100007960E941EC7BC0182E894E10E94CFC788
:10602000CE0107960E9457C8CE0101960E9457C81C
:106030006EE874E1CE0101960E94BAC8CE010196C5
:106040000E942313CE0101960E9457C8C301B201DA
:1060500025E030E040E050E00E94FEDF672B682B37
:10606000692B21F56EE47FE0CE0101960E94B1C854
:1060700045E050E070E060E0CE0101960E94151A04
:10608000CE0101960E9457C862E874E1CE010196E4
:106090000E94BAC845E050E06FEF7FEFCE01019655
:1060A0000E947B13CE0101960E9457C861E37CE0F9
:1060B0008EE894E10E949AC562E370E080E090E08F
:1060C0000E94FF6C0E94326D2D853E854F85588958
:1060D000621B730B840B950B3FEF431A530A630A41
:1060E000730A89889A88AB88BC88ED2CFC2C032D18
:1060F000122D6FCE60E08091A6040E94776C6896A6
:106100000FB6F894DEBF0FBECDBFDF91CF911F91C8
:106110000F91FF90EF90DF90CF90BF90AF909F9046
:106120008F907F906F905F904F903F902F90089549
:106130008F929F92AF92BF92CF92DF92EF92FF9297
:106140000F931F93CF93DF93CDB7DEB7EA970FB6C8
:10615000F894DEBF0FBECDBFF82E61E37CE0CE0128
:10616000C5960E94C3C88E010B5E1F4F6F2DC801DC
:106170000E94AD7018870F831D821E82198289E0EC
:106180008A8381E08B838C831C8A1B8ACE010196D3
:106190000E940270CE0101960E94A56ECE0101966A
:1061A0000E94D3C20E8110E00330110509F488C1AA
:1061B00064E47FE0CE01C5960E94D6C761E37CE02F
:1061C0008EE894E10E949AC5BE016B5C7F4FCE01C0
:1061D00083960E94BAC84AE050E070E060E0CE01C9
:1061E00083960E94151ACE0183960E9457C861E0DB
:1061F00080E00E94FAAC6DEB76E0CE01C5960E947D
:106200009AC584EEC82E8DE0D82EF12CE12CE01634
:10621000F1060CF0F0C06E2DCE0101960E94966F33
:10622000F60121913191419151916F010E9462E0FB
:106230004B015C01FFEFEF1AFF0A20E030E04CEF6A
:1062400052EC0E94C1DE87FF33C0B701CE018996B0
:106250000E94D1C565EB7AE0CE0183960E94C3C847
:10626000BE01675D7F4FCE0183960E9434C76BE904
:1062700076E00E941EC7BC018EE894E10E94CFC761
:10628000CE0183960E9457C8CE0189960E9457C8B6
:106290000130110509F055C081E0E816F10409F05C
:1062A000B6CF6EE874E1CE01C5960E94FBC7AFCFB2
:1062B00022E0B501A401CE018F960E945FC8B7010C
:1062C000CE0189960E94D1C565EB7AE0CE01839616
:1062D0000E94C3C8BE01675D7F4FCE0183960E94B6
:1062E00034C76BE176E00E941EC7BE01615D7F4F3F
:1062F0000E9434C7BC0182E894E10E94FBC7CE0132
:1063000083960E9457C8CE0189960E9457C8CE0135
:106310008F960E9457C862E874E1CE0183960E946E
:10632000BAC86EE277E0CE0183960E941EC7BC0118
:106330008EE894E10E94CFC7CE0183960E9457C891
:10634000A7CF0230110511F522E0B501A401CE015D
:1063500083960E945FC8BE016D5D7F4FCE01899616
:106360000E94BAC86EE277E0CE0189960E941EC7ED
:10637000BC01CE01C5960E94CFC7CE0189960E946E
:1063800057C8CE0183960E9457C841CF03301105EC
:1063900009F43DCF62E874E1CE0183960E94BAC849
:1063A00044E150E06FEF7FEFCE0183960E947B13B4
:1063B000CE0183960E9457C862E079E0CE018396B1
:1063C0000E94C3C8CE0183960E941B10CE01839603
:1063D0000E9457C880919D04882309F418CF8091AA
:1063E000FB04882309F413CF60ED77E080E090E0B0
:1063F0000E94FF6C0CCFCE01C5960E9422C68EE88B
:1064000094E10E9422C60115110579F561E37FE050
:106410008EE894E10E94D6C766E27FE0CE018396C3
:106420000E94B1C84AE050E06FEF7FEFCE01839643
:106430000E947B13CE0183960E9457C8CE01C59659
:106440000E9457C8EA960FB6F894DEBF0FBECDBFC4
:10645000DF91CF911F910F91FF90EF90DF90CF9040
:10646000BF90AF909F908F900895043011050CF568
:10647000BE016B5C7F4FCE0183960E94BAC84AE092
:1064800050E06FEF7FEFCE0183960E947B13CE0129
:1064900083960E9457C862E079E0CE0183960E94FD
:1064A000C3C8CE0183960E941B10CE0183960E9422
:1064B00057C867EA76E08EE894E10E94C5C7BECF70
:1064C0006AEB76E0CE01C5960E949AC5BE016B5C70
:1064D0007F4FCE0183960E94BAC84AE050E070E038
:1064E00060E0CE0183960E94151ACE0183960E9429
:1064F00057C861E37CE08EE894E10E949AC56EE89B
:1065000074E1CE01C5960E94FBC710E000E0602F49
:10651000CE0101960E94966F6B017C0122E0BC01C6
:10652000A601CE0183960115110509F077C00E94DE
:106530005FC8BE016D5D7F4F86E196E10E9452D13A
:10654000CE0183960E9457C822E0B701A601CE0172
:1065500083960E945FC8BE016D5D7F4FCE01899614
:106560000E94BAC86EE277E0CE0189960E941EC7EB
:10657000BC018EE894E10E94CFC7CE0189960E94AB
:1065800057C8CE0183960E9457C80F5F1F4F033034
:10659000110509F0BCCFCE01C5960E9422C6BE01EE
:1065A0006B5C7F4FCE0183960E94BAC84AE050E0F0
:1065B0006FEF7FEFCE0183960E947B13CE0183960F
:1065C0000E9457C862E079E0CE0183960E94C3C85A
:1065D000CE0183960E941B10CE0183960E9457C85D
:1065E0008EE894E10E9422C660EC76E0CE018396AC
:1065F0000E94C3C86EE874E1CE0183960E9434C73E
:1066000067EA76E00E941EC7BC018EE894E10E9412
:10661000FBC7CE0183960E9457C810CF0E945FC867
:10662000BE016D5D7F4FCE0189960E94BAC86EE2B1
:1066300077E0CE0189960E941EC7BC01CE01C596A7
:106640000E94CFC7CE0189960E9457C879CFAF92DA
:10665000BF92CF92DF92EF92FF920F931F93CF934F
:10666000DF93CDB7DEB72C970FB6F894DEBF0FBE21
:10667000CDBF80916D0E811102C00E945713809191
:10668000A9049091AA04029751F08091E20D909193
:10669000E30D009709F4BAC1039709F4B7C169EB98
:1066A0007EE088E894E10E94D6C768E874E1CE01F4
:1066B00001960E94BAC844E150E070E060E0CE016B
:1066C00001960E94151ACE0101960E9457C86AEAE7
:1066D0007EE088E894E10E94D6C768E874E1CE01C4
:1066E00001960E94BAC844E150E06FEF7FEFCE01FF
:1066F00001960E947B13CE0101960E9457C887E045
:106700000E942EC28C0186E00E942EC2BC0190E045
:1067100080E00E94C6DE2AE037ED43EA5CE30E9497
:1067200027DF23E333E948E853E40E9461E06B018B
:106730007C0184E0A82EB12C20E030E048EC52E44B
:10674000C701B6010E9449E218160CF05FC081E053
:10675000A81AB108E9F064E670E080E090E00E94D9
:10676000FF6C86E00E942EC2BC0190E080E00E9497
:10677000C6DE2AE037ED43EA5CE30E9427DF23E32D
:1067800033E948E853E40E9461E06B017C01D4CF17
:106790006FE97EE088E894E10E94D6C768E874E17A
:1067A000CE0101960E94BAC84AE050E070E060E075
:1067B000CE0101960E94151ACE0101960E9457C87B
:1067C0006AEC76E0CE0101960E94C3C868E874E1E5
:1067D000CE0101960E9434C7BC018EE894E10E946C
:1067E000FBC7CE0101960E9457C88091E20D90919F
:1067F000E30D049721F41092E30D1092E20D81E075
:1068000090E09093AA048093A904DFC0B80190E0BF
:1068100080E00E94C6DE2AE037ED43EA5CE30E9496
:1068200027DF23E333E948E853E40E9461E0AB014A
:10683000BC0121E0CE0101960E945FC86CED76E0BC
:10684000CE0107960E94C3C8BE016F5F7F4FCE0185
:1068500007960E9434C7BC018EE894E10E94FBC7F2
:10686000CE0107960E9457C8CE0101960E9457C8D4
:1068700083E090E09093E30D8093E20D6EE874E185
:10688000CE0101960E94BAC842E350E06FEF7FEF5D
:10689000CE0101960E947B13CE0101960E9457C83B
:1068A00062E079E0CE0101960E94C3C8CE01019654
:1068B0000E941B10CE0101960E9457C865EE76E03B
:1068C0008EE894E10E94C5C721E0B701A601CE0180
:1068D00001960E945FC86DEB76E0CE0107960E949C
:1068E000C3C8BE016F5F7F4FCE0107960E9434C7B9
:1068F000BC0184E994E10E94FBC7CE0107960E9487
:1069000057C8CE0101960E9457C86EE277E0CE01CB
:1069100001960E94C3C864E974E1CE0101960E9409
:1069200034C7BC0188E894E10E94FBC7CE01019600
:106930000E9457C868E874E1CE0101960E94BAC867
:106940004AE050E070E060E0CE0101960E945C19E0
:10695000CE0101960E9457C862E079E0CE0101960F
:106960000E94C3C8CE0101960E941B10CE01019661
:106970000E9457C865EE76E084E994E10E94C5C79D
:1069800064E974E1CE0101960E94BAC86EE277E034
:10699000CE0101960E941EC76EE874E10E9434C7C2
:1069A000BC018EE894E10E94FBC7CE0101960E94D3
:1069B00057C88091E20D9091E30D039731F484E084
:1069C00090E09093E30D8093E20D64E670E080E048
:1069D00090E00E94FF6C80916D0E882331F060E2A0
:1069E00073E080E090E00E94FF6C2C960FB6F89464
:1069F000DEBF0FBECDBFDF91CF911F910F91FF90F2
:106A0000EF90DF90CF90BF90AF90089588E390E132
:106A10000E94DCB064E670E080E090E00E94FF6CD1
:106A20006FED7EE088E894E10E94D6C768E874E1E3
:106A3000CE0101960E94BAC844E150E070E060E0E7
:106A4000CE0101960E94151ACE0101960E9457C8E8
:106A500060ED7EE088E894E10E94D6C768E874E1C2
:106A6000CE0101960E94BAC844E150E06FEF7FEF7B
:106A7000CE0101960E947B13CE0101960E9457C859
:106A80008CE40E94FAB06B017C0104E010E0A701E5
:106A90009601C701B6010E94AEE3882309F449C0FC
:106AA0000150110961F068EC70E080E090E00E9414
:106AB000FF6C8CE40E94FAB06B017C01E8CF65ECBE
:106AC0007EE088E894E10E94D6C768E874E1CE01D0
:106AD00001960E94BAC84AE050E070E060E0CE0142
:106AE00001960E94151ACE0101960E9457C86AECC1
:106AF00076E0CE0101960E94C3C868E874E1CE0139
:106B000001960E9434C7BC018EE894E10E94FBC745
:106B1000CE0101960E9457C88091E20D9091E30D3D
:106B2000039721F41092E30D1092E20D82E090E0C1
:106B300068CE21E0B701A601CE0107960E945FC88A
:106B40006CED76E0CE0101960E94C3C8BE01695F7C
:106B50007F4FCE0101960E9434C7BC018EE894E1BC
:106B60000E94FBC7CE0101960E9457C8CE0107962E
:106B70000E9457C883E090E09093E30D8093E20D6C
:106B80006EE874E1CE0101960E94BAC842E350E07B
:106B90006FEF7FEFCE0101960E947B13CE0101962D
:106BA0000E9457C862E079E0CE0101960E94C3C8F6
:106BB000CE0101960E941B10CE0101960E9457C87B
:106BC00065EE76E08EE894E10E94C5C786E60E94F5
:106BD000FAB06B017C0104E010E0A7019601C70147
:106BE000B6010E94AEE3882381F00150110909F437
:106BF00084C068EC70E080E090E00E94FF6C86E664
:106C00000E94FAB06B017C01E8CF21E0B701A60138
:106C1000CE0107960E945FC86DEB76E0CE0101962B
:106C20000E94C3C8BE01695F7F4FCE0101960E94DA
:106C300034C7BC0184E994E10E94FBC7CE010196F0
:106C40000E9457C8CE0107960E9457C86EE277E0AF
:106C5000CE0101960E94C3C864E974E1CE01019699
:106C60000E9434C7BC0188E894E10E94FBC7CE01B2
:106C700001960E9457C868E874E1CE0101960E940F
:106C8000BAC84AE050E06FEF7FEFCE0101960E9454
:106C90005C19CE0101960E9457C862E079E0CE01EE
:106CA00001960E94C3C8CE0101960E941B10CE011E
:106CB00001960E9457C865EE76E084E994E10E944F
:106CC000C5C764E974E1CE0101960E94BAC86EE2BC
:106CD00077E0CE0101960E941EC76EE874E10E9423
:106CE00034C7BC018EE894E10E94FBC7CE01019637
:106CF0000E9457C883E090E064CE61E37CE084E9C1
:106D000094E10E949AC5DDCF4F925F926F927F927D
:106D10008F929F92AF92BF92CF92DF92EF92FF92AB
:106D2000CF93DF93CDB7DEB72C970FB6F894DEBFC5
:106D30000FBECDBF0E9457130E9423B22B013C010E
:106D40000E94EAB34B015C016091EB047091EC048A
:106D50008091ED049091EE040E94C8DE6B017C01ED
:106D60000E9423B20E94C8DEA70196010E9440E162
:106D700021E03EED42E45EE30E9414E39B01AC019E
:106D800060E070E080E89FE30E9461E020E03AE28A
:106D90004DE257E40E9427DF6B017C01C301B20181
:106DA0000E94C8DE20E030E048EC52E40E9440E15E
:106DB000AB01BC0122E0CE0101960E945FC8BE017A
:106DC0006F5F7F4F82E894E10E9412C8CE01019666
:106DD0000E9457C863EC79E082E894E10E94C5C73D
:106DE00062E874E188E894E10E94FBC76FEB79E008
:106DF000CE0101960E94C3C862E874E1CE010196FB
:106E00000E9434C7BC0182E894E10E94FBC7CE0116
:106E100001960E9457C86DEB76E08EE894E10E94DF
:106E20009AC521E0B501A401CE0101960E945FC878
:106E3000BE016F5F7F4F8EE894E10E94CFC7CE0105
:106E400001960E9457C868EE76E08EE894E10E94B1
:106E5000C5C721E0B701A601CE0101960E945FC817
:106E6000BE016F5F7F4FCE0107960E94BAC868E4EB
:106E700078E0CE0107960E941EC7BC018EE894E11F
:106E80000E94CFC7CE0107960E9457C8CE01019637
:106E90000E9457C862E874E1CE0101960E94BAC808
:106EA0006EE277E0CE0101960E941EC76EE874E1A3
:106EB0000E9434C7BC018EE894E10E94FBC7CE015A
:106EC00001960E9457C821E0B501A401CE010196A8
:106ED0000E945FC8BE016F5F7F4F84E994E10E940A
:106EE00012C8CE0101960E9457C864E974E1CE0130
:106EF00001960E94BAC84AE050E070E060E0CE011E
:106F000001960E94151ACE0101960E9457C865E0AD
:106F100070E080E090E00E94FF6C62E079E0CE01DA
:106F200001960E94C3C8CE0101960E941B10CE019B
:106F300001960E9457C868E874E1CE0101960E944C
:106F4000BAC84AE050E06FEF7FEFCE0101960E9491
:106F50007B13CE0101960E9457C820E0B701A6011D
:106F6000CE0101960E945FC8BE016F5F7F4FCE01C8
:106F700007960E94BAC868E478E0CE0107960E949E
:106F80001EC7BC0184E994E10E94FBC7CE010796AD
:106F90000E9457C8CE0101960E9457C864E974E167
:106FA000CE0101960E94BAC84AE050E064EF7FEF3C
:106FB000CE0101960E947B13CE0101960E9457C814
:106FC00065E070E080E090E00E94FF6C80916D0EC3
:106FD000882331F068E572E080E090E00E94FF6C69
:106FE0002C960FB6F894DEBF0FBECDBFDF91CF91C8
:106FF000FF90EF90DF90CF90BF90AF909F908F90D9
:107000007F906F905F904F900895CF92DF92EF92B4
:10701000FF920F931F93CF93DF93CDB7DEB7E09727
:107020000FB6F894DEBF0FBECDBF8E01015E1F4FBD
:107030008130910509F0B7C06EEE76E0CE01019681
:107040000E94C3C861EF76E0CE0107960E94C3C8D4
:1070500064EF76E0CE010D960E94C3C86CE472E145
:10706000C8010E94B1C844E650E06FEF7FEFC8014D
:107070000E94151AC8010E9457C861E472E18CEAA7
:1070800094E10E94D6C76091F0047091F104CE01A2
:1070900085960E94D1C56CEA74E1C8010E94BAC805
:1070A000BE016B5D7F4FC8010E9434C7BC01CE0199
:1070B0008B960E94BAC840ED57E06FEF7FEFCE018C
:1070C0008B960E947B13CE018B960E9457C8C801F5
:1070D0000E9457C8CE0185960E9457C862E372E1AC
:1070E000C8010E94B1C844E650E06FEF7FEFC801CD
:1070F0000E94151AC8010E9457C867EF76E0C801C0
:107100000E94C3C823E030E0A801BE016F5F7F4F3B
:10711000CE0185960E94EDC9BE016B5D7F4F8CEA62
:1071200094E10E9412C8CE0185960E9457C8C801FA
:107130000E9457C88091B0149091B114892B09F422
:10714000E3C270E060E08CEA94E10E94F2C6082E8F
:10715000000C990BC0970A9708F0D6C28CEA94E10C
:107160000E9417C66B016BEF76E0C8010E94C3C88E
:1071700086E08C9DB0018D9D700D112481E090E022
:107180008C0F9D1F680F791FC8010E9434C7BC0176
:107190008CEA94E10E94FBC7C8010E9457C80E9474
:1071A0004D95182FE2C08A3F2FEF920709F023C1B7
:1071B00060E077E0CE0101960E94C3C86AE077E004
:1071C000CE0107960E94C3C862E177E0CE010D961A
:1071D0000E94C3C86AE177E0CE0143960E94C3C80B
:1071E00063E272E1C8010E94B1C844E650E06FEF6B
:1071F0007FEFC8010E94151AC8010E9457C86DE1AF
:1072000072E18CEA94E10E94D6C780910D13EE24BE
:10721000E394F12CEC0EFD1E96E08902E00CF11CCB
:1072200011246CEA74E1C8010E94BAC8B701C80110
:107230000E9434C7BC01CE0185960E94BAC840EDB9
:1072400057E06FEF7FEFCE0185960E947B13CE0152
:1072500085960E9457C8C8010E9457C86DE072E128
:10726000C8010E94B1C844E650E06FEF7FEFC8014B
:107270000E94151AC8010E9457C860E277E0C80151
:107280000E94C3C824E030E0A801BE016F5F7F4FB9
:10729000CE0185960E94EDC9BE016B5D7F4F8CEAE1
:1072A00094E10E9412C8CE0185960E9457C8C80179
:1072B0000E9457C88091B0149091B114892B09F4A1
:1072C00098C070E060E08CEA94E10E94F2C6082E5B
:1072D000000C990BC0970A9708F08BC08CEA94E1D8
:1072E0000E9417C662307105810591050CF46EC0CD
:1072F00061E072E1C8010E94B1C844E650E06FEF5E
:107300007FEFC8010E947B13C8010E9457C844EF59
:1073100051E063E070E0CE0185960E941AC966E2F2
:1073200077E0C8010E94C3C86CEA74E1C8010E94FA
:1073300034C76DE277E00E941EC7BE016B5D7F4FD0
:107340000E9434C7BC018CEA94E10E94FBC7C801CB
:107350000E9457C8CE0185960E9457C80E944D953D
:10736000182FCE0143960E9457C8CE010D960E9459
:1073700057C8CE0107960E9457C8CE0101960E94B9
:1073800057C86BE771E1111102C06CE671E1CE01E3
:1073900001960E94B1C848EC50E06FEF7FEFCE013C
:1073A00001960E947B13CE0101960E9457C8E09679
:1073B0000FB6F894DEBF0FBECDBFDF91CF911F9106
:1073C0000F91FF90EF90DF90CF90089566E277E005
:1073D000C8010E94C3C86CEA74E1C8010E9434C7A6
:1073E000BC018CEA94E10E94FBC7C8010E9457C807
:1073F000B5CF10E0B6CF0F9609F0ECC0CE010196E4
:107400007C0161E37CE0C7010E94C3C896E0E90EFD
:10741000F11C0E151F05A9F760E377E0CE01019678
:107420000E949AC580911013811130C020911113D0
:1074300030911213409113135091141360E070E0D7
:1074400080EA90E40E9440E1AB01BC0122E0CE0161
:1074500085960E945FC866E377E0C8010E94C3C8B2
:10746000BE016B5D7F4FC8010E9434C76FEE77E0AD
:107470000E941EC7BC01CE0101960E94CFC7C80161
:107480000E9457C8CE0185960E9457C866EF71E1E9
:10749000CE0107960E94D6C76AEE71E1CE010D9625
:1074A0000E94D6C76EED71E1CE0143960E94D6C709
:1074B00062ED71E1CE0149960E94D6C76CEC71E194
:1074C000C8010E94D6C76DEB71E1C8010E94B1C826
:1074D00044E650E06FEF7FEFC8010E94151AC80123
:1074E0000E9457C861E37CE08CEA94E10E949AC54F
:1074F0008091101361E070E06C0F7D1F26E0820226
:10750000600D711D1124C8010E94BAC840ED57E0FA
:107510006FEF7FEFC8010E947B13C8010E9457C81C
:107520006EEA71E1C8010E94B1C844E650E06FEF15
:107530007FEFC8010E94151AC8010E9457C86CEA63
:1075400074E1C8010E94BAC825E030E0A801BE017C
:107550006F5F7F4FCE0185960E94EDC9BE016B5DC6
:107560007F4F8CEA94E10E9412C8CE0185960E945A
:1075700057C8C8010E9457C88091B0149091B114A7
:10758000892B31F170E060E08CEA94E10E94F2C650
:10759000082E000C990BC0970A97D0F469E377E0A6
:1075A000C8010E94C3C86CEA74E1C8010E9434C7D4
:1075B000BC018CEA94E10E94FBC7C8010E9457C835
:1075C0000E944D95182FCE0149960E9457C8C9CEEA
:1075D00010E0F9CF60E477E0CE0101960E94C3C8C5
:1075E00063E477E0CE0107960E94C3C868E477E0C1
:1075F000CE010D960E94C3C86EE971E1C8010E94D8
:10760000B1C844E650E06FEF7FEFC8010E94151A41
:10761000C8010E9457C868E971E18CEA94E10E94B0
:10762000D6C7809157139091581326E0289F700178
:10763000299FF00C112481E090E08C0F9D1FE80E33
:10764000F91E6CEA74E1C8010E94BAC8B701C8010A
:107650000E9434C7BC01CE0185960E94BAC840ED95
:1076600057E06FEF7FEFCE0185960E947B13CE012E
:1076700085960E9457C8C8010E9457C868E871E102
:10768000C8010E94B1C844E650E06FEF7FEFC80127
:107690000E94151AC8010E9457C86CEA74E1C8011B
:1076A0000E94BAC823E030E0A801BE016F5F7F4F9F
:1076B000CE0185960E94EDC9BE016B5D7F4F8CEABD
:1076C00094E10E9412C8CE0185960E9457C8C80155
:1076D0000E9457C88091B0149091B114892BA1F0E9
:1076E00070E060E08CEA94E10E94F2C6082E000C83
:1076F000990BC0970A9740F48CEA94E10E9417C650
:10770000CB010E94551F4DCD10E02FCE3F924F92DE
:107710005F926F927F928F929F92AF92BF92CF9221
:10772000DF92EF92FF920F931F93CF93DF93CDB72A
:10773000DEB7CA56D1090FB6F894DEBF0FBECDBF73
:1077400069AF7AAF8BAF9CAF29962CAF3DAF4EAFF0
:107750005FAF299761E37CE0CE01C1960E94C3C868
:10776000C9ACDAACEBACFCAC28EEC21623E0D20616
:10777000E104F10454F030E9C32EDD24D394E12C6C
:10778000F12CC9AEDAAEEBAEFCAE2996CCACDDACDA
:10779000EEACFFAC299720E1C21627E2D206E10445
:1077A000F10464F020E1C22E27E2D22EE12CF12C6C
:1077B0002996CCAEDDAEEEAEFFAE299780916D0E70
:1077C000882351F0C12CD12C7601C3942996CCAEDC
:1077D000DDAEEEAEFFAE29970E94326DA1966CAF82
:1077E0007DAF8EAF9FAFA1970E94326D65966CAF53
:1077F0007DAF8EAF9FAF6597A1966CAD7DAD8EAD21
:107800009FADA19728EE33E040E050E00E94FEDFFC
:10781000AB962CAF3DAF4EAF5FAFAB97312C2196FF
:107820001CAE1DAE1EAE1FAE21978E01075E1F4F10
:107830009E01235F3F4F38AF2FABC9ACDAACEBAC46
:10784000FCACF094E094D094C094C11CD11CE11C19
:10785000F11C6196CCAEDDAEEEAEFFAE61976596E3
:107860006CAD7DAD8EAD9FAD6597A196CCACDDAC1A
:10787000EEACFFACA1976C197D098E099F09299682
:10788000CCACDDACEEACFFAC29976C157D058E055C
:107890009F050CF08FC70E94C8DE20E030E04AE769
:1078A00054E40E9440E1AB01BC0123E0C8010E9406
:1078B0005FC8B80188E894E10E9412C8C8010E941C
:1078C00057C8A70196012A303105410551058CF4AE
:1078D000AB964CAD5DAD6EAD7FADAB97C8010E9470
:1078E000A4C5B80188E894E10E9412C8C8010E94AA
:1078F00057C880916D0E6BEB77E0882309F4DCC3E9
:1079000088E894E10E949AC580910C0E90910D0E2A
:10791000039709F453C0CE0101960E9497C161E319
:107920007CE08EE894E10E949AC5AE014F5F5F4F04
:107930005A01C12CD12C7601D5014D905D906D90EE
:107940007D905D01A3019201C301B2010E9427DF76
:107950009B01AC01C701B6010E9462E06B017C0192
:1079600023E0B301A201C8010E945FC8B801CE01A3
:107970004F960E94BAC86EE277E0CE014F960E9401
:107980001EC7BC018EE894E10E94CFC7CE014F967E
:107990000E9457C8C8010E9457C8EFA9F8ADEA1560
:1079A000FB0551F6C701B6010E946AE32D966CAF44
:1079B0007DAF8EAF9FAF2D973324339480910C0E03
:1079C00090910D0E0397039708F008C289E60E9474
:1079D000DFAC68EA70E089EC94E10E94071489EC5E
:1079E00094E10E94887346E050E069E670E089EC1B
:1079F00094E10E94D47380914A0F90914B0F891BA0
:107A0000990B86309105ECF30E9427ADB82E0E94A9
:107A100027ADA82E0E9427ADD82E0E9427ADC82ED4
:107A20000E9427ADF82E0E9427ADE82EA396AFAE98
:107A3000A397A2961FAEA297A3966EAD7FADA39714
:107A40006B29072E000C880B990B0E94C8DE2B01B6
:107A50003C014092730E5092740E6092750E7092BB
:107A6000760EA596CFAEA597A4961FAEA497A59621
:107A70006EAD7FADA5976D29072E000C880B990B75
:107A80000E94C8DE4B015C018092770E9092780EC6
:107A9000A092790EB0927A0EA796EFAEA797A6960F
:107AA0001FAEA697A7966EAD7FADA7976F29072E3D
:107AB000000C880B990B0E94C8DE25966CAF7DAF39
:107AC0008EAF9FAF259760937B0E70937C0E809353
:107AD0007D0E90937E0E8091A30EC090A80ED09044
:107AE000A90EE090AA0EF090AB0E882309F4F9C21B
:107AF00020918B0E30918C0E40918D0E50918E0EF8
:107B0000C301B2010E9461E0A70196010E9427DF34
:107B100060937F0E7093800E8093810E9093820EFF
:107B200020918F0E3091900E4091910E5091920EB7
:107B3000C501B4010E9461E0A70196010E9427DF00
:107B40006093830E7093840E8093850E9093860EBF
:107B50002091930E3091940E4091950E5091960E77
:107B600025966CAD7DAD8EAD9FAD25970E9461E0F1
:107B7000A70196010E9427DF6093870E7093880EFD
:107B80008093890E90938A0E20E030E0A9016091E5
:107B9000A40E7091A50E8091A60E9091A70E0E9442
:107BA00049E218160CF081C0C0907F0ED090800E74
:107BB000E090810EF090820E20E030E0A901C70134
:107BC000B6010E9449E2181624F0F7FAF094F7F88B
:107BD000F094A70196016091970E7091980E809194
:107BE000990E90919A0E0E9449E2181644F4109250
:107BF0007F0E1092800E1092810E1092820EC09015
:107C0000830ED090840EE090850EF090860E20E0DA
:107C100030E0A901C701B6010E9449E2181624F01C
:107C2000F7FAF094F7F8F094A701960160919B0E93
:107C300070919C0E80919D0E90919E0E0E9449E243
:107C4000181644F41092830E1092840E1092850E32
:107C50001092860EC090870ED090880EE090890E0C
:107C6000F0908A0E20E030E0A901C701B6010E9421
:107C700049E2181624F0F7FAF094F7F8F094A70107
:107C8000960160919F0E7091A00E8091A10E90912F
:107C9000A20E0E9449E2181644F41092870E109228
:107CA000880E1092890E10928A0E4091830E509188
:107CB000840E6091850E7091860E8091870E909152
:107CC000880EA091890EB0918A0EC0907F0ED09040
:107CD000800EE090810EF090820ECD86DE86EF86DB
:107CE000F88A498B5A8B6B8B7C8B8D8B9E8BAF8BE1
:107CF000B88F61E37CE0CE01C1960E949AC55E0117
:107D0000FDE0AF0EB11CC12CD12C7601D5014D90F8
:107D10005D906D907D905D01A3019201C301B20160
:107D20000E9427DF9B01AC01C701B6010E9462E0FF
:107D30006B017C0120E0B301A201C8010E945FC871
:107D4000B801CE014F960E94BAC86EE277E0CE012C
:107D50004F960E941EC7BC01CE01C1960E94CFC79C
:107D6000CE014F960E9457C8C8010E9457C80A15F5
:107D70001B0561F6C701B6010E946AE325966CAF48
:107D80007DAF8EAF9FAF259721E0AB01BC01CE0147
:107D90004F960E945FC860ED7BE0C8010E94C3C897
:107DA00068E874E1C8010E9434C76CE477E00E947F
:107DB0001EC7BE01615E7F4F0E9434C760E577E059
:107DC0000E941EC7BC01CE01C1960E94CFC7C80148
:107DD0000E9457C8CE014F960E9457C8C9ACDAAC72
:107DE000EBACFCAC2DE2C21621E0D206E104F104BA
:107DF00034F00E94571360E080E00E94FAAC80915A
:107E00000C0E90910D0E039709F43DC323E02D96BF
:107E10004CAD5DAD6EAD7FAD2D97CE014F960E94FE
:107E20005FC860ED7BE0C8010E94C3C868E874E1E8
:107E3000C8010E9434C767E577E00E941EC7BE01F3
:107E4000615E7F4F0E9434C76BE577E00E941EC7DA
:107E5000BC018EE894E10E94CFC7C8010E9457C8B8
:107E6000CE014F960E9457C82AE939E949E55FE3F8
:107E70002D966CAD7DAD8EAD9FAD2D970E9449E2E4
:107E800018160CF053C123E333E343E95FE32D9667
:107E90006CAD7DAD8EAD9FAD2D970E94C1DE880F7C
:107EA000880B382280910C0E90910D0E1816190631
:107EB0000CF03EC18230910509F43DC18530910539
:107EC0000CF039C18330910509F467C4059709F4B2
:107ED00064C469E677E0C8010E94C3C86EE874E133
:107EE000C8010E9434C7BC018EE894E10E94FBC720
:107EF000C8010E9457C86EE874E1C8010E94BAC860
:107F0000C8010E942313C8010E9457C86EE874E19B
:107F1000C8010E94BAC8C8010E946018C8010E9426
:107F200057C823E02D964CAD5DAD6EAD7FAD2D975E
:107F3000CE014F960E945FC868E577E0C8010E94B5
:107F4000C3C8BE01615E7F4FC8010E9434C76BE5A4
:107F500077E00E941EC7BC018EE894E10E94FBC737
:107F6000C8010E9457C8CE014F960E9457C86EE8BC
:107F700074E1C8010E94BAC8C8010E946018C80113
:107F80000E9457C868E874E1C8010E94BAC86EE848
:107F900074E1C8010E9434C7BC018EE894E10E94DC
:107FA000FBC7C8010E9457C866E777E088E894E1FC
:107FB0000E94C5C749855A856B857C8522E0CE0124
:107FC0008B960E945FC84D815E816F81788522E02B
:107FD000CE0185960E945FC849815A816B817C8160
:107FE00022E0C8010E945FC8B801CE014F960E94EE
:107FF000BAC86EE277E0CE014F960E941EC7BE015E
:108000006B5D7F4F0E9434C76EE277E00E941EC70F
:10801000BE01655D7F4F0E9434C7BC0182E894E1D8
:108020000E94FBC7CE014F960E9457C8C8010E940C
:1080300057C8CE0185960E9457C8CE018B960E94E4
:1080400057C8C9ACDAACEBACFCAC2DE2C21621E0EF
:10805000D206E104F10484F421966CAD7DAD8EADC1
:108060009FAD219725E030E040E050E00E94FEDF28
:10807000672B682B692BF1F468E874E1C8010E9452
:10808000BAC845E050E06FEF7FEFC8010E94151AB3
:10809000C8010E9457C862E874E1C8010E94BAC8CA
:1080A00045E050E070E060E0C8010E947B13C80129
:1080B0000E9457C8312CE7C1C8010E94C3C868E8B4
:1080C00074E1C8010E9434C766E77BE00E941EC7C6
:1080D000BC0188E894E10E94FBC7C8010E9457C810
:1080E00013CCA3019201C701B6010E9427DF609360
:1080F0007F0E7093800E8093810E9093820EA50167
:108100009401C701B6010E9427DF6093830E70932C
:10811000840E8093850E9093860E25962CAD3DADF2
:108120004EAD5FAD2597C701B60124CD312CBACE37
:10813000332009F4CECE89849A84AB84BC844980F0
:108140005A806B807C80CD80DE80EF80F88420E0D8
:1081500030E0A901C501B4010E94C1DE882309F401
:1081600009C3A3019201C301B2010E9427DF6996EE
:108170006CAF7DAF8EAF9FAF6997A7019601C70126
:10818000B6010E9427DF9B01AC0169966CAD7DAD05
:108190008EAD9FAD69970E9462E00E946AE3A501DF
:1081A00094010E94E1E020EE3EE245E652E40E94A6
:1081B00027DF69966CAF7DAF8EAF9FAF699720E0E8
:1081C00030E0A901C701B6010E94C1DE882309F48D
:1081D000D6C2A3019201C301B2010E9427DF6D96AE
:1081E0006CAF7DAF8EAF9FAF6D97A5019401C501B8
:1081F000B4010E9427DF9B01AC016D966CAD7DAD93
:108200008EAD9FAD6D970E9462E00E946AE3A70168
:1082100096010E94E1E020EE3EE245E652E40E9433
:1082200027DF6D966CAF7DAF8EAF9FAF6D9720E06F
:1082300030E0A901C301B2010E94C1DE882309F424
:10824000A3C2A5019401C501B4010E9427DF4B011F
:108250005C01A7019601C701B6010E9427DF9B01BF
:10826000AC01C501B4010E9462E00E946AE3A3016F
:1082700092010E94E1E06B017C0168E874E1C801B1
:108280000E94BAC869E773E1C8010E9434C7BC0103
:108290008EE894E10E94FBC7C8010E9457C86EE8AF
:1082A00074E1C8010E94BAC8C8010E944013C80105
:1082B0000E9457C821E069964CAD5DAD6EAD7FADB3
:1082C0006997CE018B960E945FC821E06D964CADF8
:1082D0005DAD6EAD7FAD6D97CE0185960E945FC896
:1082E00020EE3EE245E652E4C701B6010E9427DFD8
:1082F000AB01BC0121E0C8010E945FC8B801CE01FA
:108300004F960E94BAC86EE277E0CE014F960E9467
:108310001EC7BE016B5D7F4F0E9434C76EE277E0DF
:108320000E941EC7BE01655D7F4F0E9434C7BC011D
:108330008EE894E10E94FBC7CE014F960E9457C879
:10834000C8010E9457C8CE0185960E9457C8CE0129
:108350008B960E9457C86EE577E0C8010E94C3C89B
:108360006EE874E1C8010E9434C7BC0182E894E160
:108370000E94FBC7C8010E9457C862E874E1C801A7
:108380000E94BAC8C8010E946018C8010E9457C85C
:108390006EE874E182E894E10E94FBC76EE874E144
:1083A000C8010E94BAC8C8010E942313C8010E94D4
:1083B00057C8C9ACDAACEBACFCAC2DE2C21621E07C
:1083C000D206E104F10484F421966CAD7DAD8EAD4E
:1083D0009FAD219725E030E040E050E00E94FEDFB5
:1083E000672B682B692BA9F564E97EE088E894E1A6
:1083F0000E94D6C762E677E0C8010E94C3C845E084
:1084000050E067EF7FEFC8010E94151AC8010E9473
:1084100057C861E37CE0C8010E94C3C8C8010E943C
:108420001B10C8010E9457C86EE874E1C8010E9481
:10843000BAC845E050E070E060E0C8010E947B13DC
:10844000C8010E9457C861E37CE08EE894E10E9475
:108450009AC569AD7AAD8BAD9CADC9ACDAACEBAC6D
:10846000FCACF7FE0CC02E966FAD2E972F967FAD0D
:108470002F9760968FAD609761969FAD61970E9430
:10848000FF6C3324339480910C0E90910D0E039762
:10849000039708F0F6C06FE777E0C8010E94C3C8F1
:1084A000BE016F5C7F4FC8010E9434C7BC01CE0182
:1084B000C1960E94FBC7C8010E9457C8BE016F5CED
:1084C0007F4FC8010E94BAC8C8010E942313C80187
:1084D0000E9457C8BE016F5C7F4FC8010E94BAC896
:1084E000C8010E946018C8010E9457C821E0259663
:1084F0004CAD5DAD6EAD7FAD2597CE014F960E9420
:108500005FC86DE477E0C8010E94C3C8BE01615E28
:108510007F4FC8010E9434C760E577E00E941EC704
:10852000BC01CE01C1960E94FBC7C8010E9457C87A
:10853000CE014F960E9457C8BE016F5C7F4FC801A5
:108540000E94BAC8C8010E946018C8010E9457C89A
:1085500068E874E1C8010E94BAC8BE016F5C7F4F31
:10856000C8010E9434C7BC01CE01C1960E94FBC75E
:10857000C8010E9457C861E977E088E894E10E9449
:10858000C5C74D895E896F89788D20E0CE018B96B5
:108590000E945FC849895A896B897C8920E0CE0195
:1085A00085960E945FC84D855E856F85788920E03D
:1085B000C8010E945FC8B801CE014F960E94BAC898
:1085C0006EE277E0CE014F960E941EC7BE016B5D42
:1085D0007F4F0E9434C76EE277E00E941EC7BE0143
:1085E000655D7F4F0E9434C7BC0182E894E10E9420
:1085F000FBC7CE014F960E9457C8C8010E9457C8BA
:10860000CE0185960E9457C8CE018B960E9457C80E
:10861000C9ACDAACEBACFCAC2DE2C21621E0D20660
:10862000E104F10484F421966CAD7DAD8EAD9FAD77
:10863000219725E030E040E050E00E94FEDF672B0C
:10864000682B692BF1F468E874E1C8010E94BAC88C
:1086500045E050E06FEF7FEFC8010E94151AC80196
:108660000E9457C862E874E1C8010E94BAC845E098
:1086700050E070E060E0C8010E947B13C8010E94D6
:1086800057C880916D0E68E874E1882309F487C0AB
:10869000C8010E94BAC84AE050E067E070E0C80133
:1086A0000E945C19C8010E9457C83320D1F06CE8C1
:1086B0007EE0C8010E94B1C845E050E070E060E093
:1086C000C8010E94151AC8010E9457C861E37CE0E6
:1086D000C8010E94C3C8C8010E941B10C8010E94A3
:1086E00057C880910C0E90910D0E039779F062E8B7
:1086F00074E1C8010E94BAC84AE050E06FEF7FEF12
:10870000C8010E947B13C8010E9457C80E94326DA5
:108710006B017C0165962CAD3DAD4EAD5FAD6597AF
:10872000C21AD30AE40AF50A2196CCAEDDAEEEAE4B
:10873000FFAE219789AD9AADABADBCADC816D906D9
:10874000EA06FB0644F4BC01CD016C197D098E09D3
:108750009F090E94FF6C0E94326D65966CAF7DAFE1
:108760008EAF9FAF659761E37CE08EE894E10E9455
:108770009AC575C86BED7FE089EC9FE314CD6BED76
:108780007FE089EC9FE347CD8BEDC82E8FE0D82E9C
:1087900089ECE82E8FE3F82E70CD312C7CCEC80109
:1087A0000E94BAC84AE050E06FEF7FEFC8010E9414
:1087B000151A78CFCE01C1960E9457C8C659DF4F0F
:1087C0000FB6F894DEBF0FBECDBFDF91CF911F91E2
:1087D0000F91FF90EF90DF90CF90BF90AF909F9060
:1087E0008F907F906F905F904F903F9008954F9241
:1087F0005F926F927F928F929F92AF92BF92CF9231
:10880000DF92EF92FF920F931F93CF93DF93CDB739
:10881000DEB7A8970FB6F894DEBF0FBECDBF8C01B0
:1088200061E37CE0CE0149960E94C3C861E37CE02D
:10883000CE014F960E94C3C8809177139091781310
:10884000019709F065C30E940FBC65E070E080E00D
:1088500090E00E94FF6C8090FC149090FD14A0901A
:10886000FE14B090FF14C0900015D0900115E09058
:108870000215F09003158091041590910515A091B3
:108880000615B09107158DA39EA3AFA3B8A722E04C
:10889000AC01BD01CE0143960E945FC822E0B70142
:1088A000A601CE010D960E945FC822E0B501A40189
:1088B000CE0101960E945FC8BE016F5F7F4FCE015F
:1088C00007960E94BAC86EE277E0CE0107960E9432
:1088D0001EC7BE01635F7F4F0E9434C76EE277E020
:1088E0000E941EC7BE016D5E7F4F0E9434C76EE2BC
:1088F00077E00E941EC7BC018EE894E10E94FBC78E
:10890000CE0107960E9457C8CE0101960E9457C813
:10891000CE010D960E9457C8CE0143960E9457C8BB
:108920006EE874E1CE0101960E94BAC8CE010196AC
:108930000E942313CE0101960E9457C8A7019601F9
:10894000C501B40190580E94E1E02BED3FE049ECF5
:108950005FE30E9462E02091E7043091E8044091D7
:10896000E9045091EA040E9462E02B013C0120E0FE
:1089700030E0A9010E94C1DE87FD5BC34092880CF4
:108980005092890C60928A0C70928B0C4090880CEB
:108990005090890C60908A0C70908B0C2BED3FE00E
:1089A00049EC50E4C301B2010E9449E2181684F474
:1089B0002BED3FE049EC50E4C301B2010E9461E0BD
:1089C0006093880C7093890C80938A0C90938B0C25
:1089D00020E030E044E353E46091880C7091890C0E
:1089E00080918A0C90918B0C0E9427DF2BED3FE049
:1089F00049E450E40E9440E16093840C7093850C3C
:108A00008093860C9093870C0E94ECE1CE01079630
:108A10000E94D1C569E977E0CE0101960E94C3C8E2
:108A2000BE01695F7F4FCE0101960E9434C763EAA1
:108A300077E00E941EC7BC0184E994E10E94FBC755
:108A4000CE0101960E9457C8CE0107960E9457C8D2
:108A50004090840C5090850C6090860C7090870C30
:108A600020E030E044EB52E4C301B2010E94C1DED9
:108A700018160CF4EFC220E030E040E05FE3C301E1
:108A8000B2010E9462E00E94ECE1CE0107960E94D2
:108A9000D1C56AEA77E0CE0101960E94C3C8BE0143
:108AA000695F7F4FCE0101960E9434C7BC01CE01A1
:108AB00049960E94FBC7CE0101960E9457C8CE017D
:108AC00007960E9457C86CE079E0CE014F960E944D
:108AD0009AC5BE01675E7F4FCE0101960E94BAC85B
:108AE0004AE050E070E060E0CE0101960E94151A65
:108AF000CE0101960E9457C80E94326DAB01BC01A5
:108B000080918C0C90918D0CA0918E0CB0918F0C5B
:108B10008C599F4FAF4FBF4F84179507A607B707D4
:108B200008F01DC361E37CE0CE0101960E94C3C83A
:108B3000CE0101960E941B10CE0101960E9457C8DB
:108B4000BE01615E7F4F86E196E10E9452D16EE2E6
:108B500077E0CE0101960E94C3C8BE01615E7F4FDF
:108B6000CE0101960E9434C7BC01CE0149960E94F5
:108B7000CFC7CE0101960E9457C80E94326D409027
:108B8000980C5090990C60909A0C70909B0C641902
:108B90007509860997090E94C6DE20E030E04AE7A1
:108BA00054E40E9440E1AB01BC0123E0CE010796F2
:108BB0000E945FC86BEB77E0CE0101960E94C3C8AC
:108BC000BE01695F7F4FCE0101960E9434C766E700
:108BD0007BE00E941EC7BC0182E894E10E94FBC7B3
:108BE000CE0101960E9457C8CE0107960E9457C831
:108BF00062E874E1CE0101960E94BAC864E974E1AA
:108C0000CE0101960E9434C7BE01675E7F4F0E946D
:108C100034C7BC01CE0149960E94FBC7CE01019624
:108C20000E9457C861E974E08EE894E10E94D6C7BB
:108C300021E0B501A401CE0101960E945FC8BE01EA
:108C40006F5F7F4F8EE894E10E94CFC7CE010196FF
:108C50000E9457C821E04DA15EA16FA178A5CE0169
:108C60000D960E945FC821E0B701A601CE010796CC
:108C70000E945FC86EE277E0CE0101960E94C3C8F1
:108C8000BE01695F7F4FCE0101960E9434C76EE23C
:108C900077E00E941EC7BE01635F7F4F0E9434C70A
:108CA00062EB77E00E941EC7BC018EE894E10E944F
:108CB000CFC7CE0101960E9457C8CE0107960E94E9
:108CC00057C8CE010D960E9457C8A5019401C50151
:108CD000B4010E9427DF4B015C01A7019601C70187
:108CE000B6010E9427DF9B01AC01C501B4010E94BF
:108CF00062E06B017C012DA13EA14FA158A5CA01E4
:108D0000B9010E9427DF9B01AC01C701B6010E9497
:108D100062E00E946AE36093800C7093810C809300
:108D2000820C9093830C66EB77E08EE894E10E94CE
:108D3000C5C74091800C5091810C6091820C70915C
:108D4000830C21E0CE0101960E945FC8BE016F5FD7
:108D50007F4FCE0107960E94BAC862E67CE0CE0142
:108D600007960E941EC7BC0184E994E10E94FBC7DC
:108D7000CE0107960E9457C8CE0101960E9457C89F
:108D800064E974E18EE894E10E94CFC7C090800C42
:108D9000D090810CE090820CF090830C20E030E0C9
:108DA0004AE754E4C701B6010E9449E287FD29C0A1
:108DB00020E030E04AE754E4C701B6010E9440E1F8
:108DC000AB01BC0123E0CE0101960E945FC8BE0149
:108DD0006F5F7F4FCE0107960E94BAC863E67CE0C2
:108DE000CE0107960E941EC7BC0184E994E10E944F
:108DF000FBC7CE0107960E9457C8CE0101960E947C
:108E000057C820E030E64AE656E46091800C709145
:108E1000810C8091820C9091830C0E94C1DEBE0176
:108E2000675E7F4F87FFBAC1CE0101960E94BAC824
:108E30006AEB77E0CE0101960E941EC76EE874E1EE
:108E40000E9434C7BC018EE894E10E94FBC7CE01AA
:108E500001960E9457C803301105A1F46EE874E131
:108E6000CE0101960E94BAC8CE0101960E9423133A
:108E7000CE0101960E9457C861E37CE08EE894E140
:108E80000E949AC56DEB77E0CE0101960E94C3C89F
:108E900064E974E1CE0101960E9434C7BC01CE01A1
:108EA00007960E94BAC84AE050E06FEF7FEFCE010C
:108EB00007960E947B13CE0107960E9457C8CE01E9
:108EC00001960E9457C86AE070E080E090E00E943E
:108ED000FF6CCE014F960E9457C8CE0149960E9462
:108EE00057C8A8960FB6F894DEBF0FBECDBFDF916E
:108EF000CF911F910F91FF90EF90DF90CF90BF9097
:108F0000AF909F908F907F906F905F904F9008955B
:108F10000E94DD7340903D0550903E0560903F05F6
:108F2000709040056091260F7091270F072E000C5E
:108F3000880B990B0E94C8DEA30192010E9427DFD3
:108F40002091390530913A0540913B0550913C05FF
:108F50000E9427DF2091120F3091130F4091140FC0
:108F60005091150F0E9462E04B015C0180921E0F30
:108F700090921F0FA092200FB092210F6091240FAA
:108F80007091250F072E000C880B990B0E94C8DEEC
:108F9000A30192010E9427DF20913505309136050B
:108FA00040913705509138050E9427DF20910E0F20
:108FB00030910F0F4091100F5091110F0E9462E0FD
:108FC0006B017C01C0921A0FD0921B0FE0921C0F14
:108FD000F0921D0F6091220F7091230F072E000C4D
:108FE000880B990B0E94C8DEA30192010E9427DF23
:108FF000209131053091320540913305509134056F
:109000000E9427DF20910A0F30910B0F40910C0F27
:1090100050910D0F0E9462E06DA37EA38FA398A7CD
:109020006093160F7093170F8093180F9093190F7A
:1090300085CC2BED3FE049EC50E4C301B2010E9426
:1090400062E06093880C7093890C80938A0C9093F3
:109050008B0C9CCC20E030E044E353E4C301B2012C
:109060000E94C1DE1816CCF0A301920160E070E806
:1090700084E393E40E9461E06093840C7093850C18
:109080008093860C9093870C0E94ECE1CE010796AA
:109090000E94D1C56DEA77E0FECC20E030E047E8E1
:1090A00053E4C301B2010E94C1DE1816CCF120E0E6
:1090B00030E044E353E4C301B2010E9461E020E0E8
:1090C00030E040E05FE30E9462E06093840C7093C4
:1090D000850C8093860C9093870C0E94ECE1CE0166
:1090E00007960E94D1C56DEA77E0CE0101960E94F5
:1090F000C3C8BE01695F7F4FCE0101960E9434C78D
:10910000BC01CE0149960E94FBC7CE0101960E9488
:1091100057C8CE0107960E9457C860EB77E0D5CCC0
:10912000A301920160E070E084EB93E40E9461E0AF
:1091300020E030E040E05FE30E9462E06093840C56
:109140007093850C8093860C9093870C0E94ECE1C1
:10915000CE0107960E94D1C56AEA77E0C6CF0E9489
:10916000326D0E94C6DE2B013C0160918C0C709127
:109170008D0C80918E0C90918F0C0E94C8DE20E0A7
:1091800030E048EC51E40E9462E09B01AC01C30175
:10919000B2010E94C1DE87FDC5CCD9CC8EE894E136
:1091A0000E94FBC790CEDF92EF92FF920F931F9326
:1091B000CF93DF93CDB7DEB72C970FB6F894DEBF11
:1091C0000FBECDBF8C0110928B0D61E37CE0CE0110
:1091D00007960E94C3C8F12CE12CDD24D3948BE9BF
:1091E0009FE00E94C3A91816190694F480918B0D74
:1091F00081110EC08BE99FE00E94A1A98A30D1F5B0
:109200008B859C85892B09F443C0D0928B0D40C07F
:1092100062E370E080E090E00E94FF6CEF2851F084
:109220008BE99FE00E94CFAB64E670E080E090E0C5
:109230000E94FF6C80918B0D811131C08B859C85C4
:10924000892B69F561E37CE0C8010E94C3C8CE01A7
:1092500007960E9457C8C8012C960FB6F894DEBF37
:109260000FBECDBFDF91CF911F910F91FF90EF9077
:10927000DF9008958D3021F290918B0D9111C0CF28
:10928000682FCE0107960E94A2C78FEFE81AF80A4E
:109290006FE070E080E090E00E94FF6CA0CF8091D2
:1092A0006E0E882379F0BE01695F7F4FCE01019673
:1092B0000E94BAC8CE0101960E942313CE010196E6
:1092C0000E9457C8BE01695F7F4FC8010E94A8C8AD
:1092D000BECF8F929F92AF92BF92CF92DF92EF92CA
:1092E000FF920F931F93CF93DF93CDB7DEB76897AD
:1092F0000FB6F894DEBF0FBECDBF6C01809157133F
:10930000909158130197C9F061E37CE0C6010E9477
:10931000C3C8C60168960FB6F894DEBF0FBECDBFB6
:10932000DF91CF911F910F91FF90EF90DF90CF9041
:10933000BF90AF909F908F90089566EC77E0CE013C
:109340000D960E94C3C8BE01635F7F4F8BE99FE00B
:109350000E9452D16CE271E080E090E00E94FF6CCC
:10936000CE0143960E94D34864E670E080E090E02E
:109370000E94FF6C10E000E085E0A82EB12C9AE07E
:10938000892E912C61ED77E0CE0101960E94C3C831
:10939000BE016F5F7F4FCE0143960E94D7C67C010E
:1093A000CE0101960E9457C8A7014F5F5F4FBE01D3
:1093B0006D5E7F4FCE0101960E945418BE016F5F13
:1093C0007F4FCE010D960E9412C8CE0101960E94D9
:1093D00057C889899A89892B09F170E060E0CE012C
:1093E0000D960E94F2C6082E000C990BC0970A97A2
:1093F000A8F463ED77E0CE0101960E94C3C8BE01D8
:109400006F5F7F4FCE010D960E9403C7E82ECE01FD
:1094100001960E9457C8FF24F394E110F12C65E5F2
:109420007FE0CE0101960E94B1C844E150E06FEFA9
:109430007FEFCE0101960E945C19CE0101960E9439
:1094400057C80F5F1F4F62E370E080E090E00E941A
:10945000FF6CC801B5010E94D8E30197D1F461E027
:1094600070E0CE0101960E9433838D819E81892B0D
:1094700009F46AC0BE016F5F7F4F8CEA94E10E94DD
:10948000FBC70E9453A2FF24F394CE0101960E94D1
:1094900057C8CE0101960E94D348BE016F5F7F4F2F
:1094A000CE0143960E9412C8CE0101960E9457C871
:1094B00062E370E080E090E00E94FF6C04361105EA
:1094C00019F0FF2009F45ECF80916E0E8823F1F031
:1094D00068E379E0CE0101960E94C3C8BE01635FD4
:1094E0007F4FCE0101960E9434C7BC01CE01079682
:1094F0000E94BAC8CE0107960E942313CE01079698
:109500000E9457C8CE0101960E9457C889899A893E
:10951000892B61F070E060E0CE010D960E94F2C6EA
:10952000082E000C990BC0970A9738F16BED77E085
:10953000C6010E94C3C8CE0143960E9457C8CE01FF
:109540000D960E9457C8E5CE043111050CF49DCF4D
:10955000C801B4010E94D8E3892B09F096CFBE015F
:10956000635F7F4F8BE99FE00E9452D168EC70E00F
:1095700080E090E00E94FF6C88CF63ED77E0CE0141
:1095800001960E94C3C8BE016F5F7F4FCE010D964A
:109590000E9403C7182FCE0101960E9457C81111CF
:1095A000C5CFBE01635F7F4FC6010E94A8C8C3CF6D
:1095B0003F924F925F926F927F928F929F92AF9263
:1095C000BF92CF92DF92EF92FF920F931F93CF93B0
:1095D000DF93CDB7DEB7E4970FB6F894DEBF0FBECA
:1095E000CDBF80918C0D8823D1F010928C0DE49624
:1095F0000FB6F894DEBF0FBECDBFDF91CF911F91A4
:109600000F91FF90EF90DF90CF90BF90AF909F9021
:109610008F907F906F905F904F903F90089581E082
:1096200080938C0D61E37CE0CE0185960E94C3C8D7
:1096300061E37CE0CE018B960E94C3C810E000E09D
:1096400082E0382E98EEC92E93E0D92EE12CF12C31
:10965000F8013197E231F105C0F48827ED5CF44B55
:109660008F4F0C94ECE31A4CB14CC64CCF4CD84CF9
:10967000E14CF24CFB4C2A4D3B4D444D4D4D564D6B
:10968000F14DFA4D034E0C4E154E61E37CE0CE01D8
:1096900085960E949AC58091571390915813892BF3
:1096A00031F469E276E0CE0185960E949AC58091F8
:1096B000571390915813019731F463E276E0CE018D
:1096C00085960E949AC580915713909158130297DE
:1096D00031F46DE276E0CE0185960E949AC589A5A7
:1096E0009AA5892B31F06EEF75E1CE0185960E9427
:1096F000CFC762E376E0CE0101960E94C3C86AE05C
:1097000076E1CE0101960E9434C7BC01CE018B9652
:109710000E94FBC7CE0101960E9457C88091571343
:1097200090915813019709F046C0BE016B5D7F4FC1
:10973000CE0101960E94BAC848EC50E06FEF7FEF6F
:10974000CE0101960E94151ACE0101960E9457C8BB
:10975000BE01655D7F4FCE0101960E94BAC840ED03
:1097600057E06FEF7FEFCE0101960E947B13CE0191
:1097700001960E9457C8CE0101960E9469498D81C9
:109780009E810097A1F0E981FA812081222379F05E
:10979000079768F061E077E0CE0185960E94D6C712
:1097A000BE016F5F7F4FCE018B960E94FBC7CE013B
:1097B00001960E9457C8BE016B5D7F4FCE01019696
:1097C0000E94BAC848EC50E06FEF7FEFCE010196DF
:1097D0000E945C19CE0101960E9457C8BE01655DCA
:1097E0007F4FCE0101960E94BAC848EC50E06FEF5F
:1097F0007FEFCE0101960E947B13CE0101960E945D
:1098000057C80E943FB4982EB12CA12C911016C2BB
:109810008FEFA81AB80A95E6A916B10409F411C287
:109820000E943FB4982E64E170E080E090E00E94D6
:10983000FF6CECCF65EF76E0CE0185960E94D6C72F
:109840000E94326D4B015C010E94326DA7019601AE
:109850000E9430E0CA01B90120E831E541E050E062
:109860000E9430E020E13EE040E050E00E94FEDF58
:1098700029AB3AAB4BAB5CAB2CE330E040E050E0C3
:109880000E94FEDF29013A01AB01BC01CE01019625
:109890000E94A4C5B301A201CE0107960E94A4C5EF
:1098A00049A95AA96BA97CA9CE010D960E94A4C50D
:1098B000C501B40120E03CE546E255E00E9430E0FD
:1098C000BA01A901CE0149960E94A4C5BE01675EF6
:1098D0007F4FCE0143960E94BAC867EE77E0CE0173
:1098E00043960E941EC7BE01635F7F4F0E9434C72C
:1098F0006AEE77E00E941EC7BE01695F7F4F0E943B
:1099000034C760E976E00E941EC7BE016F5F7F4FDB
:109910000E9434C765E577E00E941EC7BC01CE01F6
:109920004F960E94BAC8CE0143960E9457C8CE01F6
:1099300049960E9457C8CE010D960E9457C8CE0185
:1099400007960E9457C8CE0101960E9457C8BE01D3
:10995000615E7F4FCE018B960E9412C8CE014F965A
:1099600028CF8091E20D9091E30D66EE76E00197AD
:1099700011F068ED76E0CE0185960E94D6C768ECBE
:1099800076E0CE018B960E94D6C715CF68EB76E0C5
:10999000CE0185960E94D6C76BEA76E0F2CF6EE9DB
:1099A00076E0CE0185960E94D6C763E976E0E9CFDE
:1099B00067E876E0CE0185960E94D6C766E776E036
:1099C000E0CF8091E20D9091E30D6BE676E0039796
:1099D00011F061E676E0CE0185960E94D6C766E575
:1099E00076E0CFCF69E476E0CE0185960E94D6C7B7
:1099F0006AE376E0C6CF6FE276E0CE0185960E94FC
:109A0000D6C760910E1370910F13CE0107960E9476
:109A1000D1C567E377E0CE0101960E94C3C8BE01BD
:109A2000695F7F4FCE0101960E9434C768E077E0FE
:109A30000E941EC7BC01CE0185960E94CFC7CE01F1
:109A400001960E9457C8CE0107960E9457C862E24D
:109A500076E097CF8091E20D9091E30D61E176E0A1
:109A6000029711F061E076E0CE0185960E94D6C79C
:109A700064EF75E086CF68EE75E0CE0185960E94B2
:109A8000D6C768ED75E07DCF6DEC75E0CE018596AB
:109A90000E94D6C763EC75E074CF67EB75E0CE012A
:109AA00085960E94D6C767EA75E06BCFB090101319
:109AB0006CE975E0CE0185960E94D6C783E08B15D0
:109AC00024F192E0B9160CF073C0BB2031F181E0B3
:109AD000B81609F464C060911013062E000C770BC1
:109AE000CE0107960E94D1C568E47BE0CE010196C5
:109AF0000E94C3C8BE01695F7F4FCE0101960E94DC
:109B000034C7BC018EE894E13FC094E0B912E3CFC2
:109B100061EF77E08EE894E146C080901113909059
:109B20001213A0901313B090141320E030E048E417
:109B300052E4C501B4010E94C1DE87FF02C0332494
:109B40003394A501940160E070E080EA90E40E9403
:109B500040E1AB01BC01232DCE0107960E945FC8F6
:109B60006BEB77E0CE0101960E94C3C8BE01695F2E
:109B70007F4FCE0101960E9434C766EF77E00E94C6
:109B80001EC7BC01CE0185960E94CFC7CE010196AB
:109B90000E9457C8CE0107960E9457C806C06DEEB6
:109BA00077E0CE0185960E94C5C76CE875E0E9CEE6
:109BB0008B2D9AE08902B0011124CE0107960E94F4
:109BC000D1C567E377E0CE0101960E94C3C8BE010C
:109BD000695F7F4FCE0101960E9434C76FEE77E038
:109BE000CECF6CE775E0CE0185960E94D6C76CE6B5
:109BF00075E0C7CE6CE575E0CE0185960E94D6C7AC
:109C00006EE475E0BECE63E475E0CE0185960E94F9
:109C1000D6C768E375E0B5CE6BE275E0CE018596F8
:109C20000E94D6C76BE175E0ACCE6FE075E0CE0167
:109C300085960E94D6C760E075E0A3CE10928C0D89
:109C400021C061E070E0CE0101960E943383BE0125
:109C50006F5F7F4F8CEA94E10E9412C8CE0101969B
:109C60000E9457C88091B0149091B114892B51F47F
:109C700080918C0D882331F00F5F1F4F0331110548
:109C800009F0E6CCCE018B960E9457C8CE0185968E
:109C90000E9457C8ACCC2F923F924F925F926F9226
:109CA0007F928F929F92AF92BF92CF92DF92EF926C
:109CB000FF920F931F93CF93DF93CDB7DEB76697D5
:109CC0000FB6F894DEBF0FBECDBF8C01E090E00D63
:109CD000F090E10D80916E0E882349F06BE17AE0FF
:109CE00082E791E10E9472D1C8010E9469CCC8014B
:109CF0000596059710F40C94D8618091E00D909131
:109D0000E10D80179107E1F00E9457130E94C010E7
:109D10000C3E2FEF120724F01093E10D0093E00D9D
:109D2000B801CE0101960E94D1C5BE016F5F7F4F81
:109D30008AE994E10E9412C8CE0101960E9457C898
:109D400061E37CE08EE894E10E949AC56EE277E0E0
:109D5000CE0101960E94C3C84AE050E06FEF7FEF4A
:109D6000CE0101960E945C19CE0101960E9457C84F
:109D7000033EFFEF1F0714F00C94E4610E3C3FEF2D
:109D8000130749F0023E4FEF140729F078010A3B10
:109D90005FEF150751F541E050E066EA74E1CE014E
:109DA00001960E945418BE016F5F7F4F82E894E1D4
:109DB0000E9412C8CE0101960E9457C882E894E121
:109DC0000E9417C67801E61AF70A809186149091CE
:109DD0008714892B39F0E0918214F09183148081EB
:109DE000811103C08AE0E81AF108C70188960A9732
:109DF00008F0B5C062EE7FEF6E197F09CE010196C3
:109E00000E94D1C56BE778E0CE0107960E94C3C8D7
:109E1000BE016F5F7F4FCE0107960E9434C7BC0121
:109E200086EA94E10E94FBC7CE0107960E9457C8BC
:109E3000CE0101960E9457C869EF77E0CE010196E6
:109E40000E94C3C866EA74E1CE0101960E9434C73D
:109E5000BC0188E894E10E94FBC7CE0101960E94F4
:109E600057C868E874E1CE0101960E94BAC8CE01D5
:109E700001960E942313CE0101960E9457C86DEFF0
:109E800077E0CE0107960E94C3C866EA74E1CE016E
:109E900007960E9434C7BC01CE0101960E94BAC841
:109EA00048EC50E06FEF7FEFCE0101960E94151A4B
:109EB000CE0101960E9457C8CE0107960E9457C84E
:109EC00041E050E066EA74E1CE0101960E94541828
:109ED000BE016F5F7F4F82E894E10E9412C8CE01FD
:109EE00001960E9457C882E894E10E9417C6DC01DF
:109EF000CB010197A109B10961EC77E089309105A7
:109F0000A105B10508F0F9C0FC018827E557F04B21
:109F10008F4F0C94ECE37B50905093509650995097
:109F20009C509F50A250A5500E94D01066960FB62C
:109F3000F894DEBF0FBECDBFDF91CF911F910F917F
:109F4000FF90EF90DF90CF90BF90AF909F908F9059
:109F50007F906F905F904F903F902F900895C70132
:109F6000CC960A9708F04FC06EEC7FEF6E197F0910
:109F7000CE0101960E94D1C562E079E0CE0107963C
:109F80000E94C3C8BE016F5F7F4FCE0107960E943B
:109F900034C7BC0186EA94E10E94FBC7CE01079654
:109FA0000E9457C8CE0101960E9457C841E050E078
:109FB00066EA74E1CE0101960E945418BE016F5FFB
:109FC0007F4F82E894E10E9412C8CE0101960E9460
:109FD00057C882E894E10E9417C69B016A30710558
:109FE00008F095C1FB018827E750F04B8F4F0C9488
:109FF000ECE38451A850A850A850A850A850135181
:10A00000185153517D51C701805B9F4F0A9718F536
:10A010006AEB7FEF6E197F09CE0101960E94D1C5D0
:10A020006FEE77E0CE0107960E94C3C8BE016F5F56
:10A030007F4FCE0107960E9434C7BC0186EA94E1A7
:10A040000E94FBC7CE0107960E9457C8CE01019619
:10A050000E9457C80CC09EECE9169FEFF90609F460
:10A06000A5CFA2EEEA16AFEFFA0609F4E5CEF0921C
:10A07000E10DE092E00D809192149091931400977D
:10A0800099F14197A8F40230110594F06EE874E15B
:10A09000CE0101960E94BAC84AE050E06FEF7FEF10
:10A0A000CE0101960E947B13CE0101960E9457C8F3
:10A0B0006EE874E1CE0101960E94BAC8CE01019605
:10A0C0000E942313CE0101960E9457C86EE874E1E6
:10A0D000CE0101960E94BAC8CE0101960E94601876
:10A0E000CE0101960E9457C864E670E080E090E0DF
:10A0F0000E94FF6C1BCF62E378E088E894E10E9445
:10A10000D6C768E874E1CE0101960E94BAC84CED4A
:10A1100055E06FEF7FEFCE0101960E947B1396CF43
:10A1200065E278E0EACF65E178E0E7CF6BE078E0E0
:10A13000E4CF67E078E0E1CF67EF77E0DECF69EE6C
:10A1400077E0DBCF6BED77E0D8CF6EEC77E0D5CF63
:10A15000F901E050FE4F90819A3008F056C0B901E5
:10A16000CE0101960E94D1C563E078E0CE0107964A
:10A170000E94C3C8BE016F5F7F4FCE0107960E9449
:10A1800034C7BC0184E994E10E94FBC7CE01079665
:10A190000E9457C8CE0101960E9457C869E078E036
:10A1A000CE0101960E94C3C84AE050E06FEF7FEFF6
:10A1B000CE0101960E94151ACE0101960E9457C841
:10A1C00065E070E080E090E00E94FF6C64E974E17B
:10A1D000CE0101960E94BAC84AE050E06FEF7FEFCF
:10A1E000CE0101960E947B13CE0101960E9457C8B2
:10A1F0006CEA77E08EE894E10E94D6C764E974E1E6
:10A200008EE894E10E94CFC732CF86E3860F9A3062
:10A2100031F49BE0908361E00E94456C28CF9AE086
:10A22000908360E0F9CF88E390E00E94B12C1FCFCB
:10A230008091890D882321F080E00E940E2817CF9D
:10A2400060E977E08EE894E10E94D6C769E877E09C
:10A2500088E894E10E94D6C76AE777E084E994E150
:10A260000E94D6C768E874E1CE0101960E94BAC880
:10A270004AE050E070E060E0CE0101960E94151ABD
:10A28000CE0101960E9457C865E070E080E090E042
:10A290000E94FF6C64E974E1CE0101960E94BAC885
:10A2A0004AE050E036CF8091920D882349F08091AA
:10A2B000C5049091C6040E9427740E948374D7CE6F
:10A2C00061E577E08EE894E10E94D6C764E477E028
:10A2D00088E894E10E94D6C765E377E084E994E1D9
:10A2E0000E94D6C768E874E1CE0101960E94BAC800
:10A2F0004AE050E06FEF7FEFBFCF64E277E08EE897
:10A3000094E10E94D6C7B3CE63E177E0F8CF6AE06C
:10A3100077E0F5CF0E94571389E390E00E947F1207
:10A3200020E030E04AE754E40E9427DFAB01BC01A3
:10A3300021E0CE0101960E945FC865E27BE0CE017C
:10A3400007960E94C3C8BE016F5F7F4FCE0107967C
:10A350000E9434C766E178E00E941EC7BC018EE807
:10A3600094E10E94FBC7CE0107960E9457C8CE0118
:10A3700001960E9457C86AE178E088E894E10E945B
:10A380009AC568E874E1CE0101960E94BAC84AE015
:10A3900050E068E070E0CE0101960E94151ACE01EF
:10A3A00001960E9457C86EE874E1CE0101960E94A2
:10A3B000BAC84AE050E06FEF7FEFCE0101960E94ED
:10A3C0007B13CE0101960E9457C868E874E18EE8BD
:10A3D00094E10E94CFC780916D0E882309F44BCE83
:10A3E00064E670E080E090E02BC4C0900A02D09058
:10A3F0000B020E94571389E390E00E947F1220E035
:10A4000030E04AE754E40E9427DF0E94ECE1CE01ED
:10A4100001960E94D1C565E27BE0CE0107960E94BD
:10A42000C3C8BE016F5F7F4FCE0107960E9434C73D
:10A4300066E178E00E941EC7BC018EE894E10E94AC
:10A44000FBC7CE0107960E9457C8CE0101960E9415
:10A4500057C8809192149091931423E0F22E09979B
:10A4600010F092E0F92E80910D1340E050E0BA0117
:10A470008330DCF4C6010E940A124B015C0160913A
:10A480000E1370910F13072E000C880B990B0E946E
:10A49000C8DEA50194010E9427DF20E030EC4FE7E1
:10A4A00054E40E9440E1AB01BC012F2DCE01019686
:10A4B0000E945FC86BE478E0CE0107960E94C3C893
:10A4C000BE016F5F7F4FCE0107960E9434C762E2E4
:10A4D00078E00E941EC7BC018EE894E10E94CFC7BD
:10A4E000CE0107960E9457C8CE0101960E9457C818
:10A4F00065E278E042CF80916D0E882309F439C17E
:10A5000088E390E10E94DCB062E370E080E090E0DC
:10A510000E94FF6C61E08091A6040E94776C60E06D
:10A520008091A4040E94776C64E670E080E090E083
:10A530000E94FF6C6091A0047091A1048091A2041C
:10A540009091A3040E94A3100E94C70FAB01BC010D
:10A5500023E0CE0107960E945FC8BE01695F7F4F6E
:10A56000CE0101960E94BAC868E478E0CE01019657
:10A570000E941EC7BC0188E894E10E94FBC7CE017F
:10A5800001960E9457C8CE0107960E9457C864E9F9
:10A5900076E0CE0101960E94C3C868E874E1CE015E
:10A5A00001960E9434C7BC018EE894E10E94FBC76B
:10A5B000CE0101960E9457C80E94C70F6B017C0113
:10A5C0000E94DA6C4B015C018BE19EE40197F1F78C
:10A5D0000E94C70F2B013C010E94DA6C9B01AC0169
:10A5E000281939094A095B0949015A0131ED8316D5
:10A5F00037E09306A104B104CCF0A7019601C30192
:10A60000B2010E9461E06B017C0120E030E0A90111
:10A610000E9449E2181674F426EA3BE944EC5BE335
:10A62000C701B6010E94C1DE87FF0EC040E050E0C6
:10A63000BA0126C026EA3BE944EC5BEBC701B60150
:10A640000E9449E2181694F3C501B40128EE33E0E4
:10A6500040E050E00E94FEDFCA01B9010E94C8DE5E
:10A660004B015C0120E030E04AE754E4C701B60149
:10A670000E9427DFA50194010E9440E1AB01BC01CB
:10A6800022E0CE0107960E945FC8BE01695F7F4F3E
:10A69000CE0101960E94BAC867E976E0CE01019624
:10A6A0000E941EC7BC0182E894E10E94FBC7CE0154
:10A6B00001960E9457C8CE0107960E9457C86EE2C5
:10A6C00078E0CE0101960E94C3C862E874E1CE0131
:10A6D00001960E9434C7BC018EE894E10E94CFC766
:10A6E000CE0101960E9457C86EE277E0CE01019636
:10A6F0000E94C3C862E874E1CE0101960E9434C78B
:10A70000BC0188E894E10E94CFC7CE0101960E9467
:10A7100057C862E478E0CE0101960E94B1C84AE0D1
:10A7200050E070E060E0CE0101960E94151ACE0163
:10A7300001960E9457C868E874E1CE0101960E9414
:10A74000BAC845E050E06FEF7FEFCE0101960E945E
:10A750007B13CE0101960E9457C862E378E08EE831
:10A7600094E10E94C5C760E08091A6040E94776CC6
:10A7700082CC609195047091960480919704909199
:10A7800098040E947D2E77CC80918F049091900444
:10A790000E94983070CC409191044E8B60E0842FE1
:10A7A0000E94776C80916D0E811191C1809183130D
:10A7B00081118DC18FE0C82ED12CE12CF12C61E5E7
:10A7C00078E08EE894E10E94D6C76EE874E1CE018D
:10A7D00001960E94BAC84AE050E06FEF7FEFCE01C9
:10A7E00001960E94151ACE0101960E9457C8312C7D
:10A7F000212C198A1D8A1D861E861F86188AA2E3AF
:10A800006A2E712C812C912C54018E890E94B76C78
:10A81000092E000CAA0BBB0B880E991EAA1EBB1E8C
:10A8200065E070E080E090E00E94FF6C51E0651A06
:10A83000710859F74090F2045090F3046090F404CA
:10A840007090F504C501B4010E94C8DE20E030E03C
:10A8500040EA50E40E9427DF20E030E040E85AE37D
:10A860000E9427DF20E030E048E452E40E9440E10B
:10A87000A30192010E9461E020E030E040E751E452
:10A880000E9427DF4B015C01A30192016AE979E98B
:10A8900089E390E40E9461E09B01AC01C501B40131
:10A8A0000E9440E120E030E0A9010E9462E020E047
:10A8B00030E040E251E40E9427DF4B015C01232D90
:10A8C000322D49895D890E9449E2181624F4382CFA
:10A8D000292CA98ABD8A20E030E0A901B401C50174
:10A8E0000E94C1DE87FF04C0812C912CA12CB12CC9
:10A8F00022E0A401B501CE0107960E945FC8BE0107
:10A90000695F7F4FCE0101960E94BAC865E478E086
:10A91000CE0101960E941EC7BC0188E894E10E9406
:10A92000FBC7CE0101960E9457C8CE0107960E9430
:10A9300057C868E874E1CE0101960E94BAC84AE09F
:10A9400050E070E060E0CE0101960E947B13CE01E2
:10A9500001960E9457C80E94326DAB01BC018091E4
:10A96000900C9091910CA091920CB091930C8C59F9
:10A970009F4FAF4FBF4F84179507A607B70708F043
:10A98000ACC00E9439106CE370E080E090E00E945F
:10A99000FF6C8D859E85AF85B8890196A11DB11D7F
:10A9A0008D879E87AF87B88BC816D906EA06FB0647
:10A9B0000CF025CF64E670E080E090E00E94FF6C30
:10A9C0000E94571364E670E080E090E00E94FF6C04
:10A9D00069E478E088E894E10E94D6C768E874E109
:10A9E000CE0101960E94BAC844E150E070E060E0F8
:10A9F000CE0101960E94151ACE0101960E9457C8F9
:10AA000022E0432D522D69897D89CE0107960E944F
:10AA10005FC8BE01695F7F4FCE0101960E94BAC830
:10AA200065E478E0CE0101960E941EC7BC0188E86B
:10AA300094E10E94FBC7CE0101960E9457C8CE0147
:10AA400007960E9457C868E874E1CE0101960E94FB
:10AA5000BAC842E350E06FEF7FEFCE0101960E944B
:10AA60007B13CE0101960E9457C864E170E080E03C
:10AA700090E00E94FF6C0E9439106EE170E080E06F
:10AA800090E00E94FF6C6EE170E080E090E00E9438
:10AA9000FF6C6AE478E0CE0101960E94C3C868E8C2
:10AAA00074E1CE0101960E9434C76EE478E00E9402
:10AAB0001EC76EE874E10E9434C7BC018EE894E1C1
:10AAC0000E94FBC7CE0101960E9457C8D4CAB3E0CA
:10AAD000CB2ED12CE12CF12C72CE0E94326D0E9433
:10AAE000C6DE4B015C016091900C7091910C8091DD
:10AAF000920C9091930C0E94C8DE20E030E048EC6C
:10AB000051E40E9462E09B01AC01C501B4010E94C6
:10AB1000C1DE87FD36CF37CF8091930490919404A6
:10AB200099270E940A122DE038E643E55BE30E9474
:10AB300027DF6B017C012091190530911A054091A6
:10AB40001B0550911C050E94C1DE18160CF47BC039
:10AB500060910105709102058091030590910405B3
:10AB600020E030E048EC52E40E9427DF20E030E0B3
:10AB700048EA51E40E9427DF2091F6043091F7045F
:10AB80004091F8045091F9040E9440E16B017C016E
:10AB90006EE578E088E894E10E94D6C768E874E141
:10ABA000CE0101960E94BAC842E350E070E060E036
:10ABB000CE0101960E94151ACE0101960E9457C837
:10ABC00022E0B701A601CE0101960E945FC868E5A8
:10ABD00078E0CE0107960E94C3C8BE016F5F7F4F29
:10ABE000CE0107960E9434C762E578E00E941EC736
:10ABF000BC018EE894E10E94FBC7CE0107960E943B
:10AC000057C8CE0101960E9457C86EE874E1CE0184
:10AC100001960E94BAC842E350E06FEF7FEFCE0189
:10AC200001960E947B13CE0101960E9457C8809125
:10AC30006D0E882309F41FCA60E273E080E090E0A3
:10AC40000E94FF6C18CA20912D0530912E0540916D
:10AC50002F0550913005C701B6010E9449E287FFD8
:10AC600005C0C701B6010E9433AF7ACF60911505C8
:10AC700070911605809117059091180571CF0E946B
:10AC8000571362E978E08EE894E10E94D6C76EE837
:10AC900074E1CE0101960E94BAC84AE050E070E02B
:10ACA00060E0CE0101960E94151ACE0101960E9425
:10ACB00057C869E878E088E894E10E94D6C768E858
:10ACC00074E1CE0101960E94BAC844E150E06FEFF2
:10ACD0007FEFCE0101960E947B13CE0101960E9468
:10ACE00057C88091940C9091950C8230910509F091
:10ACF00041C00E946DC4811104C01092950C109245
:10AD0000940C8091940C9091950C029709F448C092
:10AD10006DE778E08EE894E10E94D6C76EE874E1B2
:10AD2000CE0101960E94BAC84AE050E070E060E0AF
:10AD3000CE0101960E94151ACE0101960E9457C8B5
:10AD40006EE874E1CE0101960E94BAC86EE277E027
:10AD5000CE0101960E941EC768E874E10E9434C7C4
:10AD6000BC018EE894E10E94FBC7CE0101960E94CF
:10AD700057C85DCF892B61F60E946DC4882339F0D6
:10AD800082E090E09093950C8093940CBACF0E944F
:10AD90006DC48111F5CF0E946DC48111F1CFB1CF87
:10ADA0008AE090E00E9493166B017C0120E030E085
:10ADB000A9010E94C1DE181634F08AE090E00E94DA
:10ADC00093166B017C01FBE0AF2EB12C20E030E04C
:10ADD00042ED53E4C701B6010E94C1DE18168CF0A3
:10ADE00091E0A91AB10869F068EC70E080E090E0A9
:10ADF0000E94FF6C83E090E00E9493166B017C013F
:10AE0000E5CF20E030E0A901C701B6010E94C1DE14
:10AE100018166CF16FE678E08EE894E10E94D6C7D0
:10AE20006EE874E1CE0101960E94BAC842E350E098
:10AE30006FEF7FEFCE0101960E947B13CE0101964A
:10AE40000E9457C866E678E088E894E10E94D6C779
:10AE500068E874E1CE0101960E94BAC842E350E06E
:10AE600070E060E0CE0101960E94151ADCCE20E071
:10AE700030E048EC52E4C701B6010E94C1DE21E097
:10AE800087FF20E0B701A601CE0101960E945FC8AE
:10AE900067E578E0CE0107960E94C3C8BE016F5FE8
:10AEA0007F4FCE0107960E9434C76CE578E00E9480
:10AEB0001EC7BC018EE894E10E94FBC7CE01079635
:10AEC0000E9457C8CE0101960E9457C8A9CF0E9480
:10AED000326D0E94231DCFC8E0908D04F0908E0447
:10AEE00060E678E088E894E10E949AC50E945713D2
:10AEF00068E874E1CE0101960E94BAC84AE050E0C9
:10AF00006FEF7FEFCE0101960E94151ACE010196D8
:10AF10000E9457C8C7010E94FC12698B7A8B8B8BE9
:10AF20009C8B8090D7049090D804A090D904B090C6
:10AF3000DA04A50194016091D3047091D404809146
:10AF4000D5049091D6040E9461E02B013C0120E0E1
:10AF500030E0A9010E94C1DE882309F48AC0C090B4
:10AF6000DF04D090E004E090E104F090E20420E0FF
:10AF700030E0A901C701B6010E94C1DE18160CF02D
:10AF800078C02091DB043091DC044091DD045091C5
:10AF9000DE042D873E874F87588BC701B6010E947C
:10AFA000C1DE882309F465C0A70196016D857E8501
:10AFB0008F8598890E9440E10E9498E26D877E8784
:10AFC0008F87988BA501940169897A898B899C89DF
:10AFD0000E9461E0A30192010E9440E12D853E851F
:10AFE0004F8558890E9427DF0E94BAE19B01AC017E
:10AFF000C701B6010E9427DF6B017C0168E874E19C
:10B00000CE0101960E94BAC84AE050E070E060E0CC
:10B01000CE0101960E94151ACE0101960E9457C8D2
:10B0200020E030E64AEE56E4C701B6010E9449E24C
:10B0300018161CF56CE978E08EE894E10E94D6C7FA
:10B040006EE874E1CE0101960E94BAC84AE050E071
:10B050006FEF7FEFCE0101960E947B13CE01019628
:10B060000E9457C864E670E080E090E00E94FF6CA8
:10B07000DECDC12CD12C7601C1CF21E0B701A601D4
:10B08000CE0107960E945FC86AE678E0CE0101967D
:10B090000E94C3C8BE01695F7F4FCE0101960E9426
:10B0A00034C76EE678E00E941EC7BC018EE894E1CA
:10B0B0000E94FBC7CE0101960E9457C8CE01079699
:10B0C0000E9457C8BDCFE0900A02F0900B020E9488
:10B0D000571365E070E080E090E00E94FF6C809183
:10B0E0000D1340E050E0BA018330DCF4C7010E9448
:10B0F0000A126B017C0160910E1370910F13072EE1
:10B10000000C880B990B0E94C8DEA70196010E94D3
:10B1100027DF20E030EC4FE754E40E9440E1AB0130
:10B12000BC0123E0CE0101960E945FC86BE478E089
:10B13000CE0107960E94C3C8BE016F5F7F4FCE014C
:10B1400007960E9434C762E278E00E941EC7BC01E5
:10B150008EE894E10E94FBC7CE0107960E9457C873
:10B16000CE0101960E9457C862E778E006C9809137
:10B17000B00C91E089278093B00C80916D0E8823EC
:10B1800031F06EE874E18BE99FE00E9460D168ECD9
:10B1900070E080E090E054CD10926D0E0C943B5026
:10B1A00081E080936D0E80939113809188138823A2
:10B1B00049F16AEF7AE08AE994E10E949AC586EE45
:10B1C0009FEF9093E10D8093E00D20918B133091D0
:10B1D0008C1380918D1390918E138217930724F016
:10B1E00010928E1310928D1310927F131092801371
:10B1F00010928113109282136CE271E080E090E073
:10B200000E94FF6C6AE974E180EA94E10E94FBC746
:10B210008091E00D9091E10D9093640E8093630E08
:10B220000C943B500E94D84A0C943B5085ED90E121
:10B230000E94DCB040E052EC61E070E085ED90E10E
:10B240000E944F168CED95E0A0E0B0E08093D910FD
:10B250009093DA10A093DB10B093DC1064E670E0FA
:10B2600080E090E00E94FF6C8091940C9091950C8E
:10B27000019709F0D3C083E090E00E94B8178111D4
:10B280000BC01092950C1092940C8091940C90919C
:10B29000950C019709F0DBC063EC78E08EE894E14F
:10B2A0000E94D6C76EE874E1CE0101960E94BAC82A
:10B2B000CE0101960E94291FCE0101960E9457C817
:10B2C00062E370E080E090E00E94FF6C6EE874E161
:10B2D000CE0101960E94BAC842E350E06FEF7FEFC3
:10B2E000CE0101960E94151ACE0101960E9457C800
:10B2F00067EB78E088E894E10E94D6C768E874E1DB
:10B30000CE0101960E94BAC844E150E06FEF7FEF92
:10B31000CE0101960E947B13CE0101960E9457C870
:10B320008BEB8F838AEA888781E08987680118011F
:10B33000412C512C3201C6016AE070E00E94D8E332
:10B34000892B49F443E050E0BE01695F7F4F85EDF2
:10B3500090E10E944CA965E070E080E090E00E94DE
:10B36000FF6C5FEFC51AD50A7801812C912C54012E
:10B3700085ED90E10E94C3A9892B39F484E08816F9
:10B380009104A104B1040CF081C096E0E916F10427
:10B390000CF07CC085ED90E10E94C3A9892B71F06F
:10B3A00085ED90E10E94A1A9E1E0F0E0EC0FFD1F26
:10B3B000EE0DFF1D8083AFEFEA1AFA0A65E070E038
:10B3C00080E090E00E94FF6CB6E0EB16F10401F51E
:10B3D00099818F8198131CC09A818885981318C011
:10B3E0009B818985981314C08D8190E0B0E0A0E026
:10B3F000BA2FA92F982F88272C81820F911DA11D6C
:10B40000B11D480E591E6A1E7B1EEFEF2E1A3E0A12
:10B41000FFEF8F1A9F0AAF0ABF0AAACF81E090E020
:10B420000E94B817882339F081E090E09093950C42
:10B430008093940C2ACF83E090E00E94B81781118A
:10B44000F3CF83E090E00E94B8178111EDCF6BED50
:10B4500078E088E894E10E94D6C768E874E1CE01FC
:10B4600001960E94BAC844E150E06FEF7FEFCE0131
:10B4700001960E947B13CE0101960E9457C86FEC83
:10B4800078E08EE894E10E94D6C74AC034E02316E3
:10B49000310434F440E9C41641E0D40609F04BCF3E
:10B4A000C301B2010E94C8DE20E030E040E251E476
:10B4B0000E9440E120E030E040E85EE30E9427DFA8
:10B4C0006B017C0120E030E040EA51E40E9449E257
:10B4D00018160CF055C021E0B701A601CE01019667
:10B4E0000E945FC86CE67AE0CE0107960E94C3C84E
:10B4F000BE016F5F7F4FCE0107960E9434C76AE797
:10B5000078E00E941EC7BC018EE894E10E94FBC750
:10B51000CE0107960E9457C8CE0101960E9457C8D7
:10B520006EE874E1CE0101960E94BAC84AE050E08C
:10B5300070E060E0CE0101960E94151ACE010196DE
:10B540000E9457C86EE874E1CE0101960E94BAC805
:10B550006EE277E0CE0101960E941EC768E874E1B2
:10B560000E9434C7BC018EE894E10E94FBC7CE0163
:10B5700001960E9457C885ED90E10E94DCB057CB40
:10B580006BEA78E07ECF66E779E0CE0101960E9413
:10B59000B1C84AE050E06FEF7FEFCE0101960E9404
:10B5A0007B13CE0101960E9457C860919E04709152
:10B5B0009F048091F0049091F1040E940E1474E1B4
:10B5C000872E912CA12CB12CD12CC12C4FEFC41A59
:10B5D000D40AC501B4010E94FF6C60919E04709171
:10B5E0009F048091F0049091F1040E940E147C015C
:10B5F00053E0C516D10434F02EE1C216D10444F450
:10B60000EF2851F034E1830E911CA11CB11CDECF58
:10B61000E114F10409F00CC18091F0049091F1045F
:10B620008B30910509F0DFC080912515909126158A
:10B63000A0912715B09128158093DC0D9093DD0D16
:10B64000A093DE0DB093DF0D80912115909122150E
:10B65000A0912315B09124158093D80D9093D90D06
:10B66000A093DA0DB093DB0D4091DC0D5091DD0D10
:10B670006091DE0D7091DF0D21E0CE0101960E94F8
:10B680005FC86DEB76E0CE0107960E94C3C8BE018D
:10B690006F5F7F4FCE0107960E9434C7BC018EE8D2
:10B6A00094E10E94FBC7CE0107960E9457C8CE01C5
:10B6B00001960E9457C84091D80D5091D90D6091C4
:10B6C000DA0D7091DB0D21E0CE0101960E945FC87A
:10B6D0006DE778E0CE0107960E94C3C8BE016F5F98
:10B6E0007F4FCE0107960E9434C7BC018EE894E1DB
:10B6F0000E94CFC7CE0107960E9457C8CE0101967F
:10B700000E9457C865E578E08EE894E10E94C5C7BD
:10B7100061E37CE0CE0101960E94C3C844E150E0A1
:10B7200070E060E0CE0101960E94151ACE010196EC
:10B730000E9457C8C090DC0DD090DD0DE090DE0D6A
:10B74000F090DF0D20E030E0A901C701B6010E94B2
:10B7500049E220E030E040E05FE387FD64C0C701DC
:10B76000B6010E9462E00E94ECE1AB01BC01CE0197
:10B7700001960E94A4C5BE016F5F7F4F88E894E1E7
:10B780000E9412C8CE0101960E9457C860E087E06F
:10B790000E94FAAC68E874E186E196E10E9452D119
:10B7A0006FED86E196E10E9435CB63E878E086E1B3
:10B7B00096E10E947CCC6091D80D7091D90D80915A
:10B7C000DA0D9091DB0D0E94ECE14AE050E086E159
:10B7D00096E10E942FCC65E578E086E196E10E9433
:10B7E0007CCC0C94F0518631910509F41DCF0C9757
:10B7F00009F03ACF8091CF0D9091D00DA091D10D4D
:10B80000B091D20D8093DC0D9093DD0DA093DE0DF1
:10B81000B093DF0D8091CB0D9091CC0DA091CD0D0B
:10B82000B091CE0D19CFC701B6010E9461E09BCF48
:10B830008FEFE816F806D4F068E679E0CE010196BD
:10B840000E94B1C84AE050E070E060E0CE0101968D
:10B850000E94151ACE0101960E9457C865E479E04E
:10B860008EE894E10E94D6C70C943B509EEFE916F7
:10B870009FEFF90681F167E379E0CE0101960E941E
:10B88000B1C84AE050E070E060E0CE0101960E944D
:10B89000151ACE0101960E9457C868E279E08EE839
:10B8A00094E10E94D6C7B701CE0101960E94D1C58E
:10B8B000BE016F5F7F4F8EE894E10E94CFC7CE013B
:10B8C00001960E9457C862E179E08EE894E10E94F7
:10B8D00047C70C943B5067E079E0CE0101960E9487
:10B8E000B1C84AE050E070E060E0CE0101960E94ED
:10B8F000151ACE0101960E9457C867EE78E0B0CFC6
:10B900008091A804882311F40C943B5061E37CE0FF
:10B91000CE0101960E94C3C84AE050E061E070E0A9
:10B92000CE0101960E94151ACE0101960E9457C8B9
:10B930000E9484360C943B5080916D0E811109C099
:10B94000809183136EE1462E512C612C712C88233B
:10B9500029F053E0452E512C612C712C64E879E0DC
:10B960008EE894E10E94D6C76EE874E1CE0101969C
:10B970000E94BAC84AE050E06FEF7FEFCE01019617
:10B980000E947B13CE0101960E9457C8812C912CF6
:10B9900054011D861E861F86188A83E20E94DFAC32
:10B9A00067E070E089EC94E10E94071489EC94E16F
:10B9B0000E94887366E970E080E090E00E94FF6C6E
:10B9C00083E20E94DFAC60E270E089EC94E10E94C7
:10B9D000071489EC94E10E94887366E970E080E0C6
:10B9E00090E00E94FF6C42E050E063E270E089EC7E
:10B9F00094E10E94D473C12CD12C760180914A0F1E
:10BA000090914B0F891B990B181619065CF40E9434
:10BA100027ADFE2CED2CDC2CCC24C80ED11CE11C57
:10BA2000F11CECCFC701B6010E94C8DE2AE939E952
:10BA300049E95FE30E9440E10E94ECE1AB01BC01F7
:10BA400084169506A606B70614F44A015C01CE01D9
:10BA500007960E94A4C5BE01695F7F4FCE01019683
:10BA60000E94BAC866E878E0CE0101960E941EC71F
:10BA7000BC0188E894E10E94FBC7CE0101960E94B8
:10BA800057C8CE0107960E9457C868E874E1CE01F6
:10BA900001960E94BAC84EE150E070E060E0CE012D
:10BAA00001960E945C19CE0101960E9457C82D850F
:10BAB0003E854F8558892F5F3F4F4F4F5F4F2D87F2
:10BAC0003E874F87588B42165306640675060CF066
:10BAD00064CFB501A401CE0107960E94A4C5BE01A2
:10BAE000695F7F4FCE0101960E94BAC866E878E090
:10BAF000CE0101960E941EC7BC0188E894E10E9415
:10BB0000FBC7CE0101960E9457C8CE0107960E943E
:10BB100057C868E874E1CE0101960E94BAC84AE0AD
:10BB200050E070E060E0CE0101960E94151ACE014F
:10BB300001960E9457C8B501A401CE0101960E944A
:10BB4000A4C565EC78E0CE0107960E94C3C8BE018B
:10BB50006F5F7F4FCE0107960E9434C76AE878E096
:10BB60000E941EC76EE874E10E9434C7BC018EE8D3
:10BB700094E10E94FBC7CE0107960E9457C8CE01F0
:10BB800001960E9457C862E370E080E090E058C8D8
:10BB9000E0900802F090090281E08093FA0464E6E4
:10BBA00070E080E090E00E94FF6C0E945713C70194
:10BBB0000E940A120E94ECE120E034E0A901461B39
:10BBC000570BBA01CE0101960E94D1C56FE878E00B
:10BBD000CE0107960E94C3C8BE016F5F7F4FCE01A2
:10BBE00007960E9434C7BC018EE894E10E94FBC70F
:10BBF000CE0107960E9457C8CE0101960E9457C8F1
:10BC000060E087E00E94FAAC64E979E0CE01019639
:10BC10000E94B1C842E350E068E070E0CE010196B6
:10BC20000E94151ACE0101960E9457C86EE874E171
:10BC3000CE0101960E94BAC842E350E06FEF7FEF59
:10BC4000CE0101960E947B13CE0101960E9457C837
:10BC500066E978E0CE0101960E94C3C86EE874E1FF
:10BC6000CE0101967BC880910602909107020E9446
:10BC70000A120E94ECE17093970C6093960C62E3B9
:10BC800070E080E090E00E94FF6C6091960C7091F3
:10BC9000970CCE0101960E94D1C5BE016F5F7F4F08
:10BCA0008EE894E10E9412C8CE0101960E9457C806
:10BCB00080911F1590912015892B09F45EC06BE1CE
:10BCC00075E1CE0107960E94BAC8BE01695F7F4F39
:10BCD000CE0101960E94BAC844E150E070E060E0F5
:10BCE000CE0101960E94151ACE0101960E9457C8F6
:10BCF00060EA78E0CE0101960E94C3C86EE874E164
:10BD0000CE0101960E9434C7BC0188E894E10E94EC
:10BD1000FBC7CE0101960E9457C868E874E1CE01C6
:10BD200001960E94BAC844E150E06FEF7FEFCE0168
:10BD300001960E947B13CE0101960E9457C8BE0156
:10BD4000695F7F4FCE0101960E94BAC86EE277E02C
:10BD5000CE0101960E941EC768E874E10E9434C7B4
:10BD6000BC018EE894E10E94FBC7CE0101960E94BF
:10BD700057C8CE0107960C9415566BEA78E088E810
:10BD800094E10E949AC568E874E1CE0101960E9490
:10BD9000BAC844E150E070E060E0CE0101960E9434
:10BDA000151ACE0101960E9457C86FE878E0CE01BF
:10BDB00001960E94C3C86EE874E1CE0101960E940C
:10BDC00034C7BC0188E894E10E94FBC7CE0101960C
:10BDD0000E9457C868E874E1CE0101960E94BAC873
:10BDE00044E150E06FEF7FEFCE0101960E947B139C
:10BDF000CE0101960E9457C860EA78E02BCF80916F
:10BE0000A804882311F40C943B5080916D0E81118D
:10BE100004C080918313882331F082E090E00E9477
:10BE2000F7430C943B50C0909504D0909604E0905A
:10BE30009704F090980420E030E040E450E4C7011B
:10BE4000B6010E9449E218160CF054C020E030E020
:10BE50004AEF54E4C701B6010E9427DF0E94ECE1DB
:10BE60006B017C010E94571360E080E00E94FAACF5
:10BE700065EA79E086E196E10E9472D161E080E0B6
:10BE80000E94FAAC6DE979E086E196E10E9472D1F8
:10BE900064E670E080E090E00E94FF6C0E94326DEA
:10BEA0006093980C7093990C80939A0C90939B0CD0
:10BEB0000E94326D8090980C9090990CA0909A0CF2
:10BEC000B0909B0C681979098A099B096C157D054E
:10BED0008E059F0514F00C943B5083E090E00E9487
:10BEE000F7430E94326D64E170E080E090E00E94D0
:10BEF000FF6CDECF30E3C32E35E7D32EE12CF12CDF
:10BF0000B1CF0E9427338BE99FE00E94CFAB0C9406
:10BF10003B5065EC79E088E894E10E94D6C768E878
:10BF200074E1CE0101960E94BAC84AE050E070E088
:10BF300060E0CE0101960E94151ACE0101960E9482
:10BF400057C830900C028091A80C811105C00E9446
:10BF5000326D81E08093A80C8091A00C811105C006
:10BF60000E94326D81E08093A00C1092D60C10924A
:10BF7000D50CE090D50CF090D60C58E2E516F10403
:10BF80000CF07EC0832D0E94B76CF701EE0FFF1FEF
:10BF9000E654F14F918380830E9409AE20E030E0A7
:10BFA00040EA50E40E9427DF20E030E040E85AE316
:10BFB0000E9427DF6B017C014090CF045090D00499
:10BFC0006090D1047090D204A30192016091CB04DF
:10BFD0007091CC048091CD049091CE040E9461E0D8
:10BFE0009B01AC0160E070E080EC90E40E9461E0B5
:10BFF0004B015C0120E030E0A9010E94C1DE20E09D
:10C0000030E040E650E481111CC0C701B6010E9437
:10C0100027DF60939C0C70939D0C80939E0C9093F3
:10C020009F0C64E170E080E090E00E94FF6C8091E2
:10C03000D50C9091D60C01969093D60C8093D50C8C
:10C0400098CFC701B6010E9427DFA30192010E9489
:10C0500062E020E030E040E850E40E9461E0A501A9
:10C0600094010E9440E120E030E040EC50E40E9466
:10C0700027DF20E030E040E850E40E9462E0C9CFD2
:10C08000C0909C0CD0909D0CE0909E0CF0909F0C6A
:10C0900020E030E0A901C701B6010E9449E287FD16
:10C0A00022C022E0B701A601CE0107960E945FC818
:10C0B0006FEA78E0CE0101960E94C3C8BE01695FB5
:10C0C0007F4FCE0101960E9434C7BC018EE894E1F7
:10C0D0000E94FBC7CE0101960E9457C8CE01079669
:10C0E0000E9457C806C066EB79E08EE894E10E9492
:10C0F000D6C76EE874E1CE0101960E94BAC84AE044
:10C1000050E06FEF7FEFCE0101960E947B135BC082
:10C110008091A804882311F40C943B5080916D0EFB
:10C1200081112EC08091831381112AC0C090950483
:10C13000D0909604E0909704F090980420E030E0CE
:10C140004AE754E4C701B6010E9427DF0E94ECE1F0
:10C150004B015C0120E030E040EA50E4C701B60149
:10C160000E9427DF20E030E040EA50E40E9462E0D5
:10C170000E94ECE1A50194010E94863B0C943B5087
:10C1800021E030E040E050E06AE070E080E090E0E4
:10C19000F3CFC7010E9405380C943B50C7010E94A1
:10C1A00015620C943B5080916E0E882311F40C9410
:10C1B0003B5063E17AE0CE0101960E94B1C8CE0106
:10C1C00001960E942313CE0101960E9457C80C9439
:10C1D0003B508091B80E9091B90E892B81F481E08B
:10C1E00090E09093B90E8093B80E8EE492E00E9496
:10C1F00010B068EC70E080E090E00E94FF6C66E0B8
:10C200007AE0CE0101960E94B1C844E650E06FEF9B
:10C210007FEFCE0101960E947B13CE0101960E9412
:10C2200057C8F0E0E0E019950C943B500E9430C5EF
:10C230000E9457130E94C0100C943B5080918813A9
:10C2400091E0892780938813882309F48BC06FEFCE
:10C2500079E08EE894E10E94D6C70E94326D609327
:10C260007F13709380138093811390938213809136
:10C270008B1390918C13181619065CF420918D1372
:10C2800030918E132817390724F010928E131092D4
:10C290008D1390918F1380918A13981724F0109228
:10C2A0008F131092901380918813809383136EE8FC
:10C2B00074E1CE0101960E94BAC84AE050E068E0FD
:10C2C00070E0CE0101960E94151ACE0101960E94DF
:10C2D00057C86AEE79E0CE0101960E94B1C84AE0E3
:10C2E00050E06FEF7FEFCE0101960E947B13CE01ED
:10C2F00001960E9457C86CED79E08EE894E10E94A7
:10C3000047C768E379E0CE0101960E94C3C86EE892
:10C3100074E1CE0101960E9434C7BC018EE894E11D
:10C320000E94FBC7CE0101960E9457C880916D0EF6
:10C33000809391138CE291E00E943BB080916D0E4E
:10C34000882311F40C943B506AEF7AE08AE994E177
:10C350000E949AC586EE9FEF9093E10D8093E00DC9
:10C360000C943B5067EF79E08EE894E10E94D6C7C9
:10C370009ACFF092E10DE092E00D8BE99FE00E94F0
:10C38000CFAB6EEC79E08EE894E10E94D6C761E312
:10C390007CE0CE0101960E94C3C84AE050E070E004
:10C3A00060E0CE0101960E94151ACE01019698CE4A
:10C3B0000E3F2FEF120711F40C94944F61E37CE0D1
:10C3C0008EE894E10E949AC5F8017C96E632F10568
:10C3D00080F68827E151FE498F4F0C94ECE3C96049
:10C3E000B9611E611661E960D360B961CE60B9615F
:10C3F000B961B961B961B9618A51F5517B52C453D0
:10C40000CB538C553F5667576C576358B758CC5829
:10C41000D058B96112591659C35A805C9C5CC85DEA
:10C42000335EFF5E815F895F8860FF920F931F9389
:10C43000CF93DF93CDB7DEB72C970FB6F894DEBF5E
:10C440000FBECDBF8C0161E37CE08CEA94E10E94D9
:10C450009AC50830110509F011C16AE371E1CE01F6
:10C4600001960E94B1C844E650E06FEF7FEFCE0125
:10C4700001960E94151ACE0101960E9457C86EE2DD
:10C4800071E1CE0101960E94B1C844E650E070E02F
:10C4900060E0CE0101960E947B13CE0101960E94BE
:10C4A00057C88BE99FE00E94CFAB4CE251E061E0BE
:10C4B00070E0CE0107960E941AC980916E0E882303
:10C4C000D1F063EB78E0CE0101960E94C3C8BE01B3
:10C4D000695F7F4FCE0101960E9434C766EB78E01A
:10C4E0000E941EC7BC0182E791E10E9460D1CE018B
:10C4F00001960E9457C86FEE77E0CE0101960E9428
:10C50000C3C8BE016F5F7F4FCE0107960E9403C76D
:10C51000182FCE0101960E9457C8112309F491C02B
:10C5200068EB78E08CEA94E10E949AC588E090E09C
:10C530009093E10D8093E00D6CEA74E1CE010196D9
:10C540000E94BAC8CE0101960E94BD84182FCE0168
:10C5500001960E9457C861E271E1CE0101960E94E6
:10C56000B1C844E650E070E060E0CE0101960E9460
:10C570007B13CE0101960E9457C88BE99FE00E9471
:10C58000CFAB48E552E061E070E0CE0101960E9439
:10C590001AC9BE016F5F7F4FCE0107960E9412C875
:10C5A000CE0101960E9457C880916E0E8823D1F06B
:10C5B00063EB78E0CE0101960E94C3C8BE01695FBB
:10C5C0007F4FCE0101960E9434C766EB78E00E944F
:10C5D0001EC7BC0182E791E10E9460D1CE010196A5
:10C5E0000E9457C86BE778E0CE0101960E94C3C84D
:10C5F000BE016F5F7F4FCE0107960E9403C7082FD1
:10C60000CE0101960E9457C80023D9F06DEB78E067
:10C610008CEA94E10E949AC56CEA74E1CE0101961D
:10C620000E94BAC8CE0101960E94BD84082FCE0197
:10C6300001960E9457C8002321F064E171E11111B5
:10C6400002C06DE071E1CE0101960E94B1C844E6DE
:10C6500050E070E060E0CE0101960E947B13CE01B5
:10C6600001960E9457C861E37CE08CEA94E10E9445
:10C670009AC5CE0107960E9457C8A7C4093F2FEF5D
:10C68000120709F025C163E071E1CE0101960E9415
:10C69000B1C844E650E06FEF7FEFCE0101960E94F3
:10C6A000151ACE0101960E9457C865EF70E1CE01C0
:10C6B00001960E94B1C844E650E070E060E0CE010F
:10C6C00001960E947B13CE0101960E9457C88BE908
:10C6D0009FE00E94CFAB4CE251E064E070E0CE01FD
:10C6E00001960E941AC980916E0E8823D1F063EBE7
:10C6F00078E0CE0107960E94C3C8BE016F5F7F4FEE
:10C70000CE0107960E9434C766EB78E00E941EC7F0
:10C71000BC0182E791E10E9460D1CE0107960E94A0
:10C7200057C870E060E0CE0101960E94F2C6082E64
:10C73000000C990BC0970A9708F0AFC063EC78E043
:10C74000CE0107960E94C3C8BE016F5F7F4FCE0126
:10C7500007960E9434C7BC018CEA94E10E94FBC793
:10C76000CE0107960E9457C889EF9FEF9093E10D85
:10C770008093E00D6CEA74E1CE0107960E94BAC87E
:10C78000CE0107960E94BD84182FCE0107960E9405
:10C7900057C867EE70E1CE0107960E94B1C844E623
:10C7A00050E070E060E0CE0107960E947B13CE015E
:10C7B00007960E9457C88BE99FE00E94CFAB48E5DF
:10C7C00052E065E070E0CE0107960E941AC9BE01F2
:10C7D000695F7F4FCE0101960E9412C8CE01079675
:10C7E0000E9457C880916E0E8823D1F063EB78E0E9
:10C7F000CE0107960E94C3C8BE016F5F7F4FCE0176
:10C8000007960E9434C766EB78E00E941EC7BC0101
:10C8100082E791E10E9460D1CE0107960E9457C83D
:10C8200070E060E0CE0101960E94F2C6082E000C76
:10C83000990BC0970A9788F568EC78E0CE010796C7
:10C840000E94C3C8BE016F5F7F4FCE0107960E9452
:10C8500034C7BC018CEA94E10E94FBC7CE01079665
:10C860000E9457C889EF9FEF9093E10D8093E00DF0
:10C870006CEA74E1CE0107960E94BAC8CE01079611
:10C880000E94BD84082FCE0107960E9457C800233E
:10C8900021F06AED70E1111102C063ED70E1CE018B
:10C8A00007960E94B1C844E650E070E060E0CE0117
:10C8B00007960E947B13CE0107960E9457C861E33A
:10C8C0007CE08CEA94E10E949AC5CE010196D3CE19
:10C8D00069EC70E1CE0101960E94B1C844E650E0D7
:10C8E0006FEF7FEFCE0101960E94151ACE010196DF
:10C8F0000E9457C861E37CE08CEA94E10E949AC5EB
:10C90000053F8FEF1807B9F46DEC78E08CEA94E1FD
:10C910000E949AC56FEB70E1CE0101960E94B1C8EA
:10C9200044E650E06FEF7FEFCE0101960E947B134B
:10C93000CE01019648C1063F2FEF120749F461ED81
:10C9400078E08CEA94E10E949AC565EB70E1E4CF4F
:10C95000013F8FEF180749F467ED78E08CEA94E126
:10C960000E949AC566EA70E1D7CF023F2FEF120707
:10C9700049F46DED78E08CEA94E10E949AC566E98D
:10C9800070E1CACF033F8FEF180709F085C06AE84E
:10C9900070E1CE0101960E94B1C844E650E06FEF0D
:10C9A0007FEFCE0101960E94151ACE0101960E94DA
:10C9B00057C86CE770E1CE0101960E94B1C844E609
:10C9C00050E06FEF7FEFCE0101960E947B13CE0106
:10C9D00001960E9457C844EF51E062E070E0CE013A
:10C9E00001960E941AC9BE016F5F7F4F8CEA94E1E5
:10C9F0000E9412C8CE0101960E9457C869EE78E0E5
:10CA0000CE0101960E94C3C86CEA74E1CE01019682
:10CA10000E9434C7BC018CEA94E10E94FBC7CE019E
:10CA200001960E9457C88091B0149091B114892B3F
:10CA300009F4CBC26CEA74E1CE0101960E94BAC837
:10CA4000CE0101960E94BD84F82ECE0101960E946F
:10CA500057C868EC70E080E090E0FF2009F4C1C2A4
:10CA60000E94FF6C65E87FE0CE0101960E94B1C88C
:10CA700044EF51E06FEF7FEFCE0101960E947B13F0
:10CA8000CE0101960E9457C81093E10D0093E00D6E
:10CA9000C8010E944B4E99C20230110509F096C0A0
:10CAA00060E770E1CE0101960E94B1C844E650E013
:10CAB0006FEF7FEFCE0101960E94151ACE0101960D
:10CAC0000E9457C860E670E1CE0101960E94B1C88D
:10CAD00044E650E06FEF7FEFCE0101960E947B139A
:10CAE000CE0101960E9457C844EF51E066E070E025
:10CAF000CE0101960E941AC9BE016F5F7F4F8CEA7A
:10CB000094E10E9412C8CE0101960E9457C88091FC
:10CB1000B0149091B1140597B0F070E060E08CEA29
:10CB200094E10E94F2C6082E000C990BC0970A9758
:10CB300050F48CEA94E10E9417C6613523EC720729
:10CB400081059105CCF462E570E1CE0101960E9469
:10CB5000B1C848EE53E06FEF7FEFCE0101960E941F
:10CB60007B13CE0101960E9457C861E37CE08CEAFA
:10CB700094E10E949AC557CF0E94C8DE20E030E0C1
:10CB800048EC52E40E9440E1AB01BC0122E0CE013E
:10CB900007960E945FC86FEB79E0CE0101960E9474
:10CBA000C3C8BE01695F7F4FCE0101960E9434C7A2
:10CBB000BC018CEA94E10E94FBC7CE0101960E9461
:10CBC00057C8CE0107960E9457C82DCF083C8FEF5B
:10CBD000180709F0A0C068E470E1CE0101960E9438
:10CBE000B1C844E650E06FEF7FEFCE0101960E949E
:10CBF000151ACE0101960E9457C86BE370E1CE0171
:10CC000001960E94B1C844E650E06FEF7FEFCE017D
:10CC100001960E947B13CE0101960E9457C860EFD7
:10CC200078E0CE0101960E94C3C8CE0101960E9411
:10CC3000BD84CE0101960E9457C86DE270E1CE011D
:10CC400001960E94B1C844E650E06FEF7FEFCE013D
:10CC500001960E94151ACE0101960E9457C861E202
:10CC600070E1CE0101960E94B1C844E650E06FEF3A
:10CC70007FEFCE0101960E947B13CE0101960E94A8
:10CC800057C844EF51E061E070E0CE0101960E9488
:10CC90001AC9BE016F5F7F4F8CEA94E10E9412C8EF
:10CCA000CE0101960E9457C88091B0149091B114A2
:10CCB000892BA9F070E060E08CEA94E10E94F2C652
:10CCC000082E000C990BC0970A9748F48CEA94E15F
:10CCD0000E9417C662307105810591051CF065E15F
:10CCE00070E133CF65EF78E0CE0101960E94C3C8B2
:10CCF000CE0101960E94BD84CE0101960E9457C8C4
:10CD00006AEF78E0CE0101960E94C3C8CE01019679
:10CD10000E94BD840DCE073C2FEF120709F0AEC074
:10CD20006BE070E1CE0101960E94B1C844E650E08C
:10CD30006FEF7FEFCE0101960E94151ACE0101968A
:10CD40000E9457C86EEF7FE0CE0101960E94B1C8E5
:10CD500044E650E06FEF7FEFCE0101960E947B1317
:10CD6000CE0101960E9457C86FEF78E0CE01019680
:10CD70000E94C3C8CE0101960E94BD84CE010196D7
:10CD80000E9457C861EF7FE0CE0101960E94B1C8B2
:10CD900044E650E06FEF7FEFCE0101960E94151A36
:10CDA000CE0101960E9457C863EE7FE0CE01019646
:10CDB0000E94B1C844E650E06FEF7FEFCE010196CC
:10CDC0000E947B13CE0101960E9457C861E37CE06C
:10CDD0008CEA94E10E949AC544EF51E061E070E072
:10CDE000CE0101960E941AC9BE016F5F7F4F8CEA87
:10CDF00094E10E9412C8CE0101960E9457C880910A
:10CE0000B0149091B114892BA9F070E060E08CEA25
:10CE100094E10E94F2C6082E000C990BC0970A9765
:10CE200048F48CEA94E10E9417C6623071058105CE
:10CE300091054CF067ED7FE0CE0101960E94B1C8EC
:10CE400048EE53E0B9CF64E079E0CE0101960E944C
:10CE5000C3C8CE0101960E94BD84CE0101960E94F6
:10CE600057C88CEA94E10E9417C6613071058105AC
:10CE7000910509F0B1CF69E079E044CF063C8FEF2E
:10CE80001807D9F56DEC7FE0CE0101960E94B1C87C
:10CE900044E650E06FEF7FEFCE0101960E94151A35
:10CEA000CE0101960E9457C860EC7FE0CE0101964A
:10CEB0000E94B1C844E650E06FEF7FEFCE010196CB
:10CEC0000E947B13CE0101960E9457C86EE079E064
:10CED000CE0101960E94C3C8CE0101960E94BD8476
:10CEE000CE0101960E9457C860ED77E080E090E0A7
:10CEF0000E94FF6C65E179E005CF0630110509F06D
:10CF000047C060EB7FE0CE0101960E94B1C844E6C5
:10CF100050E06FEF7FEFCE0101960E94151ACE010F
:10CF200001960E9457C863EA7FE0CE0101960E94F5
:10CF3000B1C844E650E06FEF7FEFCE0101960E944A
:10CF40007B13CE0101960E9457C86CE179E0CE01B7
:10CF500001960E94C3C8CE0101960E94BD84CE01F5
:10CF600001960E9457C864E670E080E090E00E945D
:10CF7000FF6C68E97FE0CE0101960E94B1C844E6EB
:10CF800050E06FEF7FEFCE0101960E94151AD0CCD2
:10CF90006FE87FE0CE0101960E94B1C844E650E000
:10CFA0006FEF7FEFCE0101960E947B13CE010196B9
:10CFB0000E9457C861E37CE08CEA94E10E949AC524
:10CFC0000B3E2FEF120709F02ECD2C960FB6F894DA
:10CFD000DEBF0FBECDBFDF91CF911F910F91FF90AC
:10CFE00008950E94FF6C69E77FE0CE0101960E94E0
:10CFF000B1C844EF51E06FEF7FEFCE0101960E9480
:10D000007B1363CC4F925F926F927F928F929F922D
:10D01000AF92BF92EF92FF920F931F93CF93DF9344
:10D02000CDB7DEB762970FB6F894DEBF0FBECDBFA7
:10D030007C015B0181EC9CE00E9486B5892BD9F4D0
:10D0400061E37CE0C7010E94C3C8C70162960FB6C6
:10D05000F894DEBF0FBECDBFDF91CF911F910F912E
:10D06000FF90EF90BF90AF909F908F907F906F90C8
:10D070005F904F9008954091C50C5091C60C6091FF
:10D08000C70C7091C80CCE0107960E94B81A809107
:10D090006E0E882359F163E279E0CE0101960E9479
:10D0A000C3C8BE01695F7F4FCE0101960E9434C79D
:10D0B00060E677E00E941EC7BC0182E791E10E9412
:10D0C00052D1CE0101960E9457C84091C50C509193
:10D0D000C60C6091C70C7091C80C20E182E791E109
:10D0E0000E94BCCA82E791E10E9408CB70E060E038
:10D0F000CE0107960E94F2C6182F8A3211F01092C4
:10D100008C0D0E94326D6093650E7093660E809355
:10D11000670E9093680E61E37CE0CE010D960E944D
:10D12000C3C8812F110F990BC0970A9708F068C0E8
:10D13000CE0107960E9417C66330710581059105DF
:10D140000CF084C001E010E082E0982E0A151B0567
:10D1500009F47CC06CE271E080E090E00E94FF6C1A
:10D1600090920F1210921212412C512C320181EB2D
:10D170009CE00E9486B5892B91F48EE148165104FB
:10D180006104710449F16EE170E080E090E00E947A
:10D19000FF6C8FEF481A580A680A780AE8CF8EE1C8
:10D1A0004816510461047104B9F04091B50C5091D6
:10D1B000B60C6091B70C7091B80CCE0101960E942C
:10D1C000B81ABE016F5F7F4FCE010D960E9412C844
:10D1D000CE0101960E9457C889899A89892B39F016
:10D1E000BE01635F7F4FCE0107960E94CFC70F5FDE
:10D1F0001F4F61E37CE0CE010D960E949AC5A6CF39
:10D200006CE271E080E090E00E94FF6C82E080932D
:10D210000F1210921212812C912C540181EB9CE080
:10D220000E9486B5892B61F58EE188169104A104D0
:10D23000B10409F043C089899A89892B39F0BE016C
:10D24000635F7F4FCE0107960E94CFC764E670E010
:10D2500080E090E00E94FF6C82E080930F121092B9
:10D260001212BE01695F7F4FC7010E94A8C8CE019C
:10D270000D960E9457C8CE0107960E9457C8E5CE6A
:10D280008EE188169104A104B104A9F24091B50C75
:10D290005091B60C6091B70C7091B80CCE0101960C
:10D2A0000E94B81ABE016F5F7F4FCE010D960E949B
:10D2B00012C8CE0101960E9457C8BDCF6EE170E042
:10D2C00080E090E00E94FF6C8FEF881A980AA80A0D
:10D2D000B80AA4CFAF92BF92CF92DF92EF92FF92A3
:10D2E0000F931F93CF93DF93CDB7DEB72C970FB675
:10D2F000F894DEBF0FBECDBF7C015B010E943FB43E
:10D30000182F811117C061E37CE0C7010E94C3C8D8
:10D31000C7012C960FB6F894DEBF0FBECDBFDF91CC
:10D32000CF911F910F91FF90EF90DF90CF90BF9022
:10D33000AF9008958A3211F010928C0D0E94326DD8
:10D340006093650E7093660E8093670E9093680EDF
:10D35000612FCE0107960E948FC8812F012E000CED
:10D36000990BC0970A9768F5CE0107960E9417C6D9
:10D3700063307105810591050CF070C001E010E08B
:10D380000A151B0509F46AC062E370E080E090E0D2
:10D390000E94FF6C0E943FB4D12CC12C81113BC074
:10D3A0008FEFC81AD80A85E1C816D10409F456C00F
:10D3B0006EE170E080E090E00E94FF6C0E943FB45C
:10D3C000EDCF612FCE0101960E948FC8BE016F5F25
:10D3D0007F4FCE0107960E9412C8CE0101960E948F
:10D3E00057C862E370E080E090E00E94FF6C0E940A
:10D3F0003FB410E000E0811121C00F5F1F4F0F31DB
:10D40000110561F16EE170E080E090E00E94FF6C38
:10D410000E943FB4F0CF682FCE0101960E948FC8C2
:10D42000BE016F5F7F4FCE0107960E94CFC7CE012E
:10D4300001960E9457C80F5F1F4FA2CF682FCE01E1
:10D4400001960E948FC8BE016F5F7F4FCE01079685
:10D450000E94CFC7CE0101960E9457C8BE01695FE6
:10D460007F4FC7010E94A8C8CE0107960E9457C8E7
:10D470004FCF8DEE99EA892B49F080E090E0892B1F
:10D4800029F00E94EDA981110E94000083EE99EA23
:10D49000892B49F080E090E0892B29F00E94E3A9D4
:10D4A00081110E94000089ED99EA892B49F080E002
:10D4B00090E0892B29F00E94D9A981110E940000D7
:10D4C0008FEC99EA892B49F080E090E0892B29F0D4
:10D4D0000E94CFA981110C940000089581508231DF
:10D4E00008F05AC0E82FF0E08827E658F5498F4F3A
:10D4F0000C94ECE39A6A9E6A8C6A926A966ACC6A89
:10D50000A16AA76AAB6AB16AB56AB96ABF6AC36A37
:10D51000CC6AC76ACD6AD16A809180008F77809388
:10D5200080000895809180008F7DF9CF80918000E8
:10D53000877FF5CF84B58F7784BD089584B58F7DBF
:10D54000FBCF8091B0008F778093B00008958091D9
:10D55000B0008F7DF9CF809190008F7780939000FD
:10D560000895809190008F7DF9CF80919000877F02
:10D57000F5CF8091A0008F778093A00008958091CF
:10D58000A0008F7DF9CF8091A000877FF5CF80919B
:10D5900020018F77809320010895809120018F7D55
:10D5A000F9CF80912001877FF5CFDC0180E06150C9
:10D5B00090F09D919827E92FEF70F0E0E456F34E3C
:10D5C0002491E92FE295EF70F0E0E455F34EE491F9
:10D5D000822F8E27ECCF089580914A0F90914B0FA8
:10D5E000891B990B08952091370E260F3327331F7F
:10D5F00021323105ECF42091720FFC0190E080E0C3
:10D60000243069F082E00895A091370E2191AC0199
:10D61000495E514FA40FB52FB11D2C93019686176B
:10D6200098F38091370E680F6093370E80E008956D
:10D6300081E00895089508950895E0914B0F809139
:10D640004A0FE81730F4F0E0E65DF04F808190E09B
:10D6500008958FEF9FEF089590914B0F80914A0F9F
:10D660002FEF3FEF981748F4E92FF0E0E65DF04F19
:10D67000208130E09F5F90934B0FC9010895CF92B6
:10D68000DF92EF92FF920F931F93CF93DF937C0172
:10D69000CB018A012091780F222389F0EB016B01E5
:10D6A000C40ED51ECC15DD0569F06991D701ED9149
:10D6B000FC910190F081E02DC7011995F3CF642F03
:10D6C0000E94F36AC801DF91CF911F910F91FF90E3
:10D6D000EF90DF90CF900895CF93DF931F92CDB757
:10D6E000DEB769832091780F2223F9F020919A0FF9
:10D6F000203258F021E030E0FC013383228390E0B7
:10D7000080E00F90DF91CF9108958091790FE82FFD
:10D71000F0E0E658F04F998190838F5F8093790F06
:10D7200080939A0F81E090E0ECCF61E0CE0101960A
:10D730000E94F36AF7CF90E080E008950C94DAE459
:10D74000E1EEF2E114A215A216A217A210A611A6EC
:10D7500012A613A681E084A729E130E036A725A709
:10D7600087A780E090E0A0EAB0E480AB91ABA2ABE9
:10D77000B3AB80E090E0A8EAB1E484AB95ABA6AB94
:10D78000B7AB8093F6049093F704A093F804B0939A
:10D79000F90480E090E0A0E8BFE380932B1390931E
:10D7A0002C13A0932D13B0932E138093F204909317
:10D7B000F304A093F404B093F5041092581310925C
:10D7C00057138BE090E090935A13809359139093E2
:10D7D000F1048093F0041092681310926713109272
:10D7E00078131092771390E080E00C9465B0FC0100
:10D7F000A48DA80FB92FB11DA35ABF4F2C91848DB2
:10D8000090E001968F739927848FA689B7892C930E
:10D81000A089B1898C91837080648C93938D848D61
:10D82000981306C00288F389E02D80818F7D808364
:10D830000895CF93DF93282F30E0F901EA56F24E96
:10D840008491F901E05BF24ED491F901E65FF24E6A
:10D85000C491CC23A1F081110E946E6AEC2FF0E0FC
:10D86000EE0FFF1FE051F34EA591B491EC91ED2323
:10D8700081E090E009F480E0DF91CF91089580E0AD
:10D8800090E0FACF862F0C94196C1F93CF93DF93FF
:10D89000282F30E0F901EA56F24E8491F901E05B5D
:10D8A000F24ED491F901E65FF24EC491CC23A9F077
:10D8B000162F81110E946E6AEC2FF0E0EE0FFF1F11
:10D8C000EA52F34EA591B4918FB7F894EC911111EF
:10D8D00008C0D095DE23DC938FBFDF91CF911F91DD
:10D8E0000895DE2BF8CF862F642F0C94456CCF93D0
:10D8F000DF9390E0FC01E05BF24E2491865F924E54
:10D90000FC0184918823C9F090E0880F991FFC01E5
:10D91000E454F34EA591B491FC01EA52F34EC59143
:10D92000D49161110DC09FB7F8948C9120958223FA
:10D930008C938881282328839FBFDF91CF910895FE
:10D94000623051F49FB7F8943C91822F80958323E5
:10D950008C93E8812E2BEFCF8FB7F894EC912E2B80
:10D960002C938FBFEACF862F642F0C94776C86336D
:10D9700008F0865320917B00982F9870277F922B78
:10D9800090937B002091FA0490E4299F9001112448
:10D990008770822B80937C0080917A0080648093D2
:10D9A0007A0080917A0086FDFCCF8091780090917A
:10D9B000790008953FB7F89480915F0E9091600EC2
:10D9C000A091610EB091620E26B5A89B05C02F3FB5
:10D9D00019F00196A11DB11D3FBFBA2FA92F982F95
:10D9E0008827BC01CD01620F711D811D911D42E090
:10D9F000660F771F881F991F4A95D1F708958F9258
:10DA00009F92AF92BF92CF92DF92EF92FF926B0103
:10DA10007C010E94DA6C4B015C01C114D104E10469
:10DA2000F104B9F00E94DA6C681979098A099B0936
:10DA3000683E73408105910580F321E0C21AD10848
:10DA4000E108F10888EE880E83E0981EA11CB11C45
:10DA5000E4CFFF90EF90DF90CF90BF90AF909F907A
:10DA60008F9008952FB7F89460915B0E70915C0EC3
:10DA700080915D0E90915E0E2FBF08951F920F92C0
:10DA80000FB60F9211242F933F938F939F93AF93D1
:10DA9000BF9380915B0E90915C0EA0915D0EB09152
:10DAA0005E0E30915A0E23E0230F2D3758F5019664
:10DAB000A11DB11D20935A0E80935B0E90935C0EB6
:10DAC000A0935D0EB0935E0E80915F0E9091600EFC
:10DAD000A091610EB091620E0196A11DB11D8093BF
:10DAE0005F0E9093600EA093610EB093620EBF9193
:10DAF000AF919F918F913F912F910F900FBE0F90FB
:10DB00001F90189526E8230F0296A11DB11DD2CFB4
:10DB10000C94E8DF0895DF92EF92FF920F931F932A
:10DB2000CF93DF937C018B01D42EDC011696ED910F
:10DB3000FC9113861586148612861186108617822C
:10DB40001682158214821382C0E0B801F701868123
:10DB500097810E9453C2D82F882329F0DC1629F020
:10DB6000CF5FDC1690F7D0E009C067E0C8010E94E3
:10DB7000D56AD80117969C918913F2CF8D2FDF912A
:10DB8000CF911F910F91FF90EF90DF900895DC01EE
:10DB90002C911196ED91FC91F8948181822B8183D7
:10DBA0009281322F30959323928387E090E0019702
:10DBB000F1F781818323818383E290E00197F1F77C
:10DBC00090817894EFECF0E03197F1F7922381E0C7
:10DBD00009F480E00895FC0190810180F281E02D3C
:10DBE000292F209560FF14C0F894828182238283BC
:10DBF0008181892B8183A3E2B0E01197F1F78281C3
:10DC0000982B9283789487ED90E00197F1F708952F
:10DC1000F8948281822382838181892B8183AFEF73
:10DC2000B0E01197F1F78281982B928378948FE07E
:10DC300090E0EBCFDF92EF92FF920F931F93CF9381
:10DC4000DF93EC01D62EE42E08E010E0FF24F394DD
:10DC500061E08D2D8F2109F460E0CE010E94EB6D13
:10DC6000FF0C01501109A1F7E11010C0F894E981EF
:10DC7000FA8191818881809589238183E981FA8164
:10DC8000928188818095892382837894DF91CF91D6
:10DC90001F910F91FF90EF90DF900895EF92FF9208
:10DCA0000F931F93CF93DF938C017B0140E065E5D9
:10DCB0000E941A6EE70188E0E80EF11C699140E0CD
:10DCC000C8010E941A6ECE15DF05C1F7DF91CF9112
:10DCD0001F910F91FF90EF900895FC0190810180BA
:10DCE000F281E02DF8948181292F20958223818370
:10DCF00078943DE743E050E0315029F1DA01119783
:10DD0000F1F780818923C1F3F89482818223828391
:10DD10008181892B81837894ABE7B7E01197F1F784
:10DD2000F894818182238183A3E1B1E01197F1F717
:10DD30008081982381E009F080E07894E3E6F6E0C2
:10DD40003197F1F7089580E008958F929F92AF92F6
:10DD5000BF92CF92DF92EF92FF92CF93DF93EC01CD
:10DD60008E819F810E946D6E40E06CEC8E819F8160
:10DD70000E941A6E488164E48E819F810E941A6E0F
:10DD80008A81882371F1E981E9508EEEC82E82E004
:10DD9000D82EE33038F4F0E0EE0FFF1FED57FA4FC6
:10DDA000C080D1808B81882339F18881811124C082
:10DDB0000E94326D4B015C010D2C000CEE08FF0837
:10DDC0008E819F810E94C76D813059F00E94326D13
:10DDD0006C197D098E099F09681579058A059B05CF
:10DDE00078F3DF91CF91FF90EF90DF90CF90BF90CD
:10DDF000AF909F908F900895B601DD0C880B990B22
:10DE0000DF91CF91FF90EF90DF90CF90BF90AF90D8
:10DE10009F908F900C94FF6C6F927F928F929F9245
:10DE2000AF92BF92CF92DF92EF92FF920F931F9328
:10DE3000CF93DF93EC017B018A018E819F810E9449
:10DE40006D6E811102C090E037C0B7018E819F8155
:10DE50000E944E6E40E06EEB8E819F810E941A6E92
:10DE60007801680189E0C80ED11CAE80BF8088E0CF
:10DE7000882E912C712C66246394C5010E94C76D75
:10DE800081117628660CE1E08E1A9108B1F7F7014E
:10DE900071927F01EC15FD0541F78E819F810E94F3
:10DEA0006D6E813081F668E0C8010E94D56A91E00C
:10DEB000F80120852813C7CF892FDF91CF911F91BB
:10DEC0000F91FF90EF90DF90CF90BF90AF909F9019
:10DED0008F907F906F900895CF93DF9300D000D004
:10DEE00000D0CDB7DEB7AE014F5F5F4F0E940C6F21
:10DEF000882331F08D818F33A9F020F48F31A1F088
:10DF000080E007C08F3521F08F37D1F78CE001C05A
:10DF10008BE029960FB6F894DEBF0FBECDBFDF9120
:10DF2000CF9108958AE0F5CF89E0F3CF0F931F9347
:10DF3000CF93DF93CDB7DEB761970FB6F894DEBF0E
:10DF40000FBECDBF8C01462FBE01665F7F4F0E9482
:10DF50008B6D81110FC060E070E08EEF92EC6196E6
:10DF60000FB6F894DEBF0FBECDBFDF91CF911F91EA
:10DF70000F910895AE014F5F5F4FBE01665F7F4F07
:10DF8000C8010E940C6F882331F36A8170E0762FFC
:10DF90006627770F770F770F298148E0249F90013C
:10DFA0001124262B372B8A858031D1F4688570E0C7
:10DFB0008F81AB01481B5109CA019695982F88277C
:10DFC000979587950E94D8E3CB014097B90153E01C
:10DFD000660F771F5A95E1F760789C01260F371F6F
:10DFE000213854EE35070CF4B6CFB901330F880B46
:10DFF000990B0E94C8DE20E030E040E05CE30E9424
:10E0000027DFADCFEF92FF920F931F93CF93DF9354
:10E0100000D000D01F921F92CDB7DEB78C01DC017B
:10E020001696ED91FC911797138615861486128625
:10E030001186108617821682158214821382149616
:10E040001C92149715961C92EE24E394BE016F5F08
:10E050007F4FF801868197810E9453C2882309F47B
:10E060006FC067E0CE0101960E94D56A988589133A
:10E07000EDCFD8018C91811125C016968D919C9180
:10E080000E946D6EBE016F5F7F4FF80186819781A0
:10E090000E944E6E40E064EBD80116968D919C91E3
:10E0A0000E941A6EF801868197810E94C76DF82E32
:10E0B000D80116968D919C910E946D6EF11002C050
:10E0C000F801E082D8011196FC9089818031A1F19C
:10E0D000BE016F5F7F4FC8010E946C6F8F15D0F437
:10E0E000F8018181D80111968C93119714968C9127
:10E0F00014978F5F14968C938981883231F0B0F435
:10E10000803119F0823209F0A1CFF80185818F5F4B
:10E1100085839CCF8981803111F48CE0E3CFBE01EF
:10E120006F5F7F4FC8010E946C6FDCCF8B3369F348
:10E13000823409F08BCFE9CFFCE0FF1588F2EDCFF8
:10E1400028960FB6F894DEBF0FBECDBFDF91CF91FA
:10E150001F910F91FF90EF9008951F93CF93DF933E
:10E16000EC01162F60E0812F0E94776C612F70E028
:10E17000FB01E05BF24EE491E883FB01E65FF24EC7
:10E18000E491F0E0EE0FFF1FE051F34E8591949182
:10E190009A8389831B861D861C861A861986188693
:10E1A0001F821E821D821C821B82DF91CF911F91D4
:10E1B00008951F920F920FB60F9211240BB60F9273
:10E1C0002F933F934F935F936F937F938F939F937F
:10E1D000AF93BF93EF93FF93809110120E94196C3D
:10E1E00020911312309114122F5F3F4F309314126D
:10E1F0002093131290911212953618F096E0909396
:10E200000F1290910F12943009F46EC0F8F492300E
:10E2100031F1933009F44CC090911112992319F007
:10E22000811171C02F9AFF91EF91BF91AF919F9192
:10E230008F917F916F915F914F913F912F910F90AF
:10E240000BBE0F900FBE0F901F901895953009F4DC
:10E2500057C0963009F791E09093DF124FC08111BB
:10E26000DBCF20911312309114122436310528F49B
:10E270001092141210921312CFCF1092DF1210923C
:10E280001212E091121291E09E0F90931212F0E0A0
:10E290002091131230911412EE0FFF1FEB5EFD4E12
:10E2A00031832083109214121092131293E019C03C
:10E2B000813009F0B1CFE091121291E09E0F90935E
:10E2C0001212F0E02091131230911412EE0FFF1F82
:10E2D000EB5EFD4E318320831092141210921312C4
:10E2E00094E090930F1298CF882359F22091131243
:10E2F000309114122536310508F48ECF95E0F1CF18
:10E3000081118ACFB5CF2F988ECFCF92DF92EF9227
:10E31000FF92CF93DF93EC01072E000C880B990B33
:10E320000E94C8DE6B017C0120E030E040E45FE346
:10E330000E9427DF20E030E048E452E40E9440E100
:10E340000E94ECE1C617D707D4F020E030E040EAA5
:10E350005FE3C701B6010E9427DF20E030E048E418
:10E3600052E40E9440E120E030E040E85FE30E9498
:10E3700062E00E94ECE121E06C177D070CF420E0E4
:10E38000822F90E0DF91CF91FF90EF90DF90CF90C0
:10E3900008950F931F93CF93DF93082F6BE778E0D7
:10E3A00082E791E10E947CCCC7E0D0E010E0B801A8
:10E3B0000C2E02C0759567950A94E2F76170772775
:10E3C00042E050E082E791E10E942FCC219778F75C
:10E3D000DF91CF911F910F9108951092720F81E0FC
:10E3E0008093710F10924C0F61E084E10E94456CA4
:10E3F00061E085E10E94456CE9EBF0E080818E7F71
:10E40000808380818D7F808388E48093B80085E459
:10E410008093BC000895CF93DF9391E09093160E04
:10E420008823B9F0C091B800D091BA008091BC00A7
:10E430008A7B8093BC0060E084E10E94456C60E0D0
:10E4400085E10E94456C0E94ED71D093BA00C093A3
:10E45000B800DF91CF91089585ED8093BC00809145
:10E46000740F9091750FA091760FB091770F07966A
:10E47000A11DB11D23E0B695A795979587952A957F
:10E48000D1F72091BC0024FD03C01092720F0895B3
:10E490004091740F5091750F6091760F7091770FC6
:10E4A000452B462B472B69F30097A105B10541F099
:10E4B00025E32A95F1F700000197A109B109E1CF01
:10E4C0008091730F0C940B721F920F920FB60F92E4
:10E4D00011240BB60F922F933F934F935F936F933B
:10E4E0007F938F939F93AF93BF93EF93FF9380910D
:10E4F000B900887F803609F44DC008F040C08832EA
:10E5000009F4A9C028F5803109F49DC0C8F4882316
:10E5100009F4FBC0883009F496C0FF91EF91BF91D8
:10E52000AF919F918F917F916F915F914F913F91AB
:10E530002F910F900BBE0F900FBE0F901F9018954C
:10E54000883109F488C0803241F78093700F14C07D
:10E55000803409F49DC040F48033B9F38833E9F680
:10E560008093700F85ECB0C0803509F485C0883584
:10E5700009F496C0883489F60E942C72CECF88396F
:10E5800009F48CC038F5883729F050F4883611F03A
:10E59000803719F683E08093720F1092590E57C09E
:10E5A000883809F47BC0803919F0803809F0B5CF7C
:10E5B0008091590E803208F071C0E091590E81E0CF
:10E5C0008E0F8093590E8091BB00F0E0E75CF14F15
:10E5D00080833DC0803B39F0E0F4803A09F479C093
:10E5E000883A09F09ACF84E08093720F1092380E27
:10E5F0001092370EE091710EF091720E1995809184
:10E60000370E81110FC081E08093370E1092170EE4
:10E6100009C0803C09F4A6CF883C09F4A3CF883B0D
:10E6200009F07BCFE091380E81E08E0F8093380E99
:10E63000F0E0E95EF14F80818093BB009091380E4D
:10E640008091370E29C080914D0F8093BB0085ECDF
:10E650008093BC0062CF90916F0F80916E0F9817DE
:10E6600058F5E0916F0F81E08E0F80936F0FF0E00F
:10E67000E25BF04F8081E9CFE0916F0F81E08E0F78
:10E6800080936F0F8091BB00F0E0E25BF04F8083DE
:10E6900090916F0F80916E0F9817C8F285E8D8CFD0
:10E6A000E0916F0F81E08E0F80936F0F8091BB0020
:10E6B000F0E0E25BF04F80838091710F81115CCFBD
:10E6C00081E080934C0F84EA8093BC001092720F1B
:10E6D00024CF85EC8093BC001092720F8091590E6C
:10E6E000803230F4E091590EF0E0E75CF14F108297
:10E6F0006091590E70E0E0916F0EF091700E89E319
:10E700009EE019951092590E08CF1092700F34CFD9
:10E7100081E00C94EFAB0F931F93CF938C01C62F26
:10E72000FC0184810E94DFACF8016385C62B6C2F4D
:10E7300070E089EC94E10E94071489EC94E1CF9198
:10E740001F910F910C9488730F931F93CF938C019B
:10E75000C62F0E948B736C2F6460C8010E948B735C
:10E760006C2F6B7FC8010E948B7383EC90E0019744
:10E77000F1F7CF911F910F9108950F931F93CF93AE
:10E780008C01C62F607F61600E94A47380E1C89FE6
:10E79000B00111246160C8010E94A47381E090E07F
:10E7A000CF911F910F910895862F642F0E943AAD4B
:10E7B00010924B0F80934A0F0895CF938EE10E94E1
:10E7C000DFAC62E070E089EC94E10E94071461E83C
:10E7D00070E089EC94E10E94071489EC94E10E94B6
:10E7E000887346E050E06EE170E089EC94E10E94AD
:10E7F000D47380914A0F90914B0F891B990B069708
:10E8000024F10E9427ADC82F0E9427AD20E0822B63
:10E810009C2B9093270F8093260F0E9427ADC82F23
:10E820000E9427AD20E0822B9C2B9093230F809396
:10E83000220F0E9427ADC82F0E9427AD20E0822B17
:10E840009C2B9093250F8093240FCF91089597FDD3
:10E8500004C09093C6048093C5048091C504909130
:10E86000C604892BC9F468E279E08BEE95E10E9439
:10E870009AC580E090E0AAE7B4E48093100E9093EC
:10E88000110EA093120EB093130E81E090E09093BE
:10E890000F0E80930E0E08958091C5049091C604CA
:10E8A0000197A9F46BE279E08BEE95E10E949AC59D
:10E8B00080E090E0A0E8BFE38093100E9093110EEB
:10E8C000A093120EB093130E83E090E0E0CF8091FE
:10E8D000C5049091C604029759F46EE279E08BEE7C
:10E8E00095E10E949AC589E898E1ADE0B0E4E4CFF3
:10E8F0006FE479E08BEE95E10E949AC583EC95EF89
:10E90000ACE1B1E4D9CFCF93DF93CDB7DEB72C978D
:10E910000FB6F894DEBF0FBECDBF84E10E940EC4D7
:10E920002091100E3091110E4091120E5091130E45
:10E930000E9427DFAB01BC0120910E0ECE01019693
:10E940000E945FC8BE016F5F7F4FCE0107960E9495
:10E95000BAC86BEE75E1CE0107960E9434C7BC01C0
:10E960008EE894E10E94FBC7CE0107960E9457C82B
:10E97000CE0101960E9457C86CE773E184E994E1E7
:10E980000E94D6C78091C5049091C60464E379E0E3
:10E99000039744F066E773E184E994E10E94D6C7E7
:10E9A00061E379E0CE0101960E94C3C86EE874E18C
:10E9B000CE0101960E9434C7BC018EE894E10E940A
:10E9C000FBC7CE0101960E9457C864E974E1CE01ED
:10E9D00001960E94BAC84AE050E06AE070E0CE01B9
:10E9E00001960E94151ACE0101960E9457C865E053
:10E9F00070E080E090E00E94FF6C6EE874E1CE0170
:10EA000001960E94BAC84AE050E06FEF7FEFCE0156
:10EA100001960E947B13CE0101960E9457C82C9646
:10EA20000FB6F894DEBF0FBECDBFDF91CF91089532
:10EA3000EF92FF920F931F93CF93DF93CDB7DEB783
:10EA400068970FB6F894DEBF0FBECDBF8C016EE2A3
:10EA500077E0CE010D960E94C3C867E379E0CE014E
:10EA600043960E94C3C86EE57AE1C8010E94B1C80E
:10EA7000BE016D5E7F4FC8010E94CFC765E57AE198
:10EA8000C8010E9447C788E8E82E83E1F82EF70105
:10EA9000608170E0CE0101960E94D1C5BE016F5F1A
:10EAA0007F4FCE0107960E94BAC8BE01635F7F4FB9
:10EAB000CE0107960E9434C7BC01C8010E94CFC78F
:10EAC000CE0107960E9457C8CE0101960E9457C8F2
:10EAD00068E47AE1C8010E9447C7F7016181062E08
:10EAE000000C770BCE0101960E94D1C5BE016F5F6D
:10EAF0007F4FCE0107960E94BAC8BE01635F7F4F69
:10EB0000CE0107960E9434C7BC01C8010E94CFC73E
:10EB1000CE0107960E9457C8CE0101960E9457C8A1
:10EB20006EE37AE1C8010E9447C7F7016281062EB1
:10EB3000000C770BCE0101960E94D1C5BE016F5F1C
:10EB40007F4FCE0107960E94BAC8BE01635F7F4F18
:10EB5000CE0107960E9434C7BC01C8010E94CFC7EE
:10EB6000CE0107960E9457C8CE0101960E9457C851
:10EB700066E37AE1C8010E9447C7F70163817481A7
:10EB8000CE0101960E94D1C5BE016F5F7F4FCE01BD
:10EB900007960E94BAC8BE016D5E7F4FCE010796F0
:10EBA0000E9434C7BC01C8010E94CFC7CE0107969E
:10EBB0000E9457C8CE0101960E9457C86FE17AE1C2
:10EBC000C8010E9447C7F70165817681CE01019691
:10EBD0000E94D1C5BE016F5F7F4FCE0107960E9494
:10EBE000BAC8BE01635F7F4FCE0107960E9434C74B
:10EBF000BC01C8010E94CFC7CE0107960E9457C82A
:10EC0000CE0101960E9457C866E17AE1C8010E94D0
:10EC100047C7F7016781062E000C770B6F5F7F4FA8
:10EC2000CE0101960E94D1C5BE016F5F7F4FCE011C
:10EC300007960E94BAC8BE01635F7F4FCE01079658
:10EC40000E9434C7BC01C8010E94CFC7CE010796FD
:10EC50000E9457C8CE0101960E9457C86BE07AE126
:10EC6000C8010E9447C7F7016085062E000C770B8C
:10EC7000CE0101960E94D1C5BE016F5F7F4FC801D2
:10EC80000E94CFC7CE0101960E9457C8CE0143967D
:10EC90000E9457C8CE010D960E9457C8C8016896B9
:10ECA0000FB6F894DEBF0FBECDBFDF91CF911F919D
:10ECB0000F91FF90EF9008954F925F926F927F9225
:10ECC0008F929F92AF92BF92CF92DF92EF92FF927C
:10ECD0000F931F93CF93DF93CDB7DEB762970FB635
:10ECE000F894DEBF0FBECDBF8EE492E00E94E8DF55
:10ECF0008093B80E8FE492E00E94E8DF8093B90E13
:10ED00008091B80E9091B90E1816190664F41092FD
:10ED1000EF04019741F41092B90E1092B80E8EE4F0
:10ED200092E00E9410B040E052EC61E070E082E7B7
:10ED300091E10E944F168091EF04882331F068EE34
:10ED400073E080E090E00E94FF6C82E791E10E9416
:10ED5000A1A9182FD82EF8E8AF2EF3E1BF2EACE210
:10ED6000EA2EFF24F394C7010E94E8DFF5018193A6
:10ED70005F01FFEFEF1AFF0A46E2E41642E0F406F5
:10ED800091F78091891318161CF41D3609F011C1F2
:10ED900061E37CE0CE010D960E94C3C810928813F7
:10EDA00088E18093891384E080938A1310928F13F3
:10EDB0001092901363E97BE0CE010D960E949AC5F4
:10EDC00082E993E1009739F044E050E0BC01CE01C4
:10EDD0000D960E948FB081E08093961383E080931C
:10EDE000971382E090E0909399138093981385E0B5
:10EDF00090E090939B1380939A1360E97BE0CE019F
:10EE00000D960E949AC58CE993E1009739F044E091
:10EE100050E0BC01CE010D960E948FB082E080933D
:10EE2000A01383E08093A11382E090E09093A3135A
:10EE30008093A21385E090E09093A5138093A41390
:10EE40006DE87BE0CE010D960E949AC586EA93E1BB
:10EE5000009739F044E050E0BC01CE010D960E94CD
:10EE60008FB083E08093AA138093AB1382E090E08D
:10EE70009093AD138093AC1385E090E09093AF1323
:10EE80008093AE136AE379E0CE010D960E949AC595
:10EE900080EB93E1009739F044E050E0BC01CE01F3
:10EEA0000D960E948FB085EF8093B41383E080931A
:10EEB000B51382E090E09093B7138093B61385E08A
:10EEC00090E09093B9138093B8138CE291E00E9484
:10EED000B2B080916E0E882311F1CE0101960E948E
:10EEE0001875BE016F5F7F4F82E791E10E9460D18C
:10EEF000CE0101960E9457C86CEB7AE182E791E15E
:10EF00000E9472D12AE04AE050E060E070E082E7BF
:10EF100091E10E94BCCA82E791E10E9408CB62E8BD
:10EF20007AE1CE0107960E94B1C8BE01695F7F4FAA
:10EF300082E791E10E9460D1F12CE12C80918A134B
:10EF4000082E000C990BE816F906A4F4B701CE01BF
:10EF500001960E942920BE016F5F7F4F82E791E1F9
:10EF60000E9460D1CE0101960E9457C88FEFE81A27
:10EF7000F80AE4CFCE0107960E9457C880916E0E22
:10EF8000882399F06CE97AE182E791E10E9472D1DD
:10EF90002AE04AEF50E060E070E082E791E10E94F1
:10EFA000BCCA82E791E10E9408CBCE010D960E9477
:10EFB00057C8809191138111809188138093831396
:10EFC0000E94326D60937F1370938013809381133E
:10EFD0009093821300E0123709F431C7E1EEEE2E70
:10EFE000E2E1FE2E4701B12CA12CC5010E94E8DF11
:10EFF000F40181934F01FFEFAF1ABF0A48E9A4164D
:10F00000B10499F78091E1129091E212A091E3127C
:10F01000B091E41285369105A105B1050CF4D9C172
:10F020008093EB049093EC04A093ED04B093EE0472
:10F030008091E5129091E612A091E712B091E8124A
:10F040008093E7049093E804A093E904B093EA0462
:10F050008091E9129091EA12A091EB12B091EC121A
:10F060008093E3049093E404A093E504B093E60452
:10F070006DEF72E1CE0101960E94C3C8BE016F5FC1
:10F080007F4F84E096E10E9412C8CE0101960E9453
:10F0900057C86BE573E1CE0101960E94C3C8BE015B
:10F0A0006F5F7F4F8EEF95E10E9412C8CE010196EF
:10F0B0000E9457C823E030E050E040E064E076E191
:10F0C000CE0107960E94D4C823E030E050E040E033
:10F0D0006EEF75E1CE0101960E94D4C82D813E816C
:10F0E0008B859C852817390709F589819A816F815D
:10F0F0007885009759F06115710509F002C1232B3D
:10F1000009F402C1FC01808190E00DC06115710518
:10F1100009F4FAC0232B09F4F7C0FB01808190E0C9
:10F1200091958195910901E0892B09F000E0CE01CC
:10F1300001960E9457C8CE0107960E9457C8011138
:10F1400006C064E076E18EEF95E10E94FBC78091F6
:10F15000ED129091EE12A091EF12B091F012809307
:10F16000DF049093E004A093E104B093E204809163
:10F17000F1129091F212A091F312B091F4128093D7
:10F18000DB049093DC04A093DD04B093DE04809153
:10F19000F5129091F612A091F712B091F8128093A7
:10F1A000D7049093D804A093D904B093DA04809143
:10F1B000F9129091FA12A091FB12B091FC12809377
:10F1C000D3049093D404A093D504B093D604809133
:10F1D000591390915A139093F1048093F004809105
:10F1E000151390911613A0911713B09118138093D3
:10F1F000F6049093F704A093F804B093F904809177
:10F200002B1390912C13A0912D13B0912E1380935A
:10F21000F2049093F304A093F404B093F504809166
:10F22000051390910613A0910713B09108138093D2
:10F23000CF049093D004A093D104B093D2048091D2
:10F24000091390910A13A0910B13B0910C138093A2
:10F25000CB049093CC04A093CD04B093CE04A090A3
:10F260006713B0906813B5010B2C000C880B990B39
:10F270000E94C8DE9B01AC010E94AEE3811104C074
:10F28000B0920D0EA0920C0E80907113909072139C
:10F29000A0907313B0907413A5019401C501B4013B
:10F2A0000E94AEE3811132C08092C7049092C804DC
:10F2B000A092C904B092CA048091751390917613FC
:10F2C0009093C6048093C5042091B3043091B40494
:10F2D00090E080E028173907A4F1F70140AD51AD67
:10F2E00057FF0AC0FC01EE0FFF1FED54FB4F40819A
:10F2F0005181F70151AF40AF0196F2E0EF0EF11CE2
:10F30000E9CF0E9485E60FCF01E011CF8091C704BD
:10F310009091C804A091C904B091CA04809371135C
:10F3200090937213A0937313B093741383E090E0DF
:10F33000909376138093751390E080E00E9465B0FF
:10F34000C3CF6091051370910613809107139091BC
:10F3500008139B01AC010E94AEE381110FC06091C4
:10F36000091370910A1380910B1390910C139B0158
:10F37000AC010E94AEE3882309F4BDC40E94A06BD7
:10F380004FE2A42E43E1B42E54EEE52E5DE0F52EBF
:10F390006CE0862E6EE0962EF501419051906190C2
:10F3A00071905F01A3019201C301B2010E94AEE31B
:10F3B000811105C0F7014082518262827382F4E0BC
:10F3C000EF0EF11C8E149F0439F781E090E00E944B
:10F3D000FC100EE8010F013009F431C51E3609F4A6
:10F3E0002DC58091E1129091E212A091E312B091AB
:10F3F000E41285369105A105B1050CF420C5809174
:10F400005713909158138D7F892B41F440E855E2B2
:10F4100060E070E08BE99FE00E944F1680915713E7
:10F4200090915813019741F440E052EC61E070E094
:10F430008BE99FE00E944F1664E670E080E090E068
:10F440000E94FF6C8091571390915813892B09F0FB
:10F45000B7C01E3671F08091E1129091E212A09136
:10F46000E312B091E41285369105A105B1050CF0C7
:10F47000A7C061E37CE0CE0107960E94C3C862E4A6
:10F4800079E0CE0101960E94C3C86EEF75E1CE010E
:10F4900001960E9434C7BC01CE0107960E94FBC7AB
:10F4A000CE0101960E9457C8BE01695F7F4F8BE96C
:10F4B0009FE00E9452D168EB7BE080E090E00E94E8
:10F4C000FF6CBE01695F7F4FCE0101960E94BAC8F2
:10F4D000CE0101960E94291FCE0101960E9457C8B5
:10F4E0006CE271E080E090E00E94FF6C40910216B7
:10F4F00050910316425051096EEF75E1CE0101960D
:10F500000E945418BE016F5F7F4FCE0107960E9484
:10F5100012C8CE0101960E9457C8BE01695F7F4F95
:10F52000CE0101960E94BAC8BE01695F7F4FCE012D
:10F5300001960E9434C7BC01CE0107960E94FBC70A
:10F54000CE0101960E9457C86AE479E0CE01019687
:10F550000E94C3C8BE01695F7F4FCE0101960E9421
:10F5600034C7BC01CE0107960E94FBC7CE010196AD
:10F570000E9457C8BE01695F7F4F8BE99FE00E94E0
:10F5800052D168EB7BE080E090E00E94FF6CBE010E
:10F59000695F7F4FCE0101960E94BAC8CE010196E5
:10F5A0000E94291FCE0101960E9457C86CE271E0AB
:10F5B00080E090E00E94FF6CCE0107960E9457C841
:10F5C000113659F082E791E10E94A1A9D82E64E694
:10F5D00070E080E090E00E94FF6C0E9417C2F12C66
:10F5E000E12C17E2812F0E94DFAC89EC94E10E94AC
:10F5F0008873811124C510931A164FEFE41AF40A88
:10F600001F5F103479F7EF2831F46CE679E082E778
:10F6100091E10E9423CB10911A1681E6D8120DC0F9
:10F6200067E77CE182E791E10E9472D140E150E01E
:10F63000612F82E791E10E940CCB8091771390912A
:10F640007813019729F4103319F487E280931A167E
:10F650000E9430C580E40E94E9AC0BEA14E093EB11
:10F66000E92E94E0F92EF80161918F0186E196E18F
:10F670000E94BD73E016F106B1F70E9457130E9475
:10F68000C01069E67CE1CE0101960E94B1C84AE053
:10F6900050E06FEF7FEFCE0101960E94151ACE0168
:10F6A00001960E9457C80E9417C264E670E080E08D
:10F6B00090E00E94FF6CF1E6DF12D2C481E00E946C
:10F6C000171C81E00E94442164E670E080E090E035
:10F6D0000E94FF6C6091691370916A1380916B13A3
:10F6E00090916C136093C70D7093C80D8093C90DF2
:10F6F0009093CA0D00916D1310916E1320916F13AA
:10F70000309170130093C30D1093C40D2093C50D59
:10F710003093C60D9B01AC010E94AEE3882381F0BB
:10F7200083E393EFACE8B4E48093C70D9093C80DE6
:10F73000A093C90DB093CA0D90E080E00E9465B01F
:10F740006091C30D7091C40D8091C50D9091C60D4F
:10F750009B01AC010E94AEE38823C1F080E090E001
:10F76000A8ECB1E48093C30D9093C40DA093C50D94
:10F77000B093C60D80936D1390936E13A0936F1387
:10F78000B093701390E080E00E9465B0F89482E03E
:10F790008093B0008093B10094E69093B3001092F0
:10F7A000B20080937000789480930F12109212121E
:10F7B0008091101260E00E94776C69E57CE1CE01D7
:10F7C00001960E94B1C84AE050E06FEF7FEFCE0192
:10F7D00001960E94151ACE0101960E9457C861E356
:10F7E0007CE08EE894E10E949AC580915713909135
:10F7F0005813892B31F469E276E08EE894E10E9497
:10F800009AC58091571390915813019731F463E290
:10F8100076E08EE894E10E949AC58091571390910A
:10F820005813029731F46DE276E08EE894E10E947D
:10F830009AC58091921490919314892BC1F06EEF28
:10F8400075E18EE894E10E94CFC76EE874E1CE01C5
:10F8500001960E94BAC84AE050E06FEF7FEFCE01F8
:10F8600001960E947B13CE0101960E9457C8809199
:10F87000571390915813019709F05CC0CE01079679
:10F880000E9469498B859C85009709F449C0EF81E6
:10F89000F8852081222309F443C0079708F440C06B
:10F8A00066E47CE18EE894E10E94D6C7BE01695F00
:10F8B0007F4F8EE894E10E94CFC76EE874E1CE01DD
:10F8C00001960E94BAC8CE0101960E942313CE0170
:10F8D00001960E9457C86DE37CE1CE0101960E941B
:10F8E000B1C848EC50E06FEF7FEFCE0101960E9467
:10F8F0005C19CE0101960E9457C8BE01695F7F4F17
:10F90000CE0101960E94BAC848EC50E06FEF7FEF3D
:10F91000CE0101960E947B13CE0101960E9457C82A
:10F9200068EE73E080E090E00E94FF6CCE010796E5
:10F930000E9457C861E27CE18EE894E10E94D6C73C
:10F9400068E379E0CE0101960E94C3C86EEF75E1CD
:10F95000CE0101960E9434C76EE874E10E9434C75C
:10F96000BC018EE894E10E94FBC7CE0101960E9483
:10F9700057C86EE874E1CE0101960E94BAC8CE0164
:10F9800001960E942313CE0101960E9457C861E39D
:10F990007CE08EE894E10E949AC564E670E080E025
:10F9A00090E00E94FF6C83E090E09093E30D8093E1
:10F9B000E20D8CE40E94FAB06B017C0162E370E01E
:10F9C00080E090E00E94FF6CA7019601C701B6019C
:10F9D0000E94AEE38823B9F086E60E94FAB06B017C
:10F9E0007C0162E370E080E090E00E94FF6CA70180
:10F9F0009601C701B6010E94AEE3882321F0109260
:10FA0000E30D1092E20D8091E20D9091E30D0397CA
:10FA100009F02BC36CE07CE1CE0101960E94B1C8D5
:10FA2000CE0101960E94291FCE0101960E9457C85F
:10FA300083E08093B2140E9417C280ED0E94BBB194
:10FA4000853509F035C38AEA0E94DEB19093B4147B
:10FA50008093B3148CEA0E94DEB19093B614809325
:10FA6000B5148EEA0E94DEB19093B8148093B71457
:10FA700080EB0E94DEB19093C4148093C31482EB98
:10FA80000E94DEB19093C6148093C51484EB0E944B
:10FA9000DEB19093C8148093C71486EB0E94DEB148
:10FAA0009093BA148093B91488EB0E94DEB19093BE
:10FAB000BC148093BB148AEB0E94DEB19093BE14F9
:10FAC0008093BD148CEB0E94DEB19093C0148093A0
:10FAD000BF148EEB0E94DEB19093C2148093C114C8
:10FAE00063ED7BE18EE894E10E94D6C70E9423B2C9
:10FAF0000E94C8DE0E94ECE10E94C8DE20E030E0F7
:10FB000048EC52E40E9440E1AB01BC0122E0CE018E
:10FB100001960E945FC8BE016F5F7F4FCE010796BE
:10FB20000E94BAC863EC79E0CE0107960E941EC716
:10FB3000BC018EE894E10E94CFC7CE0107960E94D7
:10FB400057C8CE0101960E9457C86EE874E1CE01F5
:10FB500001960E94BAC8CE0101960E94291FCE01CB
:10FB600001960E9457C86DEB7BE18EE894E10E94FC
:10FB7000D6C76091EB047091EC048091ED049091F4
:10FB8000EE040E94C8DE20E030E048EC52E40E941F
:10FB900040E1AB01BC0122E0CE0101960E945FC8AA
:10FBA000BE016F5F7F4FCE0107960E94BAC863EC1B
:10FBB00079E0CE0107960E941EC7BC018EE894E151
:10FBC0000E94CFC7CE0107960E9457C8CE0101966A
:10FBD0000E9457C86EE874E1CE0101960E94BAC82F
:10FBE000CE0101960E94291FCE0101960E9457C89E
:10FBF00064E670E080E090E00E94FF6C8091E20D8E
:10FC00009091E30D892BA1F461E08091A6040E94FC
:10FC1000776C60E08091A4040E94776C6091A004EE
:10FC20007091A1048091A2049091A3040E94A3105A
:10FC300060E08091A6040E94776C8091EF04882395
:10FC400031F068EE73E080E090E00E94FF6C60E9C4
:10FC50007BE08AE994E10E949AC582E090E090936B
:10FC6000E10D8093E00D8091EF04882309F471C3C6
:10FC700063E87BE1CE0101960E94B1C84CE251E0FD
:10FC80006FEF7FEFCE0101960E947B13CE010196AC
:10FC90000E9457C860919E0470919F048091F00467
:10FCA0009091F1040E940E1484E1C82ED12CE12C15
:10FCB000F12C10E000E00F5F1F4FC701B6010E945A
:10FCC000FF6C60919E0470919F048091F00490916C
:10FCD000F1040E940E14033011053CF00A301105A6
:10FCE0000CF0F7C1892B09F4F7C144E1C40ED11C13
:10FCF000E11CF11CE0CFC0900D136C2D0C2C000CFE
:10FD0000770B880B990B0E94C8DE9B01AC010E9407
:10FD1000AEE3811133CBE0900E13F0900F13B701D7
:10FD20000F2C000C880B990B0E94C8DE9B01AC01C4
:10FD30000E94AEE3811122CB00911013602F002EA0
:10FD4000000C770B880B990B0E94C8DE9B01AC015D
:10FD50000E94AEE3811112CB809011139090121388
:10FD6000A0901313B0901413A5019401C501B40120
:10FD70000E94AEE3811102CB6091151370911613AE
:10FD800080911713909118139B01AC010E94AEE370
:10FD90008111F4CA60912B1370912C1380912D1353
:10FDA00090912E139B01AC010E94AEE38111E6CA33
:10FDB0006091571370915813072E000C880B990B04
:10FDC0000E94C8DE9B01AC010E94AEE38111D6CA3D
:10FDD0006091591370915A13072E000C880B990BE0
:10FDE0000E94C8DE9B01AC010E94AEE38111C6CA2D
:10FDF0006091671370916813072E000C880B990BA4
:10FE00000E94C8DE9B01AC010E94AEE38111B6CA1C
:10FE100043E04C150CF4B2CA05300CF0AFCA8BEFBE
:10FE2000E816F1040CF0AACA20E030E0A901C501EF
:10FE3000B4010E94C1DE87FDA1CAA2CA0CEF809165
:10FE4000EB049091EC04A091ED04B091EE0480934A
:10FE5000E1129093E212A093E312B093E412809126
:10FE6000E7049091E804A091E904B091EA0480933A
:10FE7000E5129093E612A093E712B093E8128091F6
:10FE8000E3049091E404A091E504B091E60480932A
:10FE9000E9129093EA12A093EB12B093EC1213378D
:10FEA00051F160E084E096E10E94A2C760E08EEF2D
:10FEB00095E10E94A2C7409108165091091641157C
:10FEC000510549F08DEF92E1009729F0BC0184E0E3
:10FED00096E10E948FB04091021650910316411591
:10FEE000510549F08BE593E1009729F0BC018EEFB5
:10FEF00095E10E948FB08091DF049091E004A09181
:10FF0000E104B091E2048093ED129093EE12A0937D
:10FF1000EF12B093F0128091DB049091DC04A09179
:10FF2000DD04B091DE048093F1129093F212A0935D
:10FF3000F312B093F4128091D7049091D804A09159
:10FF4000D904B091DA048093F5129093F612A0933D
:10FF5000F712B093F8128091D3049091D404A09139
:10FF6000D504B091D6048093F9129093FA12A0931D
:10FF7000FB12B093FC1290E080E00E9465B0E4EECA
:10FF8000FDE0AFE2B3E141915191619171914D93E7
:10FF90005D936D937D934EE0EC30F407A1F766E836
:10FFA0007CE1CE0101960E94B1C8CE0101960E946B
:10FFB000291FCE0101960E9457C823EBA22E24E0F0
:10FFC000B22E39E1832E33E1932EF12CE12C809176
:10FFD000B3049091B4048E159F054CF1F501819105
:10FFE00091915F01F401819391934F0180916E0E85
:10FFF0008823C9F068E379E082E791E10E947CCC34
:020000021000EC
:100000004AE050E0B70182E791E10E942FCC6DE316
:1000100079E082E791E10E947CCCF5013297808102
:1000200091810E9469CCFFEFEF1AFF0AD0CF023016
:1000300008F0E5C990E080E00E9465B0E0C9843036
:1000400009F0DECA61E579E082E791E10E947CCCAB
:1000500040E150E0612F82E791E10E940CCBD0CAD1
:1000600080E00E94171C80E02DCB86E00E942EC20B
:10007000BC0190E080E00E94C6DE2AE037ED43EA52
:100080005CE30E9427DF23E333E948E853E40E945E
:1000900061E020E030E048E453E40E94C1DE87FFE5
:1000A000C7CC82E090E09093AA048093A904C0CCCE
:1000B00066EE7BE1CE0101960E94B1C8CE010196A9
:1000C0000E942313CE0101960E9457C81092A804E3
:1000D0008FCD892B09F0EBC18091F0049091F10450
:1000E0008B30910509F093C18091251590912615CB
:1000F000A0912715B09128158093DC0D9093DD0D0C
:10010000A093DE0DB093DF0D809121159091221503
:10011000A0912315B09124158093D80D9093D90DFB
:10012000A093DA0DB093DB0D4091DC0D5091DD0D05
:100130006091DE0D7091DF0D21E0CE0101960E94ED
:100140005FC86DEB76E0CE0107960E94C3C8BE0182
:100150006F5F7F4FCE0107960E9434C7BC018EE8C7
:1001600094E10E94FBC7CE0107960E9457C8CE01BA
:1001700001960E9457C84091D80D5091D90D6091B9
:10018000DA0D7091DB0D21E0CE0101960E945FC86F
:100190006DE778E0CE0107960E94C3C8BE016F5F8D
:1001A0007F4FCE0107960E9434C7BC018EE894E1D0
:1001B0000E94CFC7CE0107960E9457C8CE01019674
:1001C0000E9457C865E578E08EE894E10E94C5C7B3
:1001D00061E37CE0CE0101960E94C3C844E150E097
:1001E00070E060E0CE0101960E94151ACE010196E2
:1001F0000E9457C8C090DC0DD090DD0DE090DE0D60
:10020000F090DF0D20E030E0A901C701B6010E94A7
:1002100049E220E030E040E05FE387FD18C1C7011C
:10022000B6010E9462E00E94ECE1AB01BC01CE018C
:1002300001960E94A4C5BE016F5F7F4F88E894E1DC
:100240000E9412C8CE0101960E9457C860E087E064
:100250000E94FAAC68E874E186E196E10E9452D10E
:100260006FED86E196E10E9435CB63E878E086E1A8
:1002700096E10E947CCC6091D80D7091D90D80914F
:10028000DA0D9091DB0D0E94ECE14AE050E086E14E
:1002900096E10E942FCC65E578E086E196E10E9428
:1002A0007CCC64E670E080E090E00E94FF6CC0903F
:1002B000DC0DD090DD0DE090DE0DF090DF0D20E044
:1002C00030E040EF51E4C701B6010E9449E264E723
:1002D0007BE187FF28C020E030E040ED51E4C7011A
:1002E000B6010E9449E287FDB7C064E67BE1CE011A
:1002F00001960E94B1C84AE050E06FEF7FEFCE0157
:1003000001960E947B13CE0101960E9457C88091EE
:10031000EF04882331F06CED75E080E090E00E94FE
:10032000FF6C64E57BE1CE0101960E94B1C84AE012
:1003300050E06FEF7FEFCE0101960E947B13CE015C
:1003400001960E9457C862E370E080E090E00E944E
:10035000FF6C65EA7BE18EE894E10E94D6C768E312
:1003600079E0CE0101960E94C3C86EEF75E1CE011F
:1003700001960E9434C76EE874E10E9434C7BC0144
:100380008EE894E10E94FBC7CE0101960E9457C8F7
:100390006EE874E1CE0101960E94BAC8CE010196C2
:1003A0000E942313CE0101960E9457C861E97BE1A8
:1003B0008EE894E10E94D6C76EE874E1CE01019602
:1003C0000E94BAC8CE0101960E942313CE01019665
:1003D0000E9457C861E37CE08EE894E10E949AC5D0
:1003E00062960FB6F894DEBF0FBECDBFDF91CF91FE
:1003F0001F910F91FF90EF90DF90CF90BF90AF9043
:100400009F908F907F906F905F904F90089586316E
:10041000910509F469CE0C9709F086CE8091CF0D35
:100420009091D00DA091D10DB091D20D8093DC0DA3
:100430009093DD0DA093DE0DB093DF0D8091CB0D79
:100440009091CC0DA091CD0DB091CE0D65CEC70190
:10045000B6010E9461E0E7CE20E030E040EB51E4DD
:10046000C701B6010E9449E266E47BE187FF5BCFEA
:1004700067E37BE1CE0101960E94B1C84AE050E0FB
:100480006FEF7FEFCE0101960E947B13CE010196A4
:100490000E9457C88091EF04882331F06CED75E01D
:1004A00080E090E00E94FF6C69E27BE13CCF0E941B
:1004B00057136EE170E080E090E00E94FF6C0E94B4
:1004C000EAB36B017C0164E670E080E090E00E949A
:1004D000FF6C6DEB76E08EE894E10E949AC521E016
:1004E000B701A601CE0101960E945FC8BE016F5FF1
:1004F0007F4F8EE894E10E94CFC7CE0101960E9403
:1005000057C86EE874E1CE0101960E94BAC84AE06D
:1005100050E070E060E0CE0101960E94151ACE0115
:1005200001960E9457C880919D04882379F080919C
:10053000FB04882359F06FED86E196E10E9435CBEC
:1005400062E079E086E196E10E947CCC65EE76E09F
:100550008EE894E10E94C5C7C092DC0DD092DD0DFB
:10056000E092DE0DF092DF0D20E030E040EF51E44C
:10057000C701B6010E9449E269E17BE187FF28C01B
:1005800020E030E040ED51E4C701B6010E9449E2AD
:1005900087FD3EC069E07BE1CE0101960E94B1C8B3
:1005A0004AE050E06FEF7FEFCE0101960E947B138F
:1005B000CE0101960E9457C88091EF04882331F044
:1005C0006CED75E080E090E00E94FF6C69EF7AE1ED
:1005D000CE0101960E94B1C84AE050E06FEF7FEF74
:1005E000CE0101960E947B13CE0101960E9457C84E
:1005F0006CE271E080E090E00E94FF6C8091EF047B
:10060000882309F4A6CE68EE73E080E090E09FCEE8
:1006100020E030E040EB51E4C701B6010E9449E21E
:100620006BEE7AE187FFD4CF6CED7AE1CE010196D3
:100630000E94B1C84AE050E06FEF7FEFCE01019613
:100640000E947B13CE0101960E9457C88091EF044F
:10065000882331F06CED75E080E090E00E94FF6C43
:100660006EEC7AE1B5CFBF92CF92DF92EF92FF921C
:100670000F931F93CF93DF93CDB7DEB762970FB67B
:10068000F894DEBF0FBECDBF8C016B0161E37CE04F
:100690000E94C3C810928B0D61E37CE0CE010D96E1
:1006A0000E94C3C8FF24F39482E791E10E94C3A98A
:1006B00020918B0D181619067CF521112DC082E7AB
:1006C00091E10E94A1A98A3009F07FC089899A89A5
:1006D000892B09F482C0F0928B0D62E879E0CE019B
:1006E00007960E94C3C8BE01635F7F4FCE01079685
:1006F0000E9434C7BC01CE0101960E94BAC8CE0147
:1007000001960E94291FCE0101960E9457C8CE0172
:1007100007960E9457C861C0F12CE12CBB24B3940A
:10072000222309F461C089899A89019709F045C09B
:1007300065E577E0CE0101960E94C3C8BE016F5FF8
:100740007F4FCE010D960E9403C7F12C811115C079
:1007500067E079E0CE0107960E94C3C8BE01695FD9
:100760007F4FCE010D960E9403C7FF24F3948111A1
:10077000F12CCE0107960E9457C8CE0101960E9427
:1007800057C8FF20A1F050E040E0BE01635F7F4FFB
:10079000CE0101960E945418BE016F5F7F4F8AE917
:1007A00094E10E9412C8CE0101960E9457C864E1EC
:1007B00070E080E090E00E94FF6CBE01635F7F4FBD
:1007C000CE0101960E94A8C891C08D3009F47ECF59
:1007D000682FCE010D960E94A2C76AE070E080E00B
:1007E00090E00E94FF6C60CF8BE99FE00E94C3A95C
:1007F0001816190614F58BE99FE00E94A1A98A300A
:10080000A9F08D3099F090918B0D91110FC0682F48
:10081000CE010D960E94A2C78FEFE81AF80A65E094
:1008200070E080E090E00E94FF6CDECF89899A89B9
:10083000892BA9F3B0928B0DF2CF64E170E080E0D8
:1008400090E00E94FF6CEF28D1F189899A89892B69
:10085000B1F180916E0E882361F168E379E0CE01F9
:1008600001960E94C3C8BE016F5F7F4FCE010D96F7
:100870000E9403C7F82ECE0101960E9457C8F110BE
:1008800018C06BE879E082E791E10E947CCCBE0160
:10089000635F7F4FCE0101960E94BAC8BE016F5FB1
:1008A0007F4F82E791E10E9460D1CE0101960E94C4
:1008B00057C864E170E080E090E00E94FF6C898995
:1008C0009A8920918B0D211130CF009709F02DCFFF
:1008D00064E670E080E090E00E94FF6C0E94326D60
:1008E00061E37CE0CE0101960E94C3C8CE010D9663
:1008F0000E9457C8BE016F5F7F4FC8010E944BC85E
:10090000CE0101960E9457C8F80184819581892BF8
:1009100079F4B601CE0101960E946A69BE016F5F4B
:100920007F4FC8010E944BC8CE0101960E9457C854
:10093000F80184819581892B79F4B601CE01019665
:100940000E940268BE016F5F7F4FC8010E944BC8C2
:10095000CE0101960E9457C8C80162960FB6F8945E
:10096000DEBF0FBECDBFDF91CF911F910F91FF90E2
:10097000EF90DF90CF90BF9008954F925F926F926B
:100980007F929F92AF92BF92CF92DF92EF92FF92AF
:100990000F931F93CF93DF93CDB7DEB7A8970FB612
:1009A000F894DEBF0FBECDBFBC0186EA94E10E9481
:1009B000FBC70E9456C46FEB79E0CE0101960E94FE
:1009C000C3C8BE016F5F7F4F86EA94E10E9403C7F0
:1009D000182FCE0101960E9457C8112309F4F8C0C0
:1009E0008091B0149091B1144097C0F0F12C8F2DEC
:1009F000A8960FB6F894DEBF0FBECDBFDF91CF91A2
:100A00001F910F91FF90EF90DF90CF90BF90AF902C
:100A10009F907F906F905F904F90089542E050E0DC
:100A20006CEA74E1CE0101960E945418BE016F5F1A
:100A30007F4F88E894E10E9412C8CE0101960E947F
:100A400057C868E874E1CE0101960E94BAC8CE0189
:100A500001960E94291FCE0101960E9457C888E87E
:100A600094E10E940CC620E030E048EC52E40E9481
:100A700027DF0E94ECE1AB01BC014093EB045093F3
:100A8000EC046093ED047093EE04CE0101960E9495
:100A9000A4C5CE0101960E94291FCE0101960E9495
:100AA00057C86091EB047091EC048091ED04909133
:100AB000EE048B019C0100591F452140310901348E
:100AC0001C4921053105C8F162E979E0CE010196A2
:100AD0000E94C3C868E874E1CE0101960E9434C741
:100AE00065EA79E00E941EC7BC018EE894E10E948D
:100AF000FBC7CE0101960E9457C868E379E0CE019A
:100B000001960E94C3C86EE874E1CE0101960E946E
:100B100034C7BC01CE0145960E94BAC8CE014596A5
:100B20000E942313CE0145960E9457C8CE0101961C
:100B30000E9457C81092000548C21A821982FE010D
:100B4000339626E0DF011D922A95E9F70E94C8DE60
:100B500020E030E048EC52E40E9440E18E010F5F5B
:100B60001F4F22E047E00E941DDABC018EE894E1AD
:100B70000E94FDC565EB79E0CE0145960E94C3C891
:100B80006EE874E1CE0145960E9434C762EC79E0CC
:100B90000E941EC7BC018EE894E10E94FBC7CE01F3
:100BA00045960E9457C88091EB049091EC04A09167
:100BB000ED04B091EE048093E1129093E212A093C1
:100BC000E312B093E41290E080E00E9465B095CF0C
:100BD0008E010B5E1F4F65E979E1C8010E94B1C823
:100BE000B80186EA94E10E9403C7FF24F3948111BF
:100BF00016C060E979E1CE0101960E94B1C8BE013C
:100C00006F5F7F4F86EA94E10E9403C7FF24F3944D
:100C1000811101C0F12CCE0101960E9457C8C80174
:100C20000E9457C8FF2009F471C042E050E06CEA0E
:100C300074E1CE0101960E945418BE016F5F7F4F90
:100C400088E894E10E9412C8CE0101960E9457C81C
:100C50006BE879E1CE0101960E94B1C8BE016F5FD9
:100C60007F4F86EA94E10E9403C7E82ECE010196E9
:100C70000E9457C8EE2099F044E050E06CEA74E11D
:100C8000CE0101960E945418BE016F5F7F4F88E825
:100C900094E10E9412C8CE0101960E9457C888E8CC
:100CA00094E10E9417C66730710558F570930D0ED8
:100CB00060930C0E80910C0E90910D0E9093681322
:100CC0008093671390E080E00E9465B068E379E06C
:100CD000CE0101960E94C3C86EE874E1CE01019670
:100CE0000E9434C7BC01C8010E94BAC8C8010E9452
:100CF0002313C8010E9457C8CE0101960E9457C80D
:100D000076CE10920D0E10920C0ED4CF66E879E1DB
:100D1000CE0101960E94B1C8BE016F5F7F4F86EA87
:100D200094E10E9403C7F82ECE0101960E9457C895
:100D3000FF20A1F126E030E044E050E06CEA74E1ED
:100D4000CE0101960E94D4C8BE016F5F7F4F88E834
:100D500094E10E9412C8CE0101960E9457C888E80B
:100D600094E10E9417C670935A13609359137093BD
:100D7000F1046093F0046CEA74E1CE0101960E94E4
:100D8000BAC8CE0101960E94291FCE0101960E9489
:100D900057C890E080E00E9465B0CCCE6FE779E163
:100DA000CE0101960E94B1C8BE016F5F7F4F86EAF7
:100DB00094E10E9403C7F82ECE0101960E9457C805
:100DC000FF20A1F146E050E06CEA74E1CE0101960B
:100DD0000E945418BE016F5F7F4F88E894E10E9423
:100DE00012C8CE0101960E9457C880918C14909130
:100DF0008D14892B61F088E894E10E940CC6609301
:100E0000A0047093A1048093A2049093A3046CEABD
:100E100074E1CE0101960E94BAC8CE0101960E94EB
:100E2000291FCE0101960E9457C884CE67EC79E055
:100E3000CE0101960E94C3C8BE016F5F7F4F86EA54
:100E400094E10E9403C7F82ECE0101960E9457C874
:100E5000FF2009F4BDC06BE779E1CE0101960E9445
:100E6000B1C8BE016F5F7F4F86EA94E10E9403C75D
:100E7000F82ECE0101960E9457C8FF20D1F184E0E0
:100E800090E00E9447106093CF047093D004809349
:100E9000D1049093D2046BE679E18EE894E10E944C
:100EA000D6C74091CF045091D0046091D104709185
:100EB000D20422E0CE0101960E945FC8BE016F5F9E
:100EC0007F4F8EE894E10E94CFC7CE0101960E9429
:100ED00057C88091CF049091D004A091D104B091D3
:100EE000D2048093051390930613A0930713B09335
:100EF00008136AEC79E0CE0101960E94C3C8BE01D6
:100F00006F5F7F4F86EA94E10E9403C7F82ECE01FF
:100F100001960E9457C8FF20F1F18AE090E00E94FC
:100F200047106093CB047093CC048093CD049093CE
:100F3000CE046AE579E18EE894E10E94D6C740913B
:100F4000CB045091CC046091CD047091CE0422E08A
:100F5000CE0101960E945FC8BE016F5F7F4F8EE891
:100F600094E10E94CFC7CE0101960E9457C880919C
:100F7000CB049091CC04A091CD04B091CE04809389
:100F8000091390930A13A0930B13B0930C1390E0E2
:100F900080E00E9465B068E379E0CE0101960E948E
:100FA000C3C86EE874E1CE0101960E9434C7BC014B
:100FB000C8010E94BAC8C8010E942313C8010E9438
:100FC00057C8CE0101960E9457C8FF24F3940FCD55
:100FD00061ED78E0CE0101960E94C3C8BE016F5F4B
:100FE0007F4F86EA94E10E9403C7F82ECE01019656
:100FF0000E9457C8FF2009F4BDC08091B0149091A1
:10100000B1140797F8F046E050E06CEA74E1CE01C5
:1010100001960E945418BE016F5F7F4F88E894E1EB
:101020000E9412C8CE0101960E9457C888E894E138
:101030000E940CC66093F6047093F7048093F80442
:101040009093F904809193049091940499270E94BD
:101050000A122DE038E643E55BE30E9427DF6B01CF
:101060007C012091190530911A0540911B05509182
:101070001C050E94C1DE18160CF460C060910105C9
:1010800070910205809103059091040520E030E005
:1010900048EC52E40E9427DF6B017C0120E030E045
:1010A000A9010E94C1DE181634F0C12CD12CF8EA37
:1010B000EF2EF1E4FF2EC092F604D092F704E092F6
:1010C000F804F092F904C0921513D0921613E0922E
:1010D0001713F092181380916E0E882381F068E444
:1010E00079E182E791E10E9472D16091F6047091FA
:1010F000F7048091F8049091F9040E9420CC90E0CC
:1011000080E00E9465B06EE379E18EE894E10E9490
:10111000D6C74091F6045091F7046091F80470919D
:10112000F90422E0CE0101960E945FC8BE016F5F04
:101130007F4F8EE894E10E94CFC7A6C020912D0575
:1011400030912E0540912F0550913005C701B60111
:101150000E9449E287FF05C0C701B6010E9433AF74
:1011600095CF6091150570911605809117059091A6
:1011700018058CCF6AE379E1CE0101960E94B1C8CF
:10118000BE016F5F7F4F86EA94E10E9403C7F82E8D
:10119000CE0101960E9457C8FF2009F47DC07090CF
:1011A000910460E0872D0E94776CE9E1AE2EB12CAE
:1011B000C12CD12C7601872D0E94B76CBC01990FF0
:1011C000880B990B0E94C8DE9B01AC01C701B601D8
:1011D0000E9462E06B017C016AE070E080E090E0D8
:1011E0000E94FF6CB1E0AB1AB10829F720E030E0B3
:1011F00040EA50E4C701B6010E9427DF20E030EC4E
:101200004FE754E40E9440E120E030E048EC51E434
:101210000E9440E16093F2047093F3048093F4041D
:101220009093F50460932B1370932C1380932D13DC
:1012300090932E1390E080E00E9465B067E279E120
:101240008EE894E10E94D6C74091F2045091F304D5
:101250006091F4047091F50422E0CE0101960E94A1
:101260005FC8BE016F5F7F4FC8010E94BAC862E2CB
:1012700078E0C8010E941EC7BC018EE894E10E947C
:10128000CFC7C8010E9457C8CE0101960E9457C817
:101290006EE874E10C942C9367ED78E0CE01019632
:1012A0000E94C3C8BE016F5F7F4F86EA94E10E942F
:1012B00003C7F82ECE0101960E9457C8FF2009F4FB
:1012C00041C080911013082E000C990B01970397D1
:1012D00090F589E390E00E940A122AE137E64CE992
:1012E00050E40E9427DF60931113709312138093D0
:1012F00013139093141390E080E00E9465B066E0B1
:1013000079E18EE894E10E94D6C740911113509183
:101310001213609113137091141322E0CE01019601
:101320000E945FC8BE016F5F7F4FC8010E94BAC8AC
:101330006FEC79E09ECF60EE78E18EE894E10E9458
:10134000D6C7A6CF6CED78E1CE0101960E94B1C858
:10135000BE016F5F7F4F86EA94E10E9403C7F82EBB
:10136000CE0101960E9457C8FF2009F439C126E03A
:1013700030E044E050E06CEA74E1CE0101960E9456
:10138000D4C8BE016F5F7F4F88E894E10E9412C805
:10139000CE0101960E9457C888E894E10E9417C6C2
:1013A0006B015B016BE176E0CE0101960E94C3C840
:1013B000BE016F5F7F4F8CEA94E10E94CDC6AC0105
:1013C0004F5F5F4F6CEA74E1C8010E945418B80186
:1013D00088E894E10E9412C8C8010E9457C8CE0153
:1013E00001960E9457C890908F0488E894E10E946B
:1013F0000CC62B013C0180916E0E8823B9F062E28D
:1014000075E182E791E10E9472D14AE050E0B601B5
:1014100082E791E10E942FCC6EE277E082E791E1D2
:101420000E947CCCC301B2010E9420CC692DC8016E
:101430000E94AD7018870F831D821E82198289E079
:101440008A8381E08B838C831C8A1B8ACE01019660
:101450000E940270CE0101960E94A56ECE010196F7
:101460000E94D3C20E8110E00B30110514F00AE087
:1014700010E0EBE5CE16D10408F44FC074EEC72E91
:101480007DE0D72E5601412C512C3201F12CE12C5C
:101490000E151F05B9F06E2DCE0101960E94966FB4
:1014A0009B01AC01D5012D933D934D935D935D015F
:1014B000C301B2010E9462E02B013C01BFEFEB1AB5
:1014C000FB0AE6CFB7010F2C000C880B990B0E948A
:1014D000C8DE9B01AC01C301B2010E9440E12B01B7
:1014E0003C0110E000E0E016F106B9F1F6012191AF
:1014F0003191419151916F015F01F4E0AF1AB10850
:10150000C301B2010E9461E0D5016D937D938D937B
:101510009C9313970F5F1F4FE6CF1A141B040CF018
:1015200040C00A151B050CF0860101501109602FFF
:10153000CE0101960E94966F9B01AC01000F111F16
:10154000000F111F0C51124FC301B2010E9461E044
:10155000F8016083718382839383E4EEFDE0AFE260
:10156000B3E18CE09EE041915191619171914D9375
:101570005D936D937D938E179F07A9F790E080E0B0
:101580000E9465B06BEB78E18EE894E10E94D6C7CB
:1015900044E050E06CEA74E1CE0101960E945418D8
:1015A000C5CDA114B104C9F634EEE32E3DE0F32E0F
:1015B0000A151B0591F26A2DCE0101960E94966FC5
:1015C0009B01AC01C301B2010E9461E0D7016D93A0
:1015D0007D938D939D937D01BFEFAB1ABB0AE8CF3E
:1015E00069E377E0CE0101960E94C3C8BE016F5F38
:1015F0007F4F86EA94E10E9403C7F82ECE01019640
:101600000E9457C8FF2009F416C127E030E046E0E9
:1016100050E06CEA74E1CE0101960E94D4C8BE018C
:101620006F5F7F4F88E894E10E9412C8CE01019657
:101630000E9457C888E894E10E9417C67B01609316
:1016400010138CEA94E10E9422C66EE277E0CE018C
:1016500001960E94C3C8BE016F5F7F4F8CEA94E180
:101660000E94CDC6AC014F5F5F4F6CEA74E1C801C8
:101670000E945418C8010E940CC660931113709305
:1016800012138093131390931413C8010E9457C828
:10169000CE0101960E9457C86AEA78E18EE894E18B
:1016A0000E94D6C7E4E0EE16F10404F5F2E0EF166E
:1016B000F1040CF098C0E114F10419F1EA94EF2858
:1016C00009F46AC060911013062E000C770BC80154
:1016D0000E94D1C56DED79E0CE0101960E94C3C88C
:1016E000B801CE0101960E9434C749C084E0E816D3
:1016F000F10441F769E878E18EE894E10E9447C778
:101700006DC020E030E0A9016091111370911213B7
:1017100080911313909114130E94C1DE181664F087
:1017200080E090E0A0E8BFE3809311139093121340
:10173000A0931313B093141320911113309112132B
:10174000409113135091141360E070E080EA90E42C
:101750000E9440E1AB01BC0122E0C8010E945FC8C9
:1017600062ED79E0CE0101960E94C3C8B801CE01B6
:1017700001960E9434C766EF77E00E941EC7BC0145
:101780008EE894E10E94CFC7CE0101960E9457C80F
:10179000C8010E9457C822C06CE978E18EE894E144
:1017A0000E9447C720E030E048E453E46091111301
:1017B0007091121380911313909114130E94C1DE43
:1017C000181664F080E090E4ACE1B5E48093111366
:1017D00090931213A0931313B093141390E080E02E
:1017E0000E9465B055CD60E978E18EE894E10E94F1
:1017F00047C78AE08E9DB0018F9D700D1124CE01E8
:1018000001960E94D1C5BE016F5F7F4FC8010E9443
:10181000BAC86FEE77E0C8010E941EC7BC018EE80F
:1018200094E10E94CFC7C8010E9457C8CE0101961B
:101830000E9457C8B7CF64EE79E0CE0101960E94AE
:10184000C3C8BE016F5F7F4F86EA94E10E9403C761
:10185000F82ECE0101960E9457C8FF2009F4C2C09D
:1018600027E030E046E050E06CEA74E1CE010196FA
:101870000E94D4C8BE016F5F7F4F88E894E10E9448
:1018800012C8CE0101960E9457C888E894E10E94D0
:1018900017C660930D138CEA94E10E9422C688E873
:1018A00094E10E9417C6611571058105910509F043
:1018B0006DC085E090E090930F1380930E1390E03D
:1018C00080E00E9465B068E778E18EE894E10E94CC
:1018D000D6C780910D1383302CF56DE678E18EE844
:1018E00094E10E9447C760910E1370910F13CE01CF
:1018F00001960E94D1C5BE016F5F7F4FC8010E9453
:10190000BAC868E077E0C8010E941EC7BC018EE833
:1019100094E10E94CFC7C8010E9457C8CE0101962A
:101920000E9457C880910D1383300CF4B1CC6091A4
:101930000E1370910F13CE0183960E94D1C5609152
:101940000D13062E000C770BC8010E94D1C56DED5A
:1019500079E0CE0101960E94C3C8B801CE0101967C
:101960000E9434C7BE016D5D7F4F0E9434C7BC0129
:101970008EE894E10E94CFC7CE0101960E9457C81D
:10198000C8010E9457C8CE01839680CC6130710592
:101990008105910519F489E190E08DCF6EE277E041
:1019A000CE0101960E94C3C8BE016F5F7F4F8CEAD3
:1019B00094E10E94CDC6AC014F5F5F4F6CEA74E1C9
:1019C000C8010E945418C8010E9417C670930F13D3
:1019D00060930E13C8010E9457C8CE0101960E9461
:1019E00057C86DCF6BEE79E0CE0101960E94C3C857
:1019F000BE016F5F7F4F86EA94E10E9403C7F82E15
:101A0000CE0101960E9457C8FF2009F464C080915E
:101A10008D0490918E040E94FC126093D304709305
:101A2000D4048093D5049093D6046093F9127093F4
:101A3000FA128093FB129093FC1280E090E5A3ECE5
:101A4000B7E48093DB049093DC04A093DD04B093AF
:101A5000DE048093F1129093F212A093F312B093EC
:101A6000F41280916E0E882381F06FE478E182E7B2
:101A700091E10E9472D16091D3047091D40480915D
:101A8000D5049091D6040E9420CC90E080E00E9482
:101A900065B04091D3045091D4046091D504709105
:101AA000D60422E0C8010E945FC86FEE79E0CE0143
:101AB00001960E94C3C8B801CE0101960E9434C7A6
:101AC000BC018EE894E10E94FBC7CE0101960E9402
:101AD00057C8C801DBCB6AEF79E0CE0101960E94BE
:101AE000C3C8BE016F5F7F4F86EA94E10E9403C7BF
:101AF000F82ECE0101960E9457C8FF2009F488C035
:101B00008091B0149091B1140497F8F044E050E043
:101B10006CEA74E1CE0101960E945418BE016F5F19
:101B20007F4F88E894E10E9412C8CE0101960E947E
:101B300057C888E894E10E940CC66093DF04709354
:101B4000E0048093E1049093E2048091DF0490919B
:101B5000E004A091E104B091E2048093ED1290932F
:101B6000EE12A093EF12B093F01280916E0E8823C4
:101B700091F066E378E182E791E10E9472D1609191
:101B8000DF047091E0048091E1049091E20442E06E
:101B900050E00E941ECC80918D0490918E040E9492
:101BA000FC126093D7047093D8048093D904909367
:101BB000DA046093F5127093F6128093F712909303
:101BC000F81280916E0E882381F06CE278E182E752
:101BD00091E10E9472D16091D7047091D8048091F4
:101BE000D9049091DA040E9420CC90E080E00E9419
:101BF00065B04091D7045091D8046091D904709198
:101C0000DA0422E0C8010E945FC86EEF79E04FCF8E
